:020000040800F2
:1040000000500020F9DA000809B600080BB60008D5
:104010000DB600080FB6000811B600080000000039
:1040200000000000000000000000000015B60008BD
:1040300013B600080000000017B60008D587000876
:1040400019B600081BB600081DB600081FB6000808
:1040500021B6000823B6000825B6000827B60008D8
:1040600029B600082BB600082DB600080000000095
:104070000000000000000000000000000000000040
:1040800000000000000000003DB600083FB6000838
:104090004DB600085DB600086DB600087DB6000894
:1040A0007FB6000881B6000883B6000885B6000810
:1040B00087B6000889B600088BB600088DB60008E0
:1040C0008FB6000891B6000893B6000895B60008B0
:1040D00097B60008758300083D8600089DB6000865
:1040E0009FB60008A1B60008A3B6000800000000B3
:1040F00000000000000000000000000000000000C0
:0C41000000000000000000005FF800005C
:1041100030BF704720BF704740BF7047BFF36F8FFD
:104120007047BFF34F8F7047BFF35F8F704701DF5A
:104130007047EFF31480704780F31488BFF36F8FDC
:104140007047EFF30980704780F309887047EFF3F9
:104150000880704780F30888704772B6704762B66F
:10416000704771B6704761B6704780F31188704729
:10417000EFF31280704740BA704700BA70470000F2
:104180002DE9FF41514E5248012108F0BDF80420AD
:10419000012108F0A1FB1024032542F2122330462E
:1041A0006946ADF800308DF803408DF8025008F0F4
:1041B0001CF8022334614FF004087361454F4FF43B
:1041C000444330466946ADF800308DF802508DF812
:1041D000038008F00AF80820012108F07DFB41F671
:1041E0001C7338466946ADF800308DF803408DF8F1
:1041F000025007F0FAFF4FF4F8533B610C237B6148
:104200003846E0236946ADF800308DF802508DF84D
:10421000038007F0EAFF2046012108F05DFB8DF8DE
:1042200003402D4C4FF4604320466946ADF8003002
:104230008DF8025007F0D9FF4FF4204323614FF46B
:10424000804363610121404608F052FB234808F097
:10425000C5FD0DEB080008F048FF00244FF6FF7382
:104260001E480DEB0801ADF80830ADF80440ADF87C
:104270000A40ADF8064008F015FE1848012108F084
:1042800058FF1748012108F03FF80A2223464FF44F
:1042900000517161B0683161B168400458BF0133A9
:1042A000490448BF0134013AF1D10A2B0D4B03D127
:1042B0000A2C01D1012200E00022054801211A70D8
:1042C00008F022F804B0BDE8F08100BF000801400A
:1042D00000023000000C01400010014000080040C6
:1042E00000043000CC0E0020134B82B01B7803B3C7
:1042F000124B4FF400725A614FF480721A6100221F
:10430000019201994AF69B52914202D8019A0132D8
:10431000F6E74FF400721A614FF480725A6100237D
:104320000193019A4AF69B539A42E1D8019B0133CB
:10433000F6E702B0704700BFCC0E0020000C014031
:1043400010B1012802D07047082200E00422014B7E
:104350005A617047000C014010B1012802D070472B
:10436000082200E00422014B1A617047000C014052
:1043700038B50546002445FA04F3DB07E0B202D560
:10438000FFF7EAFF01E0FFF7DBFF0134082CF2D171
:1043900038BD08B503281BD8DFE800F0020B101564
:1043A000002004F015FBB0F5006F94BF0020012041
:1043B00008BD084B9868C0F3801008BD054B98688D
:1043C000C0F3C01008BD034B9868C0F3401008BD8F
:1043D000002008BD000C014030B1012809D1064B76
:1043E000D868C0F380007047034BD868C0F3C000A2
:1043F00070470020704700BF000C014038B5002412
:104400002546E0B2FFF7C5FF18B10123A3401D43C5
:10441000EDB20134082CF4D1284638BD20B9034B45
:104420009868C0F3C0307047002070470008014012
:1044300010B9C90805F0D8B9704708B108F08AB8B2
:1044400008F090B862B6704772B6704718B9024B60
:104450004FF480625A617047000C014018B9024B5A
:104460004FF480621A617047000C0140034B4FF417
:10447000005208B11A6170475A617047001001403C
:10448000074B9A88C2F30722042A06D19A88D2B22F
:10449000892A02D1188980B270470020704700BF76
:1044A000006C0040034B4FF4804208B11A61704722
:1044B0005A61704700100140F8B51C4D0121284693
:1044C00009F05EF91A4C08B92068F8BD04F0E6F965
:1044D000FF2160600022032000F066FA01220646F8
:1044E000FF21032000F060FA4CF221530746AB8411
:1044F0002846012109F04AF947EA062010F0020394
:104500004FEA900018BF0123C204237203D5237A17
:1045100043F002032372830403D5237A43F0040398
:104520002372E36823EA00002060F8BD0008004021
:104530006805002070B5FFF7BFFF5C494C69086152
:10454000A04234DD8B69051B9D42594B0CDA1C6877
:10455000D1E908236C43121943EBE473C1E9082342
:104560008B6A1D448D6259E091F82C6072070CD55E
:10457000CC681A68041B624326F00406D317C1E90D
:1045800008238C6281F82C6033E0CE681B68241A03
:10459000344404FB0334D1E90823121B63EBE473B6
:1045A000C1E90823F6438B6A35442B4411E035DA20
:1045B0008B69221A9A423E4B0DDA1D68041B554343
:1045C000D1E90823521B63EBE573C1E908238B6A29
:1045D00023448B6222E091F82C506A070ED51A68AA
:1045E00025F004054243D317C1E90823886281F806
:1045F0002C5000220023C1E90C230FE0CA681D687B
:104600000132041B14446543D1E90823521943EBDA
:10461000E573C1E908238B6A1C448C628C6A8D6B3C
:10462000CA6B651B85EAE576A6EBE57696421F4BDD
:104630002ED95E681A6CB21A642A29D91E6442F215
:10464000107675435A6495FBF2F23C256A43DE68A6
:104650009C63013692FBF6F29A6440F6B834002A65
:10466000B8BF5242A24201DDC82203E0B2F57A7F10
:1046700002DD6422DA6316E0322A01DD0A22F9E75C
:104680000A2A01DD0522F5E7012A0CDD0122F1E706
:104690004C680A6C054BA21AB2F5FA6F03D90122D5
:1046A000DA6300229A64486170BD00BF680500208B
:1046B0000400002008B568B9FFF73CFF0649D1E9BE
:1046C0000823D1E90C01121A63EB0103100A40EA36
:1046D000036008BD002008BD6805002038B50D4600
:1046E000F8B9104CFFF726FFD4E90801E26800286A
:1046F00071F100034FEA022202DA404261EB41010C
:10470000D3170BF0D1FAC4E90C23E9170B022A02E4
:10471000D4E90C0143EA1563121843EB0103C4E921
:10472000082338BD6805002010B9024B0901196043
:10473000704700BF0400002010B9024B83F82C1012
:10474000704700BF68050020014B986C704700BFA0
:104750006805002010B9024B187A70470020704796
:104760006805002038B5214B214A1B69214C5909A5
:10477000090103F01F0311600320FE21002284F8C9
:104780002C3000F011F940210122032000F00CF937
:1047900000210A46032000F007F900210546012206
:1047A000032000F001F9082D05D140F6FF73E36006
:1047B0004FF4006304E040F2FF33E3604FF4007312
:1047C000E72100220320A36100F0EEF8002101227E
:1047D000032000F0E9F8FFF76FFE60610002C117E7
:1047E000C4E90C01C4E9080138BD00BF200F002056
:1047F000040000206805002008B5082004F0E8F84F
:104800005E2805D9074B93F84C2052B9012206E0E7
:10481000082004F0DDF8542803D8024B002283F866
:104820004C2008BD68050020044B93F84C0001386B
:1048300001288CBF00200120704700BF68050020C0
:10484000044B93F84C00012806BF022283F84C2049
:10485000002070476805002008B5FFF72DFE0528E9
:1048600008D9FFF729FE40F2F933984294BF00209F
:10487000012008BD012008BD2DE9F04F4FF4804014
:1048800089B0012108F034F8434C0120014608F0BA
:1048900023F803264FF420434FF0180A204602A9BC
:1048A000ADF808308DF80BA04FF0040B8DF80A60BE
:1048B00007F09BFC4FF48043204602A9ADF8083076
:1048C0008DF80A608DF80BB007F08FFC0823ADF867
:1048D0001830324B002401254FF482794FF0020842
:1048E0004FF40077184603A9ADF80C40ADF810401E
:1048F000ADF81A40ADF81C400193ADF80E90ADF83C
:104900001280ADF81450ADF8167008F09DF8019BB8
:104910002946184608F01EF929464FF4805007F042
:10492000DBFF2846214607F0EFFC8DF80BA0DFF8EF
:1049300074A0A023504602A9ADF808308DF80A6093
:1049400007F053FC4023504602A9ADF808308DF81B
:104950000A608DF80BB007F048FCADF80C40ADF8DC
:104960001040ADF81A40ADF81C400D4C1023204605
:1049700003A9ADF81830ADF80E90ADF81280ADF87F
:104980001450ADF8167008F05FF82046294608F07C
:10499000E1F809B0BDE8F08F000C0140003800409C
:1049A000003001400008014070B504460E4615462F
:1049B00003286AD8DFE800F002070A0E344B4FF4F0
:1049C00080525A6112E01022324B0DE04FF4006227
:1049D0002F4B09E0304A138823F002031B041B0C01
:1049E00013802E4B4FF400425A6110E02C480221F4
:1049F00008F034F90028F9D02948314608F0DAF8EF
:104A00002748012108F02AF90028F9D016E02248A9
:104A1000022108F023F90028F9D01F48314608F098
:104A2000C9F81D48012108F019F90028F9D0FDB195
:104A3000032C2AD8DFE804F003080B10F5B1144B5F
:104A40004FF480521A6119E01022124B02E0104B11
:104A50004FF400621A6113E0104B4FF400421A61E8
:104A600003F500531A8892B242F002021A8007E05E
:104A7000032C0AD8DFE804F002040404084800E02C
:104A8000054808F099F8C0B270BD002070BD00BFA5
:104A9000000C0140000801400030014000100140BE
:104AA0000038004037B5C44DA8786B782C4608B163
:104AB0000422E9E2A42B00F0378269D8852B00F0AC
:104AC0000F8127D8072B00F03F810FD8032B00F070
:104AD000078105D8012B00F0D48040F2C880DFE0C8
:104AE000052B00F0188140F2068120E1812B00F0B7
:104AF000C88009D80D2B00F04381802B00F0B780CF
:104B00000C2B40F0C0822BE1832B00F0F48040F2AC
:104B10004981C5E0952B00F071811FD88C2B00F0E6
:104B2000648110D8872B00F04481C0F0F4808A2B78
:104B300040F0A9820020142101AA06F095F8EB7834
:104B40008DF8063046E1932B00F01A8100F20881BF
:104B50008D2B40F0988200201A2125E1A02B00F037
:104B6000CF8109D8992B00F060819A2B00F08281C7
:104B7000962B40F0888250E1A22B00F0C78100F212
:104B8000CC81D5F803100020C9B204F0E9FC7DE225
:104B9000B62B00F0438236D8AC2B00F0108215D82B
:104BA000A82B00F0F88105D8A62B00F0DD8140F29B
:104BB000CB81E9E1AA2B00F0F48100F2F981D5F86C
:104BC00003100020C9B204F0A9FD5FE2B02B00F091
:104BD00011820BD8AE2B00F0FF8100F20482D5F8D1
:104BE00003100020C9B204F0EBFD4FE2B22B00F03D
:104BF0000E82C0F00582B52B40F04582D5F8032027
:104C00006E4B9A6142E2C82B00F04F8114D8C12B41
:104C100000F03D8108D8B82B00F01782C0F0078261
:104C2000C02B00F091802EE2C32B00F03981C0F040
:104C30003281C72B7BD026E2D42B00F044810DD8E3
:104C4000D12B00F00982D22B00F00C82CC2B40F04B
:104C50001A82D5F80320594BDA8117E2D62B00F0DF
:104C60003C81C0F03581FE2B00F03C810BE204F06A
:104C70004BFF20B9A178490101F0E0010BE00622C9
:104C800002E204F041FF0028F9D1A178490141F086
:104C9000020101F0E201D4F8032005F050FFF5E134
:104CA00004F032FF05460028E9D1A178D4F80320AA
:104CB000490141F0080101F0E80105F02EFFA1785B
:104CC000D4F80320490141F0060101F0E60128462D
:104CD000002AB8BF524205F020FFA378012117E057
:104CE00004F012FF0028CAD1A178490141F00A015D
:104CF00001F0EA0158E00621D4F80320002005F075
:104D00000CFFD4F80310A3782D4A42F82310002199
:104D10002C4AD154BAE1D4F80310002006F017F859
:104D2000A378D4F80310284A42F823109DE0274BBB
:104D300001221A70E178214B5972254B1B78022B06
:104D400040F0A48100207DE1204B01221A70E1781F
:104D50001A4B99721E4B1878002840F0978171E128
:104D600001AA0020142105F07FFFD4F803209DF84C
:104D7000053012B143F0020311E023F002030EE00C
:104D800001AA0020142105F06FFFD4F803209DF83C
:104D9000053012B143F0010301E023F001038DF867
:104DA000053017E000200421D4F8032005F0B5FEFB
:104DB0006CE100200E21F7E7200A0020200F0020E0
:104DC000A40E0020B8050020A00A0020840F0020B7
:104DD000870F0020A1780020490141F0140101F063
:104DE000F40101AA05F074FE50E1E978A84BD972EC
:104DF000C1F10801C9B204F099FB47E101AA1421ED
:104E000005F032FFD5F803209DF8053012B143F0CC
:104E10000403C4E723F00403C1E7D5F803209D4B46
:104E2000002A00F0328101222FE101AA002018217E
:104E300005F01AFFEA789DF8053002F00F0223F022
:104E40000F031343A1780020490141F0180101F03C
:104E5000F80101AA8DF8053005F03AFE8E4BA078D6
:104E600053F8201005F073FFA3788C4A13440022F6
:104E70005A700BE101AA0020182105F0F5FE9DF8FB
:104E80000530EA7803F00F0343EA0213DAE7EA7821
:104E90007F4B1A72FAE0D5F803207D4B1A60F5E0DB
:104EA000D5F803207A4B5A60F0E07D4B01221A704E
:104EB000774BD5F80320DA777A4B1B78032B40F039
:104EC000E580E978BEE0D5F80320714B5A61DDE05A
:104ED000D5F803206E4B9A77D8E0D5F803206C4BB9
:104EE0009A83D3E0D5F80330052B694B05D86E4A79
:104EF000D0781873FFF7D6FAC8E000221A73C5E01D
:104F0000D5F80310C9B204F01FFBBFE0D5F80310B9
:104F10000020C9B204F044FBB8E0D5F8031000202B
:104F2000C9B204F047FBB1E004F0A6FBAB78D5F8BA
:104F3000031020B91846C9B204F050FBA6E0184689
:104F4000C9B204F073FBA1E0002004F095FBD5F892
:104F5000031020B9A878C9B204F04AFB96E0A878FB
:104F6000C9B204F077FB91E0002004F085FBD5F88E
:104F7000031020B9A878C9B204F044FB86E0A878F1
:104F8000C9B204F05DFB81E0D5F803100020C9B27E
:104F900004F042FB7AE0D5F80310C9B204F0B4FB88
:104FA00074E0D5F803100020C9B204F0C1FB6DE035
:104FB000D5F803100020C9B204F0C4FB66E0D5F8B0
:104FC0000310C9B204F0C8FBAA78384B03EBC20344
:104FD000D5F803205A7159E0D5F80310002049B2E2
:104FE00004F0F8FB52E0D5F803100020C9B204F039
:104FF00021FC4BE0D5F80310C9B204F025FC45E0D4
:10500000D5F803100020C9B204F028FC3EE0D5F822
:1050100003100020C9B204F02BFC37E0D5F80300E0
:10502000224B186090BB597904F096FB2EE01F4B81
:10503000D5F803201A711B4B1B78012B26D11A4B74
:105040000020D978FFF7F4F920E0D5F8031000200C
:10505000C9B204F0B9FA19E00020D5F80310FFF73F
:105060003DFB13E0D5F80320094BE9781A610020D5
:1050700001F01F01FFF760FBD5F80310A878491174
:10508000FFF752FB02E00322094B1A7003B030BD58
:10509000200F00208E0F0020A00A0020B80500205D
:1050A000840F0020870F0020200A0020B40E00206B
:1050B000940A002073B5CD4ECD4CB0787378354648
:1050C00010B1042323705BE2A52B00F0EF8100F206
:1050D0009180852B00F02A8138D8092B00F03F8180
:1050E0001AD8042B00F027810CD8012B00F0158171
:1050F000002B00F00F81022B00F01581032B00F034
:1051000015812BE2062B00F01A81C0F01681072BC7
:1051100000F01881082B56E0802B00F0FB8009D8A6
:105120000B2B00F02181C0F030810C2B00F00D81A1
:105130000D2B29E0822B00F03681C0F0EE80832B0E
:1051400000F0F980842B00F0EE8007E2992B00F04C
:1051500044812BD88D2B00F0348110D8872B00F0A0
:105160002581C0F0EA808A2B00F023818C2B40F04F
:10517000F581002004F0FCF9C0F10800D1E0942B87
:1051800000F0E3800AD8932B40F0E881002014213E
:1051900001AA05F069FD9DF8053001E1952B00F0AD
:1051A0001281962B40F0DA81924BBDE1A02B00F0EA
:1051B000628113D89B2B00F0D780C0F029819C2BF3
:1051C00000F0E3809D2B40F0C981002005F047FDF1
:1051D000AB785B00184100F00103B6E1A22B00F0B0
:1051E0005181C0F04B81A32B00F05081A42B00F023
:1051F0005181B3E1C02B00F0A58047D8AF2B00F060
:10520000838121D8AA2B00F071810ED8A72B00F042
:105210006581C0F05781A82B00F06481A92B40F074
:105220009D81002004F0ACFA7BE0AC2B00F065819E
:10523000C0F05F81AD2B00F06381AE2B40F08E811A
:10524000002004F0E5FA6CE0B42B00F06C810ED87D
:10525000B12B00F06081C0F05A81B22B00F05F8169
:10526000B32B40F07B81002004F062FB59E0B62BA9
:1052700000F05F81C0F05A81B72B00F05D81B82B40
:1052800040F06C81002004F0FFF94AE0CF2B00F0E1
:10529000D8801FD8C52B00F0CC800CD8C22B00F0D2
:1052A000C380C0F0BE80C32B00F0C080C42B40F090
:1052B0005581514B3EE1C82B00F0BD8002D8C72B71
:1052C0003DD04BE1CC2B00F0B980CE2B40F0468195
:1052D0004A4B2FE1D52B00F0C8800DD8D12B00F020
:1052E0002E81C0F0C080D22B00F02D81D42B40F055
:1052F0003581434B5B6928E1D72B00F02881C0F052
:10530000B780DB2B00F02681FE2B40F027813C4B41
:105310001B7B1AE10020014601E00020022105F07C
:10532000A1FE60601CE10020082101E000200A21AC
:1053300005F0B1FCF5E7334BFCE0334BFAE0304BC2
:105340005B7A02E12E4B9B7AFFE00020142101AA38
:1053500005F08AFC9DF80530C3F34003F5E02B4BC4
:105360009B68C3F34013F0E001AA00207C2105F004
:105370007BFCAA780223520003FA02F29DF8063061
:105380001A420CBF00230123DFE001AA00207C2188
:1053900005F06AFCAB789DF806205B0042FA03F347
:1053A00003F00103D1E000200421C1E700200E2119
:1053B000BEE70020142101AA05F056FC9DF8063036
:1053C000C3E01A21B4E70020142101AA05F04CFC27
:1053D0009DF80530C3F38003B7E0182101AA05F05A
:1053E00043FC9DF8053003F00F03AEE0200A0020D7
:1053F000940A00208E0F0020AC0E0020C80E002062
:10540000200F0020A40E0020A00A0020000C014064
:105410000020182101AA05F027FC9DF805301B0982
:1054200093E0584B1B7A90E0564B83E0554B5B68FA
:105430008BE0554B7EE0534BDB7F86E0514BDB89A5
:1054400083E0524B60601A780AB101226260002248
:105450001A704F4B1A781AB1626842F00202626009
:1054600000221A707CE04B4B5EE0464B9B7F6CE069
:10547000444B9B8B69E004F083F852E7002004F072
:1054800087F84EE7002004F0EFF84AE7002004F028
:10549000F3F846E7002004F0EFF818B9B07804F00C
:1054A000FBF83EE7B07804F017F93AE704F0E4F8C7
:1054B000B37818B9184604F0F7F832E7184604F044
:1054C0001BF92EE7002004F0D7F818B9B07804F0E3
:1054D000F3F826E7B07804F007F922E7002004F09B
:1054E000F3F81EE7002004F041F91AE704F050F940
:1054F00017E7002004F054F913E7274B5B7924E009
:10550000002004F07BF90CE704F0EAF909E7002039
:1055100004F0EEF905E7002004F0F2F901E70020BD
:1055200004F0F6F9FDE61D4B1B780EE0154B9B6968
:105530000BE0194B1B6808E0174B1B7905E00020B6
:10554000FFF7B8F8EDE60F4B1B69636008E0FEF764
:10555000B3FFE6E60020FFF7FDF8E2E60323237041
:105560000F4B1B7863B10F4B62681A600E4B1AB970
:105570001A6842F0080202E01A6822F008021A6073
:1055800002B070BD200F0020440F0020180F002033
:10559000BD0E0020190F0020B40E0020B20E002016
:1055A0008F0A0020800A0020280A002038B5B34A5C
:1055B00095781446022D00F03B81032D00F03F81C9
:1055C000002D40F0BC8153784F2B00F0C68044D8AA
:1055D000462B00F09A8016D8422B00F0848009D820
:1055E000402B7CD0412B40F0A881D178A44B0020E7
:1055F00019707CE0442BA24A7DD000F28280E178D1
:105600000420117173E0492B00F091800BD8472BD7
:1056100000F08680482B40F09081D378984926206E
:1056200001F8263FD9E04C2B00F08D804D2B00F087
:105630008F804B2B40F08181914CD1780320E17019
:1056400002F05DFCE07802F019FFE07802F016FF4E
:10565000E078BDE8384003F093B8572B00F0CB80DA
:1056600013D8522B00F0A08006D8502B00F0888071
:10567000512B00F08A8060E1542B00F0A380C0F031
:105680009A80552B00F0AB8057E1832B00F0C1804E
:105690001AD8592B00F0B5805A2B40F04E81784D26
:1056A000D378294601F8283F2820012202F086FC01
:1056B00095F82800BDE8384010F001001ABF00201E
:1056C0000121014605F01CBD852B00F0AC80C0F027
:1056D000A580FF2B40F03181D2786A4B31E140F256
:1056E000FF70D17803E0D178654B01205970BDE897
:1056F000384002F004BCD4F803301C20D361624966
:1057000009E0E17805205171F1E7D2F803305C49F6
:105710000C2041F80C3F0422BDE8384002F04EBC9A
:10572000D2F803305649082041F8083FF3E7D27811
:10573000534B0AB9DA7503E054490122DA754A601D
:105740001720D97DD3E7D1784D4B02209970CEE751
:10575000D1784B4B15205975C9E7D2F80310484C46
:10576000C9B21920617602F0CAFB607E10F0010018
:105770001ABF284601210146BDE8384005F0AEBCFD
:10578000D1783F4B16209975B1E73D4B1A7D1D46E8
:1057900012F0010F04D0E378DB0701D402F013FB11
:1057A000E17814202975A2E7D2F80330344920208B
:1057B00041F8203FAFE7D2F803303149102041F8DB
:1057C000103FA8E7D2F80330012B00F2B8802B4B32
:1057D0002B49DB781A2001F81A3F01229CE7D2F806
:1057E0000330012B00F2AB80244B2549DB781B20D2
:1057F00001F81B3FF1E7D3782149272001F8273F23
:10580000EBE7D2F803301E49242021F8243F02227E
:1058100082E7D2F803201E4B5A6038BDD2F803202D
:105820001C4B1A6038BDD2F80320194B9A6038BD62
:105830005178194BD2F8032043F8212038BD537812
:10584000272B62D02CD8022B48D00CD8002B3CD070
:10585000012B72D1114BD2F803205A6003F01EF8CD
:105860000B4B186138BD1B2B41D01C2B46D0092B8C
:1058700063D1D2F80320094BDA6038BD200A00203A
:10588000080000208E0A002024000020940A002036
:10589000B8050020900A0020A40A0020480F00202C
:1058A0002B2B3BD007D8292BD2F80320264B31D005
:1058B00032D85A6138BD2D2B3AD034D32E2B3CD15F
:1058C000D2F80320204BDA6238BD1F4BD2F80320F8
:1058D0001A6002F0E3FF1D4BD86038BD1A4BD2F8B6
:1058E00003209A6002F0DAFF184B586138BD00209F
:1058F000D2F80310BDE8384005F015BB0020D2F8FF
:105900000310BDE8384005F038BBD2F803200E4B39
:105910001A6138BD9A6138BDDA6138BDD2F803200A
:10592000094B1A6238BDD2F80320074B5A6238BDC2
:10593000D2F80320044B9A6238BD032200E004220F
:10594000034B1A7038BD00BF480F0020B805002077
:10595000940A00202DE9F843054614460E46002916
:105960004DD000284BD0814249D04FEA42185FFA0F
:1059700088F848F006073946002005F073FB48F028
:105980000C018146002005F06DFB8046284609F099
:105990004DFF0546304609F049FF014628460AF00A
:1059A00051F80646484609F041FF31460AF04AF8E8
:1059B0000AF05AF90546404609F038FF31460AF028
:1059C00041F80AF051F9002D08BF01250D490028C2
:1059D00014BF80464FF0010830460AF01DF90A4E08
:1059E00030B12046414605F0B2F9331901225A7010
:1059F000002039462A4605F0A2F801233355BDE8B8
:105A0000F88300BF0000A041B805002038B50E4D56
:105A100004462B5C63B10D4B410141F0060153F884
:105A20002420002001F0E60105F077F800232B5533
:105A300025446B783BB1064BE0B253F8241005F0D7
:105A400086F900236B7038BDB8050020A40E002035
:105A5000A00A00202DE9F341B94EBA4F3378D6F8A9
:105A600003006422222B7B703A70786035463C46F6
:105A700001F052815BD80F2B00F0CB8526D8072B85
:105A800000F0D28111D8032B00F0D88007D8012B69
:105A900000F0BD80022B00F0C58001F0BBBB052BE0
:105AA00000F0BA8140F2DF80BAE10B2B00F00B85E9
:105AB00005D8092B00F0C38340F28182C3E30D2B8C
:105AC00000F0348540F21C8500F07BBD192B00F0FE
:105AD000F18614D8152B00F0508607D8132B00F050
:105AE000EF85142B00F0278601F094BB172B964B03
:105AF00000F0C68600F2D186D86101F00EBC1E2BE4
:105B000000F0F2840CD81B2B00F0F686C0F0E38680
:105B10001C2B41F07F838C4B00221A7601F0FDBBD9
:105B2000202B01F0528041F2178001F0A1B8812BA7
:105B300001F07B8135D8412B01F0658117D8252BE9
:105B400001F0258107D8232B01F0ED80242B01F0F3
:105B5000F18001F05FBB272B01F04781C1F020816C
:105B6000402B41F0578303F090FA01F0D6BB452B50
:105B700001F0528108D8432B01F0488101F249819C
:105B800003F085FA01F0C9BB472B01F04B81C1F04E
:105B90004681802B41F03E836B4B00221A7601F048
:105BA000BCBB882B01F0CB811BD8842B01F06E810C
:105BB0000DD8822B01F04D81832B41F02B83624B5A
:105BC000002183F8441083F82C1101F046B9862B8C
:105BD00001F07B8101F2E8815B4B00221A7601F033
:105BE0009CBB8C2B01F03B8206D88A2B01F01B82D8
:105BF00041F2018201F02EBAF22B01F0BB82FF2BA1
:105C000001F0FE828D2B41F0058301F04CBAB37890
:105C100053B903F079FF002801F0FF8206232370B7
:105C200001F07BBBB3781BB10423237001F075BB7B
:105C300003F06AFF002801F01583EFE7B578002D27
:105C4000F2D1424B28461D70414B1D7004F096FE68
:105C500028462946022205F036F82846082104F095
:105C6000E7FF01F05ABB03F04FFF0028D6D1B3780D
:105C7000002B40F09980324B5B78032B00F2C880F8
:105C8000DFE803F002296C960020FFF7BFFEB17831
:105C90002F4B00245C542D4B2E4E5C5401238B4023
:105CA0003278490122EA0303204601F0E001D5F8E9
:105CB0000320337004F043FFA9782246204605F004
:105CC00002F8AB78244901EB4312927F002A41F09D
:105CD000F08201F022BB0020FFF798FEB3781C4A47
:105CE0000026D654194A3046D6545B0143F00201CF
:105CF00001F0E20105F0B6F9A97801238B40154FB8
:105D0000D5F803803A788044490122EA03033046FB
:105D100001F0E00142463B7004F011FF304632468C
:105D2000A97804F0D0FFA8780B4AC4F8048002EBED
:105D300040139B7F002B41F0D58201F0EEBA00BFEB
:105D4000200A0020940A0020B8050020180F002027
:105D5000BD0E0020B10E0020200F0020D5F803302A
:105D6000CC4E142B20DCCC4A002052F82350FFF7F5
:105D70004DFEB17801228A40C84B00245C54C84BC8
:105D80005C54C84B4901187801F0E00120EA020296
:105D90001A7020462A4604F0D2FE2046B1782246E8
:105DA00004F091FF01F0B9BA0423237001F0B5BAF1
:105DB000D6F80330B74C142B01F3AF820221002038
:105DC00005F050F9A378D4F80310B34A194452F8F7
:105DD0002160002506441846FFF718FEA17801222D
:105DE0008A40AE4B5D54AE4B5D54AE4B49011878C2
:105DF00001F0E00120EA02021A702846324604F05F
:105E00009EFE2846A1782A4604F05DFF01F085BA7F
:105E100003233B7001F081BAFEF744FE01F07DBA26
:105E2000FFF748F901F079BAB078737800287FF469
:105E3000FBAE9A2B2AD8992B79D2822B65D00BD81E
:105E4000062B54D003D8042B4BD0052B0AE0072B8C
:105E500054D00C3B012B11E08C2B5BD00AD8832B48
:105E60003FD0862B40F0A78000200C2105F023F8BE
:105E700001F053BA8D2B54D0933B022B00F29B8040
:105E80000020142105F017F801F047BAC82B6FD095
:105E90000DD8C12B57D004D8B52B4DD0C02B2DD049
:105EA00089E0C32B5DD055D3C72B20D083E0D42B02
:105EB0006CD00AD8CC2B62D0D22B7CD150207A491E
:105EC000042202F07BF801F028BAD62B6CD064D300
:105ED000FE2B70D14C207549012202F06FF801F0C1
:105EE0001CBA0020062104F0E6FF01F016BA704B40
:105EF0004920597A02F003F801F00FBA6C4B4A209E
:105F0000997A01F0FCFF01F008BA042104F0D3FFF4
:105F100001F003BA4B206749012202F04FF801F06B
:105F2000FCB900201A2104F0C6FF01F0F6B91821CF
:105F300004F0C1FF01F0F1B958205F49042202F0DA
:105F40003DF801F0EAB95A4B4820197A01F0D7FF21
:105F500001F0E3B940205949042202F02FF801F082
:105F6000DCB944205649042202F028F801F0D5B9E2
:105F70005F205449012202F021F801F0CEB94E20F1
:105F80005149022202F01AF801F0C7B954204F49D2
:105F9000042202F013F801F0C0B95E204C4901223E
:105FA00002F00CF801F0B9B95C204A49022202F073
:105FB00005F801F0B2B90323237001F0AEB973788C
:105FC000B678344F002E7FF42FAE9A2B47D8992BFA
:105FD00080F0F080822B00F0CF800ED8062B00F0EE
:105FE000BD8004D8042B00F0A380052B0DE0072B07
:105FF00000F0BB800C3B012B29E08C2B00F0C28011
:1060000020D8832B00F09480862B40F01481002050
:106010000C2104F02DFFAC780020610141F00C014F
:1060200001F0EC0104F037FE2B4B2C4A43F824001E
:10603000A87800210244517053F8201004F087FE24
:1060400001F06BB98D2B00F0AF80933B022B00F277
:10605000F2800020142104F00BFF01F05EB9C72B81
:106060007CD03DD8C12B00F0BC8005D8B52B00F00A
:10607000B180C02B79D0DEE0C22B00F0B980C32BF9
:1060800040F0D98044200E49042202F02AF801F0A1
:1060900044B900BF200A00202C0A0020BD0E0020B9
:1060A000180F0020B10E0020300F00202C0F002010
:1060B000200F00202B0F0020380F0020200F002081
:1060C000240F00203F0F00202E0F0020340F00204F
:1060D0003E0F00203C0F0020A00A0020B805002041
:1060E000D42B00F093800CD8C82B00F08880CC2BE8
:1060F00040F0A1804E20B149022201F0F2FF01F0F0
:106100000CB9D62B00F09080C0F08780FE2B40F0B9
:106110009280AB4C4C2004F10C01012201F0E1FF14
:10612000BB7804EB4314207BFEF7BCF901F0F5B813
:106130000020062104F09CFEAC780020610141F0B3
:10614000060101F0E60104F0A6FD9E4B9E4A43F8CD
:106150002400AB780021D15401F0DFB8492001F0D0
:10616000A7FF974B587201F0D8B84A2001F0A0FF62
:10617000934B987201F0D1B83046042104F078FEB8
:1061800001F0CBB88E4C4B2004F10B01012201F041
:10619000A8FFB87804EB4014E17AC1F10801C9B254
:1061A00003F0C4F901F0B9B830461A2104F060FEDA
:1061B00001F0B3B83046182104F05AFE834BB8788A
:1061C00053F8201004F0C3FDBB787F4A13445E707F
:1061D00001F0A3B858207E49042201F082FF01F0AB
:1061E0009CB8482001F064FF754B187201F095B817
:1061F00040207849042201F074FF01F08EB85F203E
:106200007549012201F06DFF01F087B854207349F0
:10621000042201F066FF01F080B85E20704901227F
:1062200001F05FFF01F079B85C206E49022201F0B5
:1062300058FF01F072B80323237001F06EB8FFF726
:10624000B5F901F06AB8B278674B022A00F0B18064
:10625000032A00F0D780002A40F01D815B78512B83
:1062600000F086802CD8472B70D014D8432B68D0F0
:106270000AD8412B60D061D8402B40F00A8140F20F
:10628000FF7001F015FFEDE0452B584A5CD040F25D
:106290008380D368FBE04C2B61D008D8492B5BD0BE
:1062A00056D34B2B40F0F580504BDB78EFE04F2B73
:1062B00058D05AD84D2B40F0EC804C4B5B7DE6E03B
:1062C000802B66D013D8552B59D005D8532B474A6D
:1062D00051D052D8136ADAE0592B53D05A2B54D0EC
:1062E000572B40F0D680414B93F82730CFE0842BDA
:1062F00056D008D8822B344A4ED04FD8137E1E1F5A
:1063000073427341C3E0F02B4CD00DD8852B40F085
:10631000C0802D4A364993684B4303F540533933C7
:10632000936023F00043B2E0FE2B3BD0FF2B40F004
:10633000B080304B1B7838E02C4B34E02B4B5B7833
:10634000A5E02A4B1B79A2E05379A0E0274B84E01B
:10635000264B93F826309AE0244BDB7D25E0234B37
:106360009B7894E0214B5B7E91E0204B9B7D8EE0FF
:106370001E4B1B7D8BE0136989E0937E87E01B4BEE
:10638000DB7E84E0194B9B8C81E0184B93F828301E
:106390007DE00D4B1B7E7AE0D36978E0536876E0B0
:1063A000154B57E0154B1B7871E0003318BF0123E4
:1063B0006DE05A78124B53F8223068E02E0F00201F
:1063C000200F0020A40E0020B8050020A00A002005
:1063D000380F0020200F00203F0F0020340F002036
:1063E0003E0F00203C0F0020200A00200800002063
:1063F0006D4EC6418E0A0020900A00207C0F0020BE
:10640000A40A00205B78272B32D011D8022B23D08E
:1064100005D8F3B1012B3CD19F4B5B6837E01B2BB8
:106420001DD01C2B20D0092B33D19B4BDB682EE0D9
:106430002B2B24D005D8292B974B1CD01DD85B695A
:1064400025E02D2B21D01DD32E2B22D1924BDB6AA0
:106450001DE0914B1B681AE08F4B9B6817E00020F2
:1064600004F0B5FD606018E0002004F0C5FDF9E718
:10647000894B1B690BE09B6909E0DB6907E0864BF0
:106480001B6A04E0844B5B6A01E0834B9B6A636098
:1064900003E0032300E004232370804B1B78002BD0
:1064A00000F03B877E4B62681A607E4B2AB91A68FF
:1064B00042F008021A6000F030BF1A6822F00802A9
:1064C0001A6000F02ABFB378022B15D17378372BEE
:1064D0000ED8754903F5A770800001EB83010422F3
:1064E00001F06CFD00F019BF7378142B40F20383A8
:1064F0000323237000F011BF04233B7000F00DBF95
:10650000B378022B0ED1694B5B78372BF0D86649F4
:1065100003F5A770800001EB8301042201F0E1FD87
:1065200000F0FBBE04233B7000F0F7BEB378002BF5
:106530007FF47AAB6B785D4E012B21D002D3022B16
:1065400023D03AE003F0E0FA00287FF467ABB0789C
:1065500004F00CFAB17839B9554B01221A70554B39
:1065600000221A7000F0D9BE534A937F002B00F02E
:10657000D48602EB4112927F9A4240F0CE86EBE73E
:10658000002004F0FBF900F0C8BE002004F0FEF982
:10659000424B78601B78002B00F0BF86404B1860A0
:1065A000404B1A6820B942F008021A6000F0B5BEEC
:1065B00022F008021A6000F0B0BE03233B7000F026
:1065C000ACBEB37813B1022B04D01EE0FDF74EFF32
:1065D00000F0A3BE354B5B78072B0AD820B91846CC
:1065E000FDF7AEFE00F099BE1846FDF7B5FE00F0CF
:1065F00094BEFF2B7FF47CAF451C0ABF284BC0B272
:106600001878FDF7B5FE00F088BE04233B7000F05B
:1066100084BEB378012B23D005D3022B24D170780C
:10662000FDF7DAFE0DE07078082802D8FDF7B1FE1C
:1066300007E00A2801D100230BE00B2803D1FEF765
:106640000BF9606012E00C2805D11C4B9B68C3F36A
:10665000401363600AE0FF2808D1FDF7CFFEF0E7A2
:10666000707802F0B5F9ECE704233B700B4B1B7814
:10667000002B00F052860A4B62681A60094B2AB957
:106680001A6842F008021A6000F047BE1A6822F049
:1066900008021A6000F041BE480F00208F0A002057
:1066A000800A0020280A0020A40A0020200A0020D6
:1066B000B8050020BD0E0020200F0020000C014076
:1066C0007278944B092A27D8DFE802F005080B0EF0
:1066D00012181B1E21251A6810441CE01A68101A93
:1066E00019E01A68504316E01A6892FBF0F012E0C5
:1066F0001A6892FBF0F100FB11200CE01A681040C0
:1067000009E01A68104306E01A68504003E01A686E
:10671000D2431A6000E018601A687F4B2AB91A68E1
:1067200042F008021A6000F0F8BD1A6822F0080270
:106730001A6000F0F2BD774B1A68774B82421968F5
:1067400004DD21F0030141F0040108E00BBF21F05A
:10675000060121F0050141F0010141F0020119603B
:106760002AB91A6842F008021A6000F0D6BD1A6809
:1067700022F008021A6000F0D0BD73780C2B00F2F2
:10678000CC85DFE803F0071019222B343E4750591F
:10679000626B7400604B1B681C0740F1BE855F4B49
:1067A000D86100F0BABD5C4B1B68190700F1B585D4
:1067B0005A4BD86100F0B1BD574B1B68DA0740F166
:1067C000AC85564BD86100F0A8BD534B1B68DB0766
:1067D00000F1A385514BD86100F09FBD4E4B1B6863
:1067E0005F0740F19A854D4BD86100F096BD4A4B4A
:1067F0001B6813F0050F00F09085484BD86100F03E
:106800008CBD454B1B689E0740F18785434BD86183
:1068100000F083BD404B1B689D0700F07E853F4B19
:10682000D86100F07ABD3C4B1B68DC0640F17585F1
:106830003A4BD86100F071BD374B1B68990640F1A7
:106840006C85364BD86100F068BD334B1B685A0627
:1068500040F16385314BD86100F05FBD2E4B1B6862
:106860001B0640F15A852D4BD86100F056BD2A4BCE
:106870001B68DF0540F15185284BD86100F04DBD04
:106880001A6A072A00F24985511C1962D96903EB7B
:1068900082025162D86100F040BD1B6A1F4A002B82
:1068A00000F03B85013B136202EB83035B6AD3611B
:1068B00000F033BD73782E2B04D8194A0121D1542E
:1068C00000F02BBDFF2B7FF413AE144B012283F895
:1068D000442000F022BD73782E2B04D8104A0021EA
:1068E000D15400F01ABDFF2B7FF402AE0B4B0022F7
:1068F00083F8442000F011BD084C94F84530CBB922
:10690000461C4FF00A030DD1024A10684343A364AA
:106910000AE000BF800A0020280A0020B8050020F5
:106920008F0F00205843A06401F0B8FF0123E064FA
:1069300084F845306B78042B00F2EF84DFE803F035
:10694000034372A7190001F0A9FFE26CA16C801A41
:1069500080EAE072A2EBE0728A42AE4B04D90022D8
:1069600083F8452000F0D9BCDA69013ADA6100F019
:10697000D4BCA87804F00AF840B9A74B84F84500C5
:106980001A6822F010021A6000F0C7BCA36CA14D77
:10699000A3B101F083FFEB6CAA6CC01A80EAE0732C
:1069A000A3EBE073934209D9002385F845309A4B55
:1069B0001A6842F010021A6000F0AFBCE369013BB4
:1069C000E36100F0AABC002004F049F9AB785B0059
:1069D000184110F0010609D0002384F845308E4B91
:1069E0001A6822F010021A6000F097BCA36C894D5F
:1069F0009BB101F053FFEB6CAA6CC01A80EAE07304
:106A0000A3EBE073934208D9834B85F845601A687D
:106A100042F010021A6000F080BCE369013BE361C0
:106A200000F07BBC6A4600207C2104F01DF9AA78A6
:106A30000223520003FA02F29DF8023012EA030721
:106A400009D0002384F84530734B1A6822F01002F5
:106A50001A6000F062BCA16C6E4D99B101F01EFF8E
:106A6000E96CAE6C401A80EAE071A1EBE071B142D2
:106A700008D9694B85F845701A6842F010021A600F
:106A800000F04BBCE369013BE36100F046BC6A46A1
:106A900000207C2104F0E8F8AB789DF802205B0030
:106AA00042FA03F313F0010609D0002384F84530BD
:106AB000594B1A6822F010021A6000F02EBCA26C2A
:106AC000544D9AB101F0EAFEEA6CA96C801A80EA92
:106AD000E072A2EBE0728A4208D94F4B85F845601C
:106AE0001A6842F010021A6000F017BCE369013B1B
:106AF000E36100F012BCB2789AB9484A4849927EE4
:106B000041F82300002A00F00884002B00F00584DF
:106B100003F28510800001EB8301042201F04EFA9C
:106B2000FBE3FF2A7FF480A863B94FF4C3643D49B7
:106B3000204621440422043401F040FAB4F5CD6F1C
:106B4000F5D1EAE3364903F28510800001EB8301B9
:106B5000042201F033FAE0E37378142B3FF6C8AC5B
:106B6000314A9278B2B92E4A52F823202F4B7A60DC
:106B70001B78002B00F0D1832D4B1A60264B22B9D5
:106B80001A6842F008021A60C7E31A6822F0080285
:106B90001A60C2E3FF2A7FF447A863B94FF4C364C5
:106BA0002049204621440422043401F09AFAB4F525
:106BB000CD6FF5D1B1E31A4903F28510800001EBE6
:106BC0008301042201F08DFAA7E37678142E3FF6B4
:106BD0008FACA878144F01062CD5C20706D500202B
:106BE000022104F03FFA0E4B43F826000B4B9B7E2C
:106BF000002B00F092836B78002B00F08E83084905
:106C000003F28510800001EB8301042201F0D6F924
:106C100083E300BFB8050020280A002008000020F8
:106C20002C0A002018040020200A00208F0A0020CF
:106C3000800A002000287EF4F7AF022104F012FA47
:106C4000994B9A4A9B7E42F82600002B00F0658300
:106C50007B78002B00F06183B97803F2851008443B
:106C6000194402EB81018000042201F0A7F954E3EA
:106C700072788F4B0A2A42D8DFE802F0060B111611
:106C80001C24292E33383C008A491A6809680A44B2
:106C900003E088491A680968521A1A602FE085498A
:106CA0001A6809684A43F8E782491A68096892FB3A
:106CB000F1F2F2E77F4A1968126891FBF2F002FBE9
:106CC0001012EAE77B4A11681A680A40E5E7794A38
:106CD00011681A680A43E0E7764A11681A684A4060
:106CE000DBE7744A1168C943116008E01A6871490A
:106CF0000A6004E06F4A18681168106019601A6829
:106D00006D4B22B91A6842F008021A6005E31A684E
:106D100022F008021A6000E3654B1B68C6F80330D6
:106D2000FDF7C0FEF9E2624B1B68C6F80330FEF7C0
:106D30003DFCF2E27378052B00F2EF82DFE803F00E
:106D400003090F151B215C4B1A6802F00F021A6031
:106D5000E3E2594B1A6822F010021A60DDE2564B4A
:106D60001A6822F020021A60D7E2534B1A6822F008
:106D700040021A60D1E2504B1A6822F080021A6079
:106D8000CBE24D4B1A6822F480721A60C5E2737828
:106D90002E2B3FF6ADAB494A02EB83031865BCE2EC
:106DA000464B4349D3F80C210A60D3F810214149DE
:106DB0000A60D3F814214049DA61D3F818210A6037
:106DC000D3F81C213E4983F84520D3F82021DA640A
:106DD000D3F824219A6493F82821885C08B1012013
:106DE0008854002283F82C2197E2B378002B7EF49C
:106DF0001BAF7378142B3FF67BAB2D4A11682B4ADF
:106E000042F8231089E202F041F986E202F040F9EB
:106E100083E202F04FF980E202F04DF97DE202F0E8
:106E20004BF97AE202F049F977E2737813B1012B5A
:106E300004D00BE0214B01221A766EE2B0F5006F10
:106E4000BEF4F2AE1D4A1376D06166E203233B70B6
:106E500063E21A4B02221A765FE2184A4FF0FF30C3
:106E600002F1500343F82100154800234354013137
:106E70002F29F2D11376D361136282F845300C4A80
:106E800013600C4A13600C4A136046E2064B1B7DEC
:106E90009B0717D4B0F5006FBEF4C6AE074B0422B3
:106EA0001A76C3F8300138E2080000202C0A0020CE
:106EB000800A00209C0A0020280A0020B805002033
:106EC0008F0F002008233B7027E2994B01221A7094
:106ED000984B994C9A78B0F5006F227025D21B7DA3
:106EE00013F0010521D1694600F02CFF9DF8003018
:106EF000257263709DF80130A3709DF80230E37035
:106F00009DF8063023719DF8053063719DF80430BB
:106F1000A3719DF80330E3710123E15C227A013310
:106F20000A44082B2272F8D1F7E101230021E15431
:106F30000133082B804AF9D113781372EDE173788D
:106F4000012B1DD00AD3022B2BD1794B01221A70B1
:106F5000784B794A9B781370002319E0744B012217
:106F60001A70744B744A9B781370744B1868002322
:106F70000133C11811F8011C082BD154F8D1CCE110
:106F80000422FA717B7189222A23BA713B71C4E110
:106F90006B490133194411F8091C082BD154F7D15E
:106FA000BBE103233B70B8E17378032B00F2B5819A
:106FB000DFE803F0020E191D624B1A7EFA7193F896
:106FC0004520D3F83031BA711A0A7A713B71A4E1C5
:106FD0005C4B1A7EFA7193F84520DB69BA711A0A84
:106FE0007A713B7199E1584B1B687B6095E1574B77
:106FF0001B687B6091E17378002B40F08E81544BCD
:107000009978002940F0898140F2D243984240F0BB
:10701000848140F2FF7000F072FF00F0D4FE012086
:10702000FDF70BFA79E172784A4B02B101221A702E
:10703000EA78494B1A70434B93F83411474B197057
:10704000474900230B7047490B70474B19780A4397
:107050001A7062E13B4B012283F835215DE17578BE
:1070600015B1012D0FD01BE0042240F2FB706946E0
:1070700001F037F8009BD6F803209A4206BF01239F
:107080007B607D6049E1B3782A2B06D140F2FB702A
:107090003649042200F092FF3FE103233B703CE1BC
:1070A00003233B7039E17378032B3DD8DFE803F00D
:1070B00008022E39234A0023D2F83811154610E071
:1070C000204BD3F83821092A07D8511CC3F83811AE
:1070D00003EB8203C3F83C011FE109233B701CE171
:1070E00001338B4200F01981214A9E0052F823405F
:1070F0008442F5D13244481E834204D250680133A1
:1071000042F8040BF7E7C5F8380106E10D4A002301
:10711000C2F83831164A002199500433282BF9D18E
:10712000FBE00A237B60F8E003233B70F5E000BF3F
:10713000840A002008000020850A002000000020AA
:1071400000400008B8050020800A00209C0A0020AA
:10715000200A0020B00E0020C40E0020860F002060
:10716000BE0E0020BE0F0020B10E0020230A00201A
:10717000F40600207378812B40F0CF80B278684B02
:10718000922A40F0CA809A79A32A40F0C6805A79A0
:10719000B42A40F0C2801A79C52A40F0BE80DB785C
:1071A000D62B40F0BA805F4B4FF480621A6101F039
:1071B0000BFF01F073FB044601F070FB001B00287D
:1071C000B8BF4042B0F57A7FF6DBFDF73DF905F038
:1071D000DBF8002005F0ACFD0021534804F0ADFCC5
:1071E000514804F00FFC514804F06EFA04F0EAFC38
:1071F0004FF0804005F0F2FD0020FDF71EF98CE015
:1072000040F2D243984240F08880494B012283F8F3
:10721000642182E0022323707FE0B37843B1454AC2
:1072200002EB43139B7F002B77D0927F9A4274D15D
:107230003F4B01221A70404B00241C703F4B2046EC
:10724000214602221C7003F03EFD2046062140F23A
:10725000FF7203F062FC20460821D5F8032003F0FA
:107260005CFC5AE02E4B9B7843B1324A02EB43134D
:107270009B7F002B51D0927F9A424ED12C4B012202
:107280001A702D4B00241C702C4B204621460222E4
:107290001C7003F018FD2046062140F2FF7203F037
:1072A0003CFCD5F8032020460821524203F035FC6F
:1072B00033E0002B31D08B7F93422ED12046FEF756
:1072C000A5FB3378204623F001033370144B21468D
:1072D000D3F8032003F033FC20462146224603F076
:1072E000F2FC1AE0C8B1927F9A4216D1FEF78EFBEB
:1072F0000221304603F0B6FE094B3146D3F8032095
:107300003B78024423F0010330463B7003F017FC46
:1073100030463146324603F0D6FC02B0BDE8F0817B
:10732000200A0020000C0140080002400024014017
:10733000B8050020200F0020180F0020BD0E0020EF
:107340003749002370B50B603649374A0B6037491F
:10735000D36113620B6082F8453082F8443082F8C2
:107360002C311546324A4FF0FF3142F82310314A92
:107370000024D45401332F2BF4D10621204603F0EE
:1073800071FE2D4B0C211860204603F06BFE2B4E36
:107390002B4BF17A1860C1F108012046C9B202F006
:1073A000C5F8307BFDF77EF8264B0022E25004340E
:1073B000B4F5806FF8D1244EB37E13B9F37E6BB170
:1073C00018E04FF4C36421492046214404220434C8
:1073D00000F087FEB4F5CD6FF5D1EFE74FF4A76469
:1073E0001B49204621440422043400F07AFEB4F5FF
:1073F000C36FF5D1337903F0EF02012A01D0212BBD
:1074000001D1012300E0002385F86531737D23B1AC
:10741000FDF70AFA08B1012300E000232B7670BDC6
:10742000800A00209C0A0020B8050020280A0020BD
:10743000080600208F0F0020A40E0020200F00203F
:10744000A00A0020A40A0020080000201804002040
:107450006C050020F7B50F4E0F4CC6F803300F4BEC
:1074600086460F46B270002294E803001A708DE839
:10747000030086F800E07770FEF7ECFA2178636885
:10748000074A82F866119DE8030084E80300184665
:1074900003B0F0BD200A0020940A00208F0A0020CB
:1074A000B8050020014B93F866017047B80500202D
:1074B000F7B51F4E024653780C4696E803008DE858
:1074C00003001C4900270B7093786D464B70D378EE
:1074D0008B7013798B7153794B7193790B71D379CD
:1074E000CB70154B1F70FEF7B5FA144B1978334665
:1074F00071B9217032786170A2707278E270F2799D
:107500002271B27962717279A2713279E27109E005
:10751000012907D13A460A4911444978A154013258
:10752000082AF8D195E8030083E8030003B0F0BD12
:10753000940A0020200A00208F0A0020840A0020DC
:10754000850A00202DE9F043A64B89B01B78A64C94
:1075500013B994F8673163B1A44B1B78062B08D09C
:107560000A2B06D003F0EF030F2B1CBF002384F877
:10757000343194F834319C4A032B9D4E2AD192F831
:1075800065511DBB33788BB99A4F9B4DB87897F8EE
:1075900001802A78804490446A789044EA79904443
:1075A000AA7990446A7990442A7920E0012B40F02E
:1075B000E580924B585D013500F02EFF092DF8D182
:1075C000DCE0052B50D192F8655175B38A4803F081
:1075D000FDFFD3E0042BF4D1864F874DB87897F8A0
:1075E0000180002301226B702A706B6080449044FC
:1075F00000F012FF787800F00FFF287800F00CFF01
:10760000687800F009FFE87900F006FFA87900F03B
:1076100003FF687900F000FF5FFA88F8287900F02E
:10762000FBFE404600F0F8FEA8E033788BB9714FBE
:10763000714DB87897F801802A78804490446A7830
:107640009044EA799044AA7990446A7990442A79DE
:1076500017E0012B40F09280684B585D013501F036
:1076600059F8092DF8D189E0062B28D1614F624DD8
:10767000B87897F80180002301226B702A706B6044
:107680008044904401F046F8787801F043F8287877
:1076900001F040F8687801F03DF8E87901F03AF837
:1076A000A87901F037F8687901F034F85FFA88F8C2
:1076B000287901F02FF8404601F02CF85EE0072B06
:1076C0003CD192F86531002B80D132782ABB494BEE
:1076D00093F802C093F80180474B8DF808C01F78DB
:1076E0005D78C444D8798DF80A70674499798DF82B
:1076F0000B503D445A798DF80C0028441B798DF8C5
:107700000D1001448DF80E200A448DF80F301344FB
:107710008DF809808DF8103008E0012A06D1374A2B
:10772000995C02AA99540133092BF8D1344B1B7888
:1077300023B302A8092101F07BFC1FE0082B1DD117
:107740002D4A00230120537010705360294A8DF890
:107750000A00917852788DF808108DF809200A44B3
:1077600002448DF80B308DF80C308DF80D308DF80B
:107770000E308DF80F308DF81020D7E7214B1A7896
:107780009846002A6BD0204B204D1B78032B02D04B
:10779000072B3DD05FE0174F2A78B87897F8019013
:1077A000814409F10A09914400F036FE787800F02E
:1077B00033FE802000F030FE8A2000F02DFE0020F5
:1077C00000F02AFE002000F027FE002000F024FE3A
:1077D0005FFA89F9287800F01FFE484600F01CFE89
:1077E00039E000BF8E0A0020B8050020200A0020E2
:1077F000840A002008000020940A0020850A002046
:10780000A80E0020BE0F0020860F0020BE0E002014
:10781000BD4B2A789878597880238DF816308A23C2
:107820008DF8173000238DF818308DF819308DF849
:107830001A30B64B8DF8151001440A311B788DF8BB
:107840001B200A448DF814008DF81C201BB105A8DC
:10785000092101F0EDFB00232B7088F80030002394
:1078600084F83431337084F8673194F8643113B19B
:107870000120FCF7E2FD94F83521A54B52B193F8B5
:107880006521D2F1010238BF002283F86521002270
:1078900083F8352194F86551002D62D10DF1070070
:1078A00000F0D4FD00285CD000F0EEFD10B1984B44
:1078B00083F8685194F868119DF807004A1CD2B209
:1078C0002144092A924B84F8682181F8690140F02B
:1078D0004481002283F868218B4A93F869315178FA
:1078E000994207D092F82710002900F036818B4288
:1078F00040F0338192F827209A4204BF012384F894
:10790000673100231A46824D05F26911595C013333
:107910000A44082BD2B2F6D195F8713193421ED1A8
:107920007C4B95F86A211A7095F86B215A7095F87E
:107930006C219A7095F86D219A7195F86E215A71A3
:1079400095F86F211A7195F87021DA7000F0A6FF92
:10795000714B724A186000231370032279E00423EC
:1079600086E094F865316A4D7BB16A4803F0E1FC2A
:1079700058B100F093FF684B684A186000231370F9
:10798000032285F834212A7EB0E094F86551002D59
:1079900071D10DF1070000F0DBFE00286BD000F084
:1079A000F5FE10B15A4B83F8685194F868119DF8B0
:1079B00007004A1CD2B22144092A554B84F8682199
:1079C00081F8690140F0C980002283F868214E4A9D
:1079D00093F869315178994207D092F8271000291D
:1079E00000F0BB808B4240F0B88092F827209A428A
:1079F00004BF012384F8673100231A46444D05F281
:107A00006911595C01330A44082BD2B2F6D195F8BA
:107A1000713193422BD13F4B95F86A211A7095F83A
:107A20006B215A7095F86C219A7095F86D219A71B6
:107A300095F86E215A7195F86F211A7195F8702199
:107A4000DA7000F02BFF344B344A186000231370B7
:107A50000522297E85F834214A1E012A85F86831DD
:107A60002F4A02D9052918BF0123137075E0062398
:107A700085F8343171E094F86561002E52D1234BC2
:107A80001B78002B4ED005AD284601F0BBFA00282C
:107A900048D033463246E95C01330A44082BD2B25F
:107AA000F9D19DF81C1091422BD11A4B9DF815204D
:107AB0001A709DF816205A709DF817209A709DF83C
:107AC00018209A719DF819205A719DF81A201A7180
:107AD0009DF81B20DA7000F0E1FE0F4B0F4A186092
:107AE00000231370072284F83421227E511E0129BD
:107AF00019460B4B03D9052A01D0012229E0197040
:107B00002BE084F8343128E008000020A80E002083
:107B1000B8050020200A0020800F0020850F0020DB
:107B20008F0A0020237E7E4D013B012B15D8EB6987
:107B3000B3F5006F0FD2FCF777FE60B1E8697949C1
:107B4000431CEB6100F0FEF8092385F83431764BD5
:107B500001221A7001E000232376237E704D042B4E
:107B600004D1704E3278170640F1AD8094F834316C
:107B700013F0FB0F05D0082B03D0062B01D0FDF727
:107B800069FF94F83431092B79D100F087FE644AFB
:107B9000664DD2682B68801A80EAE072A2EBE07230
:107BA0009A4208D9624B1A78012A04BF02221A703D
:107BB00000F074FEE06000F071FE23696A68C01A8C
:107BC00080EAE073A3EBE073934208D9584B5A78EC
:107BD000012A04BF02225A7000F060FE206100F00A
:107BE0005DFE6369AA68C01A80EAE073A3EBE073E4
:107BF000934208D94E4B9A78012A04BF02229A7008
:107C000000F04CFE606194F84430002B37D0444BB8
:107C100093F82C21002A32D145498B5C022B2BD1C1
:107C20003F4B03F1500050F82200451C22D041493F
:107C300083F8282109680022C3F80C113E4909681D
:107C4000C3F81011D969D861C3F814113B49096808
:107C5000C3F8181193F8451083F84520C3F81C1198
:107C6000D96C0122C3F82011996C83F82C21C3F838
:107C7000241104E000238B5401322F2ACCD194F834
:107C80003411274B092904D11A7E022A04BF052288
:107C90001A76D4F83821224B002A3ED009293CD14B
:107CA000197E012939D1D86900231D4901F59E7437
:107CB00054F82340A04202D105230B762DE0013376
:107CC0009342F2D129E095F8343113F0FB0F24D020
:107CD000082B22D0062B20D0D5F83001184CD6F82E
:107CE0000330B0F5006F6270636012D2314600F06D
:107CF0003CF9D5F83001314600F0A9F830B1D5F89B
:107D000030310133C5F83031652300E0072323709B
:107D100003E00723237000232B7609B0BDE8F0832E
:107D2000B8050020200A00208F0A0020480F0020FC
:107D30008F0F0020800A00209C0A0020280A0020C3
:107D4000940A0020C0EBC00038B500F500650020A3
:107D50000C4602460321FCF727FE0020C5F307214D
:107D60000246FCF721FE0020E9B20246FCF71CFEA9
:107D7000002001460246FCF717FE20700020014655
:107D80000246FCF711FE6070002001460246FCF737
:107D90000BFEA070002001460246FCF705FEE070D5
:107DA000002001460246FCF7FFFD2071002001463D
:107DB0000246FCF7F9FD6071002001460122FCF744
:107DC000F3FDA07138BD38B54FF4006400200621E2
:107DD0000122FCF7E9FD002005210246FCF7E4FD45
:107DE000002001460122FCF7DFFD8307F3D50020C8
:107DF00002210246FCF7D8FD0020C4F30721024609
:107E0000FCF7D2FD0020E1B20246FCF7CDFD0025D3
:107E1000B5F13F0EDEF100024FF0000052EB0E0212
:107E200001460135FCF7C0FD402DF1D100200521B0
:107E30000246FCF7B9FD002001460122FCF7B4FD23
:107E4000C307F3D44034B4F5804FBFD138BDF7B584
:107E5000C0EBC00000F5006500200C46024603217F
:107E6000FCF7A2FD0020C5F307210246FCF79CFDAC
:107E70000020E9B20246FCF797FD002001460246C9
:107E8000FCF792FD0746002001460246FCF78CFDF8
:107E90000646002001460246FCF786FD0546002006
:107EA00001460246FCF780FD8DF8030000200146E4
:107EB0000246FCF779FD8DF80400002001460246D9
:107EC000FCF772FD8DF80500002001460122FCF749
:107ED0006BFD23788DF80600BB420DD16378B34269
:107EE0000AD1A378AB4207D1DDF80300D4F8033000
:107EF000C31A5842584100E0002003B0F0BD38B525
:107F0000012204460D4600200621FCF74DFD00200D
:107F100005210246FCF748FD002001220146FCF73E
:107F200043FD8207F3D5002002210246FCF73CFD09
:107F30000020C4F307210246FCF736FD0020E1B221
:107F40000246FCF731FD002029460122FCF72CFDFA
:107F5000002005210246FCF727FD002001460122F2
:107F6000FCF722FDC307F3D438BD38B5C0EBC0051C
:107F70000C4605F500600978FFF7C1FF05F6010022
:107F80006178FFF7BCFF05F60200A178FFF7B7FFA5
:107F900005F60300E178FFF7B2FF05F6040021794A
:107FA000FFF7ADFF05F605006179FFF7A8FF05F6BD
:107FB0000600A179BDE83840FFF7A1BF2DE9F041E7
:107FC00004460F461646002006210122FCF7ECFC71
:107FD000002005210246FCF7E7FC002001460122B3
:107FE000FCF7E2FC8507F3D5002002210246FCF7EE
:107FF000DBFC0020C4F307210246FCF7D5FC00207F
:10800000E1B20246FCF7D0FC0025B54242D0013473
:1080100014F03F08795D04D0721EA81A4242424112
:1080200000E001220020FCF7BFFCB8F1000F2FD1C7
:10803000731E9D422CD2002005210246FCF7B4FCA1
:10804000002001460122FCF7AFFC10F00100F2D144
:1080500006210122FCF7A8FC002005210246FCF7BE
:10806000A3FC002001220146FCF79EFC8207F3D509
:10807000002002210246FCF797FC0020C4F30721F0
:108080000246FCF791FC0020E1B20246FCF78CFCB2
:108090000135BAE7002005210246FCF785FC0020E7
:1080A00001460122FCF780FCC307F3D4BDE8F08150
:1080B00010B50446002003210246FCF775FC0020A1
:1080C000C4F307210246FCF76FFC0020E1B2024630
:1080D000FCF76AFCBDE81040002001460122FCF7D5
:1080E00063BC70B5044600200E46154603210246C7
:1080F000FCF75AFC0020C4F307210246FCF754FCAD
:108100000020E1B20246FCF74FFC0024AC420AD04A
:108110006A1EA31A00205A4201465A41FCF744FC49
:1081200030550134F2E770BD37B500200521024615
:10813000FCF73AFC002001460122FCF735FC10F068
:108140007104F2D100F0AAFB054600F0A7FB401B2A
:108150000028B8BF4042B0F5FA6F09DA4CB940F2D6
:10816000FF70FFF7A5FFB0F142035C425C41ECE712
:1081700014B1224B1B78ABB340F2FF700021FFF724
:10818000BEFEFFF720FE00201D494022FFF716FF2C
:108190004FF480701B49B422FFF710FF40201A49AA
:1081A0002022FFF70BFF002301934FF4C364204606
:1081B00001A904220434FFF701FFB4F5FF6FF6D1E3
:1081C000002301934FF4A764204601A9042204343C
:1081D000FFF7F4FEB4F5C36FF6D140F2FF70422111
:1081E000FFF78DFE002006494022FFF77AFF40206E
:1081F00006492022FFF775FF03B030BDCC0E0020EA
:1082000008000020E40A0108C40A0108200F002029
:1082100030B5054687B0524805F0CCFA4FF480409F
:10822000012104F059FB0420002104F06DF8032320
:108230008DF8063018230DEB03048DF807304FF44A
:10824000007324F8143D4748214603F0CEFF48232D
:108250008DF8073043484FF480632146ADF8043071
:1082600003F0C3FF02A805F033FB0B2D25D8DFE890
:1082700005F02406090C0F1215181B1E20224FF4BE
:1082800061531CE04FF4964319E04FF4E14316E0CC
:108290004FF4164313E04FF4614310E04FF496336C
:1082A0000DE04FF4E1330AE04FF4613307E02E4B69
:1082B00005E02E4B03E02E4B01E04FF416530293E2
:1082C000029B02A95B082648029305F0BDFA25230C
:1082D000002401258DF80030684607238DF8013011
:1082E0008DF802408DF8035004F08AF81C4840F2E3
:1082F000FF3105F0D5FB22461948282105F015FB72
:108300002A46174840F2277105F00FFB2A46144809
:1083100040F2266105F009FB2A46114840F225513A
:1083200005F003FB22460E4840F2244105F0FDFA19
:1083300022460B4840F6460105F0F7FA2246084867
:1083400040F66A1105F0F1FA22460548602105F071
:10835000ECFA0348294605F0DCFA07B030BD00BF4F
:10836000003801400008014090D0030020A1070020
:1083700040420F00684620F007018D46224919B59A
:108380000B88980614D5214B1A6858680132202AA8
:1083900008BF0022824205D01C6888881919C0B223
:1083A00008721A601A4A0A2111609A6A194B1A60F7
:1083B000154803881A0618D5164B1A68AAB9134B24
:1083C000DC6A196B8C420CD0196B4C1C1C63194471
:1083D00091F83410C9B28180196B202905D11A6334
:1083E00003E040F2277105F0A0FA074803885B0616
:1083F00006D540F2266105F077FB044B1A6BDB6A69
:10840000BDE8194085467047003801402C07002020
:10841000CC0F0020C40F00200A4BDA6A196B01321E
:10842000202A08BF00228A420AD0D96A194481F85A
:108430003400DA62044840F22771012205F075BA6F
:10844000704700BF2C070020003801400A4B5968D4
:108450001A6891420BD05A68511C59601A44127A1A
:1084600002705A68202A04D100225A6001E00020DC
:1084700070470120704700BF2C070020014B986215
:10848000704700BF2C070020044B1A7802F0FF0051
:1084900012B100221A700120704700BFD00F0020D7
:1084A00008B5FBF7D1FF044B00225A601A60BDE803
:1084B0000840FBF7C7BF00BF2C07002010B5441EC3
:1084C00014F8010F10B1FFF7A7FFF9E710BD30B5A1
:1084D000054687B0544805F06DF94FF4003001218E
:1084E00004F006FA0420012104F0F6F9042000212A
:1084F00004F00AFA0820002103F006FF03238DF898
:10850000063018230DEB03048DF80730042324F8FC
:10851000143D4648214603F068FE48238DF8073095
:10852000424808232146ADF8043003F05EFE02A85D
:1085300005F0CEF90B2D25D8DFE805F02406090C4F
:108540000F1215181B1E20224FF461531CE04FF42C
:10855000964319E04FF4E14316E04FF4164313E05D
:108560004FF4614310E04FF496330DE04FF4E133E4
:108570000AE04FF4613307E02D4B05E02D4B03E09B
:108580002D4B01E04FF416530293029B02A95B08A6
:108590002548029305F058F92623002401258DF87B
:1085A0000030684607238DF801308DF802408DF8C1
:1085B000035003F025FF1C4840F2FF3105F070FA2C
:1085C00022461948282105F0B0F92A46164840F2FB
:1085D000277105F0AAF92A46134840F2266105F0F2
:1085E000A4F92A46104840F2255105F09EF922468A
:1085F0000D4840F2244105F098F922460A4840F619
:10860000460105F092F92246074840F66A1105F046
:108610008CF922460448602105F087F90248294672
:1086200005F077F907B030BD004400400008014074
:1086300090D0030020A1070040420F00684620F0C0
:1086400007018D462E4919B50B889C061BD52D4B6D
:10865000DB68980701D58B8815E02B4B5A6D986D18
:108660000132202A08BF0022824206D05C6D888831
:108670001919C0B281F85C005A65244A0A211160B8
:10868000DA6F234B1A601E4803881A0621D5204B47
:108690001A68F2B91C4BD3F88040D3F884108C428E
:1086A00013D0184902240C61D3F884104C1CC3F871
:1086B0008440194491F88810C9B28180D3F884109D
:1086C000202906D1C3F8842003E040F2277105F089
:1086D0002CF90B4803885B060DD540F2266105F0A6
:1086E00003FA094BD3F88420D3F880309A4202D1A0
:1086F000044B02225A61BDE819408546704700BF0D
:1087000000440040000801402C070020C00F00205A
:10871000C80F00200C4BD3F88020D3F8841001320E
:10872000202A08BF00228A420CD0D3F880101944B6
:1087300081F88800C3F88020044840F227710122A4
:1087400005F0F3B8704700BF2C070020004400403C
:108750000A4B996D5A6D91420CD09A6D511C9965D6
:108760001A4492F85C2002709A6D202A04D10022EB
:108770009A6501E000207047012070472C07002017
:10878000014BD867704700BF2C070020044B1A78B4
:1087900002F0FF0012B100221A700120704700BFE2
:1087A000D10F002008B5FBF74FFE044B00229A655D
:1087B0005A65BDE80840FBF745BE00BF2C07002006
:1087C000684620F007018D4601B5BDE801408546A9
:1087D00070470000684620F007018D4601B51B4B2D
:1087E00019781A46A9B15B6801335360184B1968B0
:1087F00001311960174B196811B1196801391960F5
:10880000154B196811B119680139196000231370EB
:1088100001E001221A70114B1A683AB11A68013A44
:108820001A601B6813B90E4B01221A700D4B1A689F
:108830003AB11A68013A1A601B6813B90A4B01224F
:108840001A70BDE801408546704700BFD40700207C
:10885000900A0020C40F0020C80F0020CC0F002079
:10886000D00F0020C00F0020D10F002008B5042039
:1088700004F038FA4FF4FA5004F040FA012004F002
:1088800043FA05480321002203F090FEBDE80840AA
:10889000012004F04DBA00BF9AC30200014B586892
:1088A000704700BFD407002070B592B001240326A2
:1088B0000025414801A9ADF804408DF806608DF807
:1088C000075003F092FC3D4801A9ADF804608DF813
:1088D00006608DF8075003F088FC2046214603F01F
:1088E000EFFF21464FF4007003F0F6FF344803F029
:1088F00089F8344B32480793334B07A908938023F8
:108900000C934FF480730D934FF480630E932023E8
:108910000F934FF40053109309950A960B951195F8
:1089200003F0E0F82648214603F007F94FF46023EE
:10893000264802A9049302958DF80C408DF80D404D
:1089400005958DF8186002F0EBFE204808212246BC
:10895000334602F05DFF1D4829460222334602F0ED
:1089600057FF334619480921324602F051FF2A4683
:1089700016484FF4FC6102F012FF1448214602F041
:1089800005FF1248214602F0F8FE104802F010FFE1
:108990000E4802F012FF0028FAD10C4802F011FF35
:1089A0000A4802F013FF0028FAD10848012102F01A
:1089B00011FF12B070BD00BF00080140000C014063
:1089C000080002404C240140DC0700200024014044
:1089D0000828F8B507D009280DD0002858D13A4BFF
:1089E000188880B2F8BD384B588840F26B1380B2BB
:1089F00058430013F8BD344B988880B206F016FF38
:108A000006F0F8FA0022314B06F048FB22A3D3E926
:108A1000002306F043FB04460D4622462B461EA1CA
:108A2000D1E9000106F086F91DA3D3E9002306462B
:108A30000F462046294606F05BFC02460B463046B0
:108A4000394606F055FC06F0EBFD06F0D3FA00229D
:108A50001F4B06F04DFC07F095FD13A3D3E900234F
:108A600006F01CFB12A3D3E9002306F065F90246C9
:108A70000B4611A1D1E9000106F03AFC10A3D3E99D
:108A8000002306F057F906F0CBFD07F0EDF8F8BD2E
:108A90000020F8BDAFF300806666666666660A4031
:108AA0009A99999999990140C3F5285C8FA27240CF
:108AB0000000000000FEAA409A999999FD6F2F418D
:108AC000C3F5285C8F127140DC0700200000303FA6
:108AD00000002440AFF30080014B00221A60704771
:108AE000E4070020034B9B7A13B1034B05225A6025
:108AF000704700BFE00F0020E4070020014B042274
:108B00005A607047E4070020034B1A7A202A04BFFA
:108B100000221A72704700BFE40700207047212826
:108B200010B508D1104B1B681B7803F07F03212B75
:108B300010D0022010BD2028FBD10B4B0B4A1B6824
:108B40001B78107203F07F03212B094B18BF002301
:108B50000BB9EEE7074B044A0024126820469361E4
:108B600054829847204610BD40100020E4070020A2
:108B7000C58B0008AD8B0008074B1B681B7803F002
:108B80007F03212B06D100F0DF0002280CBF00205C
:108B900002207047022070474010002021B90228AF
:108BA00034BF0020022070470220704720B9034BD9
:108BB00008221B681A827047014870474010002045
:108BC0004800002020B9034B08221B681A82704716
:108BD00001487047401000204800002008B50320DD
:108BE00005F024FF064B0246D8604FF48871054813
:108BF00005F0CEFCBDE80840032005F096BD00BF9F
:108C0000E40700204610002038B5334B00241B68D1
:108C1000C0259C725D72DC72204605F0F5FC204692
:108C20004FF4007105F00DFD2046102105F020FDE8
:108C30002046402105F07CFE8021204605F067FE9D
:108C4000204605F09EFD254B204693F8341005F094
:108C5000BCFE204605F069FD0120214605F0F1FC2F
:108C60000120294605F053FE0120202105F000FDDA
:108C70000120214605F011FD02204FF4C06105F0EE
:108C8000E0FC02204FF4807105F041FE02202146F5
:108C900005F003FD0220202105F0EAFC0320214617
:108CA00005F0CFFC03204FF4887105F041FE03204E
:108CB000402105F08AFE03204FF4405105F0EDFC01
:108CC0000320214605F0D4FC204605F0FFFA044BB2
:108CD00001225A6038BD00BF40100020480000202B
:108CE000E4070020014905F0EBB800BF8000002038
:108CF000014905F0E5B800BF88000020054B1B685E
:108D0000DB78042B04D8044901EBC30105F0D8B883
:108D100000207047401000209000002008B501207E
:108D200003F058FDBDE808404FF40000012103F0B6
:108D3000DFBD024B03225A60704700BFE4070020EA
:108D4000044B9A7A044B0AB1052200E001225A60D2
:108D5000704700BFE00F0020E407002007B5142390
:108D60008DF8043000238DF805308DF8063001A809
:108D700001238DF8073003F043FB03B05DF804FBDB
:108D800018B10448102103F098BA0248102103F0EA
:108D900096BA00BF000C01407047684620F00701FA
:108DA0008D4679B5154D164B2A681C4692B21A802D
:108DB000144A188811881646014011F4806F05D0B6
:108DC0004FF6FF332B60104BDB68984723883288BF
:108DD0001340990507D54FF6FF532B600B4B197CB9
:108DE0000131C9B2197423881A40130401D505F062
:108DF000D5FABDE879408546704700BF445C004025
:108E0000D60F00208610002048000020E407002034
:108E100008B50848102103F050FA074B01221A60E8
:108E2000064A00200649186010604FF4E0520A809C
:108E30001A6008BD000C0140405C0040445C0040EA
:108E400086100020084B10B51B6800249C72FFF7A9
:108E5000DFFF064B064A1C604FF406431380054AA9
:108E60001360054B5C6010BD40100020445C004066
:108E700086100020405C0040E407002038B5064D15
:108E800001232B60054B00241C602046FFF778FF70
:108E900003232B60204638BD405C0040445C00400A
:108EA000074B1A6892B242F008021A601A6892B22E
:108EB00042F004021A60034B03225A60704700BF5D
:108EC000405C0040E407002010B5064C4FF6FB73F1
:108ED000226813402360FFF733FF4FF406432360FB
:108EE00010BD00BF405C004010B51E4C072818BFE5
:108EF00020702378052B32D8DFE803F003060A0E32
:108F00001621FFF7E1FF2AE0FFF7DEFF042327E049
:108F100002236370032323E06378013BDBB26370B9
:108F20006378F3B9042217E00F4B1A6892B242F04B
:108F300010021A60052323700A23637010BD637842
:108F4000013BDBB2637063785BB9074A4FF6EF739E
:108F500011680B4013600622024B1A7010BD0623E5
:108F6000237010BD44100020405C004007B5FFF79F
:108F7000D5FEFFF7F3FE05F0F5F90820012103F017
:108F8000ABFC10230322064801A9ADF804308DF88C
:108F900006208DF8073003F028F903B05DF804FBD4
:108FA000000C014007B514238DF8043000238DF820
:108FB00005308DF8063001A801238DF8073003F045
:108FC0001FFA03B05DF804FBFFF758BF0B4910B55B
:108FD000CA6882B14B68052B0CD10023CC68A34230
:108FE00004D2074C1C5DC4540133F7E7034B002146
:108FF000D96000E00022104610BD00BFE407002049
:1090000046100020084BDA68082A1A460AD90023BD
:109010000649595CC1540133092BF9D10023D360AF
:109020000120704700207047E40700204610002010
:1090300010B5084C0A46216092B2C02105F090FAA2
:109040000120218805F0A0FCBDE81040012005F0BA
:109050005DBB00BFE4070020704710B5FFF71EFCA2
:10906000074C2368C01AB0F5FA7F07D9054BDA68B8
:1090700082F40072DA60FFF711FC206010BD00BFBF
:1090800088100020000C01407047704770477047FF
:10909000054B064AD3F80310054B09B9928800E046
:1090A000128992B25A607047200A0020006C00407A
:1090B000940A002070477047704710B5FBF7FCF921
:1090C00005280E4C01D8012306E0FBF7F5F940F224
:1090D000F9339842F7D800236360094B1B7863B1DA
:1090E000084B62681A60084B1AB91A6842F0080205
:1090F00002E01A6822F008021A6010BD940A0020EB
:109100008F0A0020800A0020280A002070B505463A
:10911000C5F3074100220120FBF746FC0A4C06027A
:10912000C5F30721002201202660FBF73DFC3043F8
:1091300006020120E9B202462660FBF735FC304307
:109140000609266070BD00BFF807002038B5484CFE
:109150000B2303FB004203FB004311790433032973
:1091600084BF032111719A78032A84BF03229A7065
:109170000B2303FB004203FB0043117A04320F2947
:1091800084BF0F2111715A7A0433072A84BF072242
:109190005A710B2303FB004203FB0043917A043214
:1091A0000F2984BF0F2191715A7B0C330F2A84BF82
:1091B0000F225A700B2202FB004302FB0042997BF4
:1091C0000C330F2984BF0F21997013795279DB0377
:1091D00043F4002121611AB1254943F404230B61B2
:1091E0000B2101FB0041C979214B19B1196941F4E7
:1091F000005119610B2372B903FB0043197A9A7964
:10920000C90141EAC221043322695B790A4342EA77
:10921000031222611AE003FB00431B7B144A1BB1BB
:10922000136943F4805313610B2202FB0042917BCC
:10923000557B22690E4B42EAC51201F0070542EA4E
:109240000512090748BF42F400621A610B2202FBB3
:109250000040C27A064B04301AB91A6981790A4370
:109260001A612069FFF752FF2369636138BD00BFAF
:10927000F807002010B5114C0023C000236123180B
:109280005B7F13B14FF4007323612218927F0B4B65
:109290001AB11A6942F480721A612318DA7F2044E5
:1092A0000F2A84BF0F22DA77C07F23691843206119
:1092B000FFF72CFF2369236210BD00BFF8070020D1
:1092C00010B5224C4FF46023C0002361231893F89B
:1092D0002B3013B14FF470232361231893F825200A
:1092E00093F82410120342EA813293F82630216960
:1092F000012B42EA0102226103D1144B42F4806245
:109300001A61221892F82710236992F8282043EA5C
:109310000123012A236103D10C4A43F08003136126
:10932000221892F82920094B012A03D11A6942F028
:1093300040021A612044236990F82A0043EA001091
:109340002061FFF7E3FE2369E36210BDF807002008
:1093500038B52A4C43001A18224492F931103032A1
:109360003F29C4BF3F2151701A18224492F931108D
:1093700030323F31BCBFC12151701A18224492F8DB
:10938000321030321F2984BF1F2191704FF44022C8
:1093900022611A18224492F83020012A03D1174A78
:1093A0004FF45021116104EBC00191F82B10134AC6
:1093B00051B91918114491F83150116905F07F0520
:1093C00041EA052111610CE01D18154495F8315052
:1093D00001F0030105F07C052943156945EA0125E3
:1093E00015610344234493F8320023691843206134
:1093F000FFF78CFE2369636338BD00BFF8070020C8
:1094000010B58300244C1A18224492F83810012910
:1094100084BF012182F838101A18224492F83910BA
:109420003832032984BF032151701A18224492F85C
:109430003A1038320F2984BF0F2191701A18224434
:1094400092F83B103832032984BF0321D1701A18D7
:10945000224492F83C1003440F2902F1380284BFE1
:109460000F211171234493F83C0003F1380293F863
:10947000383040F4202040EAC330537840EA43308B
:10948000937840EA0320D37840EA43102061FFF745
:109490003DFE2369236410BDF8070020224B012004
:1094A00010B503220024052183F8300083F8290039
:1094B000022083F8264083F8274083F8284083F869
:1094C0002A0083F82B4083F8384083F8394083F82A
:1094D0003A4083F83B4083F83C405C779C77DC77EC
:1094E00018715C71DC719C711872DC721C735C7396
:1094F00083F8311083F8321083F8242083F8252074
:109500005A7299729A732046FFF77AFF2046FFF746
:109510001FFF2046FFF7D4FE2046FFF7ABFE204694
:10952000BDE81040FFF712BEF8070020054B0429E4
:1095300003EBC00318BF0022D97718BF5A77FFF793
:1095400099BE00BFF8070020044B03EBC003597716
:1095500009B10422DA77FFF78DBE00BFF8070020BB
:10956000024B03EBC0039977FFF784BEF807002096
:10957000024B03EBC000C07F704700BFF80700201C
:10958000024B03EBC000407F704700BFF80700208C
:10959000024B03EBC000807F704700BFF80700203C
:1095A000034B0B2202FB00331971FFF7CFBD00BF45
:1095B000F8070020034B0B2202FB00335971FFF721
:1095C000C5BD00BFF8070020034B0B2202FB003390
:1095D000D971FFF7BBBD00BFF8070020034B0B227A
:1095E00002FB00339971FFF7B1BD00BFF8070020FF
:1095F000034B0B2202FB00331972FFF7A7BD00BF1C
:10960000F8070020034B0B2202FB00335972FFF7CF
:109610009DBD00BFF8070020034B0B2202FB003367
:109620009972FFF793BD00BFF8070020034B0B2290
:1096300002FB00331973FFF789BD00BFF807002054
:10964000034B0B2202FB00335973FFF77FBD00BFB2
:10965000F8070020034B0B2202FB00339973FFF73E
:1096600075BD00BFF8070020024B0B2202FB003043
:1096700000797047F8070020024B0B2202FB0030F4
:1096800040797047F8070020024B0B2202FB0030A4
:10969000C0797047F8070020024B0B2202FB003014
:1096A00080797047F8070020024B0B2202FB003044
:1096B000007A7047F8070020024B0B2202FB0030B3
:1096C000407A7047F8070020024B0B2202FB003063
:1096D000807A7047F8070020024B0B2202FB003013
:1096E000007B7047F8070020024B0B2202FB003082
:1096F000407B7047F8070020024B0B2202FB003032
:10970000807B7047F8070020034A00EB8003134476
:1097100083F83810FFF774BEF8070020034B00EB06
:10972000800213445970FFF76BBE00BF3008002061
:10973000034B00EB800213449970FFF761BE00BF3A
:1097400030080020034B00EB80021344D970FFF770
:1097500057BE00BF30080020034B00EB80021344CB
:109760001971FFF74DBE00BF30080020034B00EB1E
:109770008000184490F83800704700BFF8070020B8
:10978000024B00EB800018444078704730080020FE
:10979000024B00EB800018448078704730080020AE
:1097A000024B00EB80001844C0787047300800205E
:1097B000024B00EB8000184400797047300800200D
:1097C000034A00EB4003134483F83010FFF7C0BD99
:1097D000F8070020034B00EB400213445970FFF7D9
:1097E000B7BD00BF28080020034B00EB4002134424
:1097F0009970FFF7ADBD00BF28080020034B00EBB8
:109800004000184490F83000704700BFF80700206F
:10981000034B00EB4000184490F90100704700BF73
:1098200028080020024B00EB400018448078704765
:1098300028080020034B03EBC00383F82410FFF734
:109840003FBD00BFF8070020034B03EBC00383F8C4
:109850002510FFF735BD00BFF8070020034B03EBD1
:10986000C00383F82610FFF72BBD00BFF8070020C8
:10987000034B03EBC00383F82710FFF721BD00BFA4
:10988000F8070020034B03EBC00383F82810FFF711
:1098900017BD00BFF8070020034B03EBC00383F89C
:1098A0002910FFF70DBD00BFF8070020034B03EBA5
:1098B000C00383F82A10FFF703BD00BFF80700209C
:1098C00010B5064B044603EBC00383F82B10FFF7DB
:1098D000F7FC2046BDE81040FFF73ABDF80700202E
:1098E000024B03EBC00090F824007047F8070020FB
:1098F000024B03EBC00090F825007047F8070020EA
:10990000024B03EBC00090F826007047F8070020D8
:10991000024B03EBC00090F827007047F8070020C7
:10992000024B03EBC00090F828007047F8070020B6
:10993000024B03EBC00090F829007047F8070020A5
:10994000024B03EBC00090F82A007047F807002094
:10995000024B03EBC00090F82B007047F807002083
:109960002DE9F0472E4D1E462B1893F8443004463F
:109970008A469146DDF82080099F042B1AD8DFE83B
:1099800003F003080D121700FFF7E0FB2B1901226B
:1099900012E0FFF795FC2B1902220DE0FFF730FDD6
:1099A0002B19032208E0FFF7D3FC2B19042203E054
:1099B000FFF760FC2B19002205EBC40483F8442058
:1099C00094F82A20164B012A13D002D3022A15D06C
:1099D00021E0BAF1000F03D01B689B0C8AF800301D
:1099E000B9F1000F17D02B68C3F38923A9F8003011
:1099F00011E086B11B689B0A33600CE01EB11B6846
:109A0000DB0B5B013360B8F1000F04D02B68C3F3AC
:109A1000842388F800300FB12B683B70BDE8F087D5
:109A2000F807002030B9044BDA7A1AB90122DA7249
:109A3000FFF78CBB704700BFF807002028B9034B25
:109A4000D97A11B1D872FFF781BB7047F8070020AF
:109A50002DE9F041114AC700D31993F82A60054651
:109A6000032E904604D0032283F82A20FFF728FC17
:109A70002846FFF725FCD8F80040230344BF6FEACF
:109A800004346FEA1434032E05D0474487F82A6063
:109A90002846FFF715FC2046BDE8F081F8070020B6
:109AA00070B5084C9DF810609DF8145004EBC0048C
:109AB00021766276A376E6762577BDE87040FFF7DB
:109AC000D9BB00BFF807002006281AD8DFE800F04D
:109AD00004070A0D101316000A4B1B6810E0094B0F
:109AE0001B6A0DE0074B5B690AE0064B1B6C07E045
:109AF000044B5B6B04E0034BDB6A01E0014BDB7A58
:109B00000B607047F8070020014B1878704700BFC2
:109B100040080020034B00201870034B997AFAF795
:109B200087BC00BF870F0020200F00202DE9F04FD9
:109B30008D4C87B0637823B96FF0004363600123D5
:109B40006370257A894F4DB9E8B2FAF722FC78554F
:109B50000135082DF8D1844B01221A7227250026E1
:109B6000F0B2FAF716FCBB5D83421AD07F4B321D70
:109B7000F0547F4B53F82230022B05D0032B0AD030
:109B8000012B0ED168B106E058B97A4A515D01291E
:109B900007D1535505E0774B5A5D012A04BF0222D5
:109BA0005A550136082E05F10105D9D1724EF369D7
:109BB00093B1724D2F787FB9FEF770FE704B1B6822
:109BC000C01AF3690028B8BF4042984204D9384609
:109BD00001F094F901232B70336AA3B1694D2E78FB
:109BE0008EB9FEF75BFE684B634A1B68126AC01AA7
:109BF00080EAE073A3EBE073934204D9304601F0AE
:109C00007DF901232B70607C604D574E05EB4013AE
:109C10001F7B002F00F0FB805D4B5E4F03440093E1
:109C2000C31901935C4B002103EB80030A46FFF745
:109C300097FE707C4301EA18127B013A042A00F275
:109C4000D480DFE802F0033AAF3AAF00534A544EF3
:109C5000926812F0200F04EB0002927C10D0022ACE
:109C600003D1325C002A00F0C0801D44697AFAF703
:109C7000DFFB607CFFF7E2FE637C0221E21818E064
:109C8000012A03D1325C002A00F0AF802B44997A7C
:109C9000FAF7CEFB607C05EB4015AB7A13B9FFF702
:109CA000C1FE03E0335C0BB1FFF7C8FE637C01210A
:109CB000E21891740022F25497E03A56384E002A86
:109CC00019DB2218927C022A01D1325C62B12B444A
:109CD000597AFAF7ADFB607CFFF7B0FE637C022196
:109CE000E21891740022F254667CFEF7D7FD04EB73
:109CF0008606706032E02044837C1B4F012B03D129
:109D0000637CF35C93B929E0FEF7C8FD7B7C0A21F4
:109D100007EB830705EB43139B8B7A684B43801A51
:109D200080EAE072A2EBE0729A42E9DD607C05EB2A
:109D30004013997AFAF77CFB607C05EB40139B7A21
:109D400013B9FFF76FFE03E0335C0BB1FFF776FE4C
:109D5000637C0121E21891740022F254637C05EBCC
:109D600043152B7B042B36E04008002049080020D7
:109D7000480F00208F0F002008000020850F0020D2
:109D8000800F0020A90E0020780F0020200F002057
:109D9000B20E0020190F0020C80E0020000C014058
:109DA000840F00202218927C954E022A01D1325C49
:109DB00062B12B44597AFAF73BFB607CFFF73EFE19
:109DC000637C0221E21891740022F254637C05EB5B
:109DD00043152B7B052B08D18A4B9A6812F0200F74
:109DE0004FF4806214BF5A611A61FEF757FD636930
:109DF000C01A80EAE073A3EBE0730A2B40F3F2820F
:109E0000FAF798FBFEF74AFD7F4B5861EAE2FAF752
:109E100091FBFAF709FD88B9367886B97B4F00F0D7
:109E2000ADFD304601F06AF83B7823B13046A97A9F
:109E3000FAF7FEFA3E700123237000E03770207EAF
:109E4000714F00F0E1FA00233B76FEF727FD6369CE
:109E5000C01A80EAE073A3EBE0730A2B40F3C282DE
:109E60003878002840F0B882797C490141F00A0135
:109E700001F0EA0100F00FFF0646787C002840F070
:109E8000028201F083F9787C0C22424360495F4FE3
:109E90008B18D3F804808A581B7ADFF87C91002B4A
:109EA00018BF90463B5C032B00F2C880DFE803F04C
:109EB00002611440002E00F0C18005EB4013D97FF1
:109EC00021B1FAF7B5FA637C03227CE0597AFAF7FC
:109ED000AFFA637C022276E06EB94E4B1B5C002B1E
:109EE0004BD1400140F0080101F0E801304600F09C
:109EF000D2FE002841D086EAE673A3EBE673B8F100
:109F0000000FB8BFC8F100084345607C02D0002EA6
:109F100040F0848059F83020934280F089803E4B95
:109F200003EBC0031979FAF783FA374B5B7C17E030
:109F300086EAE673A3EBE673B8F1000FB8BFC8F189
:109F40000008434501D0002E72D159F830209342C9
:109F500008D2314B03EBC0031979FAF769FA637C35
:109F6000012264E005EB4013597AFAF761FA637C49
:109F700043E056BB274B1B5CD3B1FEF78FFC637CE1
:109F80004FF00A0E04EB83025268801A05EB43126D
:109F9000918B0028B8BF40420EFB01F188424DDD95
:109FA0001846917AFAF744FA174B00225B7C0AE0D4
:109FB000400140F0080101F0E801304600F06BFE7E
:109FC0000028DAD001E0FA5438E086EAE673A3EB21
:109FD000E673B8F1000FB8BFC8F100084345607CD4
:109FE00000D0DEB959F83020934221D305EB40135D
:109FF000597AFAF71DFA044B5B7C022217E000BF86
:10A00000840F0020000C014040080020870F002032
:10A01000D00E00208E0F0020B40E002005EB401360
:10A02000D97F29B1FAF704FA864B03225B7CFA54F4
:10A03000677CFEF733FC04EB87077860607C824B1B
:10A04000002103440093814B0A4603440193804B53
:10A05000DFF8F08103EB8003FFF782FC607C7D4F2B
:10A0600005EB40139B694BB3FAF7D8F930B398F876
:10A07000110086EAE672A2EBE67207EB40139B69D9
:10A080009A421BD900F03AFF98F81130724A012128
:10A09000D15407EB43139B7F43B1BA7F9A4205D15A
:10A0A000002000F02BFF002000F068FC637C6B4A6E
:10A0B0000F33D15C012904BF0221D154627CDFF847
:10A0C000848151016B185B69DFF888A1002B6AD08D
:10A0D000634B9F5C9B46002F65D1002E64D041F0FE
:10A0E000020101F0E201384600F0BCFF024698F898
:10A0F00011000392FAF7DEFA98F81110039A0AEBAE
:10A1000041135B69101A80EAE072A2EBE07283EA05
:10A11000E37EAEEBE37E724554DD002B10DD084696
:10A1200000F0ECFE98F811300AEB43139B7F5BB311
:10A130009AF81E209A4227D1384600F0DFFE20E030
:10A140003846022200F0BFFD98F811103846490148
:10A1500041F0080101F0E80100F06AFD98F81130C3
:10A160000AEB43139B7F7BB19AF81E209A420BD1D6
:10A1700038463946022200F0A6FD3846082100F094
:10A1800057FD384600F0FAFB607C344A00F11503B5
:10A19000D15C012904BF0221D15401230BF8003006
:10A1A00000F0ECFB0EE06EB941F00801002001F078
:10A1B000E80100F070FD28B9637C05EB4312D289F9
:10A1C00062B10EE0677C274BDB5D002BF4D1FEF71C
:10A1D00065FB1C4B03EB8707F8611EE0214AD35C4B
:10A1E000DBB1FEF75BFB637C04EB8302D26905EB1A
:10A1F0004315801AE98980EAE072A2EBE0720A2036
:10A2000041438A4209DD184DEA5C32B91846FFF72E
:10A2100009FC0C4B01225B7CEA54607C002EB8BF29
:10A22000764259F83030074F9E42104D20D2FFF74A
:10A23000BFFA7B7C05EBC3056A79824223D11846BD
:10A2400000211EE040080020B20E0020190F00205F
:10A25000C80E0020200F0020180F00208F0F0020B4
:10A26000BD0E00208C0F00208D0F0020B40E0020AA
:10A27000FFF79EFA7B7C05EBC3056979884202D023
:10A280001846FFF769FA002000F0E9FC94F8202056
:10A29000C70702F0F802554B48BF42F001024607DB
:10A2A00083F8202005D594F8203043F0020384F889
:10A2B0002030C50605D594F8203043F0040384F817
:10A2C00020304B4B1A78D10716D594F82020D207AE
:10A2D00012D5484A1178CF070ED441F00101117010
:10A2E000454A117841F001011170444A0121117071
:10A2F000434A127802B91A7094F82030DE070AD562
:10A300003A4A92F82120D50705D43E4AD17801294E
:10A3100004BF0221D170990709D594F82120920732
:10A3200005D4384A1179012904BF022111715F0750
:10A3300009D594F82120560705D4324A51790129CC
:10A3400004BF02215171050684F82130617C43D598
:10A35000490141F01601002001F0F60105AA00F0C4
:10A3600083FC9DF81630580609D5204A2549527CB1
:10A3700052001B32885C012804BF02208854190651
:10A3800009D5617C1F4A0E3112F81100012804BF63
:10A39000022002F81100DA0608D5627C1949520041
:10A3A0001B32885C012804BF022088549B0609D513
:10A3B000627C144B0E3213F81210012904BF0221E3
:10A3C00003F81210617C0020490141F0160101F0F0
:10A3D000F60105AA00F07CFB044B00225A74FEF73C
:10A3E0005DFA606107B0BDE8F08F00BF4008002053
:10A3F000C40E0020B10E0020BE0E0020BE0F0020B3
:10A40000B00E00208F0F00202DE9F04FBB4D85B01E
:10A410002B5C0446002B00F0A2824FEA40195FFA41
:10A4200089F646F07C0103AA002000F01DFCB44B25
:10A43000600003EB0907397A022211F0400F9C46B5
:10A440007F689DF80E3002FA00F20DD04FF001083F
:10A4500008FA00F81A4003EA08085CF80930C7F166
:10A46000000AC3F1000B07E002EA03080122824060
:10A470005CF809B01A40BA46A24B11F0800F9B68F5
:10A4800001F03F0718BF83F02003791EC3F3401388
:10A49000072900F26482DFE811F0080008000800D4
:10A4A00008001B011B011B011B012B5D0F2B00F280
:10A4B0005682DFE813F05402100053013C007B0188
:10A4C000480051005D007000A100D900DE00540278
:10A4D000F80001013E0246F0140103AA002000F03A
:10A4E000C3FB46F006069DF80D3005EB84053146AA
:10A4F00000206B6000F0CFFB2146A8600222002004
:10A5000000F0E1FB0020314640F2FF7200F005FB55
:10A5100000202146032200F0F8FB023F012FDFF864
:10A52000DC8194BF0223042308F8043017E2002AD8
:10A5300000F01582002046F0020100F093FD724BFE
:10A5400043F8240029E1B8F1000F00F0088220460A
:10A5500000F0D4FC062301E221460020032200F093
:10A56000D4FB002046F00801524600F0D6FA46E13E
:10A57000B8F1000F40F0F38146F00806404631463E
:10A58000424600F0CAFA40463146CAF1000200F0E5
:10A59000C4FA0823E2E1B8F1000F00F0E08146F0D0
:10A5A0000201002000F05EFD07460020024646F052
:10A5B000080100F0B2FA544B002053F82420214641
:10A5C000D21B43F82420032200F09FFB002046F01A
:10A5D00006018AEAEA72A2EBEA7200F09EFA002013
:10A5E00009F0E0013A4600F0AAFA002021460246AE
:10A5F00000F069FB0923B1E1002000F030FB6300AB
:10A600001841C10740F1AB8146F0020841460020E5
:10A6100000F028FD3D4B46F0080643F824000020DA
:10A620000246314600F079FA00202146022200F06D
:10A630004AFB00200246414600F081FA0020024613
:10A6400009F0E00100F07BFA033F20460021FAF711
:10A6500045F8012F00F2788100202146022200F007
:10A6600032FB00203146F6E0B8F1000F40F00381E4
:10A6700075E1B8F1000F40F0728146F002014046EA
:10A6800000F0F0FC46F0080107464246404600F064
:10A6900044FA0222404609F0E00197FBF2F200F092
:10A6A0004EFA404612E1002000F0D9FA630018414A
:10A6B000C20740F1548147E105EB8407002046F0D2
:10A6C0000601BA6800F029FA002021463A7942E1F1
:10A6D000295D0F2900F24381DFE811F041011A00E2
:10A6E0003E00590066008200410193004101410192
:10A6F000C300CF00A900FE0038012B016408002030
:10A70000200F0020000C0140AC0E0020440F002060
:10A7100046F0140103AA002000F0A6FA9DF80D20CF
:10A7200005EB84035A6000202146022200F0CBFA98
:10A73000002046F0060140F2FF7200F0EEF9002022
:10A740002146032200F0E1FA062F51D0082F4FD006
:10A75000844B04221A5502E1062F09D105EB84032C
:10A760005A68002002F00402214642F0010204E08F
:10A77000082F04D100202146032200F0C6FA002051
:10A7800046F008015A4600F0C8F90323E6E0791FB5
:10A79000012904D81AB1062F2CD10423DEE0002BA6
:10A7A00000F0DD800C23D9E0052F09D105EB8403EF
:10A7B0005A68002002F00402214642F0020204E03E
:10A7C000072F04D100202146032200F09EFA00202A
:10A7D00046F00801CBF1000200F09FF90523BDE02F
:10A7E0007A1F012A08D8B8F1000F05D0052F01D132
:10A7F0000223B3E00F23B1E0002B00F0B080072369
:10A80000ACE0002B40F0AB80073F012F0AD905EBED
:10A8100084025268184602F00402214642F0010206
:10A8200000F073FA002046F00801524615E0002BB4
:10A8300040F09580073F012F0AD905EB840252684A
:10A84000184602F00402214642F0020200F05DFACE
:10A85000002046F00801CAF1000200F05EF90A2368
:10A860007CE0002B7BD0002046F0020100F0FAFBD8
:10A8700005EB8403D8600B2370E0002B6FD11846E2
:10A8800046F002018DE8081000F0ECFBDDF804C092
:10A89000009B0CEB09025373074646F0060118466D
:10A8A0008AEAEA72A2EBEA72009300F048F905EB3B
:10A8B0008402D268009B17440222184609F0E00186
:10A8C00097FBF2F200F03BF9009B18462146024646
:10A8D00000F0F9F90D2341E0002000F0C0F9630019
:10A8E0001841C3073BD50E232B5546F002052946D8
:10A8F000002000F0B7FB1C4B46F0080143F8240091
:10A900000020024600F009F921460020022200F052
:10A91000DAF900202946024600F011F9002009F07A
:10A92000E001024600F00BF920460021F9F7D6FEBF
:10A9300015E000202146022200F0C5F9002046F073
:10A940000801024600F0E9F80E2307E005EB840356
:10A950001A790020214600F0D8F900232B5505B0C4
:10A96000BDE8F08F64080020440F0020024B1A5C01
:10A970000AB901221A54704764080020024B1A5C7D
:10A980000AB10F221A54704764080020014B185C6A
:10A99000704700BF640800202DE9F041144612788A
:10A9A0000746C2F341150E466DBB444901EB451104
:10A9B00001F10803187930BBD00724D45F2A22D8CC
:10A9C0003F48405DF8B912F0970F1CD1DFF8F880CE
:10A9D00018F8050060B9C97F19B1F9F729FD0323FB
:10A9E00004E008465978F9F723FD022308F80530FA
:10A9F000DFF8D88018F805302BB10020FFF71EF8DB
:10AA0000002308F80530217800220220F9F7CCFF56
:10AA10003070617800220220F9F7C6FF7070A178CB
:10AA200000220220F9F7C0FFB07001220220E17875
:10AA3000F9F7BAFFF0702378DA073DD45F2B3BD8E3
:10AA400003F01E02082A12D0142A2BD0062A33D172
:10AA5000242257435B090C2202FB0373A178E2789E
:10AA6000184F42EA01223B445A60BDE8F08124219C
:10AA700079435B090C2000FB0313A678E578114AA3
:10AA800045EA0625D550A3781B0715D527787F09F9
:10AA900000FB0717D3596FEA03536FEA1353D351DF
:10AAA000BDE8F08124214F435B090C2101FB0373B6
:10AAB000044FE2783B441A72BDE8F081200F002079
:10AAC0008C0F0020D00E0020870F00208D0F00205B
:10AAD00007B513788DF800108DF80130537801A96F
:10AAE0008DF8023093786A468DF80330FFF754FFF3
:10AAF00003B05DF804FB07B58DF802309DF8103007
:10AB00008DF800108DF8012001A96A468DF80330F8
:10AB1000FFF742FF03B05DF804FB07B500238DF893
:10AB200000108DF801308DF80320131201A96A4638
:10AB30008DF80230FFF730FF03B05DF804FB5F29AA
:10AB40002DE9F34105460E46144658D811F01E076C
:10AB5000C1F3411202D0022F1DD050E000EB4003A0
:10AB60001A4430491201881843688C50C3EB040E14
:10AB7000BEF1000FB8BFCEF1000EBEF5000F08DB2E
:10AB80009C42CCBF284C294C0A441C44012313731B
:10AB900035E0077333E000EB4007224B17443F01D9
:10ABA000D91924F07F4EC1F808E04C6001F108008B
:10ABB000D9599846C4EB010EBEF1000FB8BFCEF1D3
:10ABC000000EBEF5000F18DBA142CCBF164B174B91
:10ABD000520123448DF800201A148DF801201A1216
:10ABE0008DF80220284601A96A468DF803304744B3
:10ABF000FFF7D2FE01233B7301E00023037123140E
:10AC00008DF801302846231201A96A468DF80060AC
:10AC10008DF802308DF80340FFF7BEFE02B0BDE8AC
:10AC2000F08100BF8C100020FFFF7F00010080FF3B
:10AC300007B511F01C0202D1FFF781FF0CE00023E1
:10AC40008DF800106A4601A98DF801308DF80230A8
:10AC50008DF80330FFF7A0FE03B05DF804FB01217F
:10AC600002200A46F9F7A0BE13B541F001011446CF
:10AC70008DF8041001AA6946FFF78EFE9DF8013099
:10AC80009DF8000023709DF8023063709DF803303A
:10AC9000A37002B010BD07B541F001018DF804109A
:10ACA00001AA6946FFF778FE9DF803309DF802007F
:10ACB00043EA0020030544BF6FEA00506FEA1050DA
:10ACC00003B05DF804FB73B54901CCB244F0150341
:10ACD000164601A96A4605468DF80030FFF75CFE6E
:10ACE0009DF8053044F014048DF801309DF80630CD
:10ACF000284601A96A468DF800408DF802308DF88B
:10AD00000360FFF749FE02B070BD73B54901CCB2D4
:10AD100044F01503164601A96A4605468DF8003031
:10AD2000FFF73AFE9DF8053044F014048DF8013029
:10AD30009DF80730284601A96A468DF800408DF835
:10AD400002608DF80330FFF727FE02B070BD2DE9D9
:10AD5000F3474001C7B2C1F30A06002047F01801CB
:10AD600001AAFFF781FF9DF8058030464FEA1819C8
:10AD700008F00F08C8450FDB04F01AF9C9EB080802
:10AD80000446012000FA08F00D4604F021F90022E3
:10AD9000354B04F083F910E004F00AF9C8EB090818
:10ADA0000446012000FA08F00D4604F011F90246AD
:10ADB0000B4600202C4904F09BFA02460B46204625
:10ADC000294604F095FA04F02BFC04F013F924A3AF
:10ADD000D3E9002304F062F904F022FC04F00AF93C
:10ADE0000022224B04F05AF94FF0FF3904460D4679
:10ADF000CA464FF00008012000FA08F004F0E8F815
:10AE000002460B462046294604F048F904F0E0FBD0
:10AE1000A0F18002802A38BFC14608F1010828BF8E
:10AE20005046B8F10E0F01D08246E4E700248DF8B9
:10AE3000050047F01201204601AA8DF804408DF864
:10AE40000690FFF745FE204647F00C013246FFF71B
:10AE500064FE204602B0BDE8F08700BFAFF300807B
:10AE600004560E2DB29DEF3F0000604000002040D0
:10AE700073B54C0804EB4404B42304F5807403FB5D
:10AE80000044054620460E46FDF712F98DF80400F1
:10AE9000601CFDF70DF98DF80500A01CFDF708F901
:10AEA00046EA45118DF80600C9B2002001AAFFF755
:10AEB0000FFE02B070BD37B50C46640841EA401180
:10AEC00001AA0546C9B2002004EB4404FFF7CCFEFA
:10AED00004F58074B42303FB05449DF80410204658
:10AEE000FDF70DF8601C9DF80510FDF708F8A01C93
:10AEF0009DF80610FDF703F803B030BD10B5C4B2DD
:10AF000021466401E4B200200222FFF7DCFE44F097
:10AF100008010020FFF78CFE44F00A010020BDE884
:10AF20001040FFF785BE37B5400140F01604E4B28B
:10AF30000D4601AA21460020FFF796FE9DF8053038
:10AF400015F0010F14BF43F0400323F040038DF8C8
:10AF500005309DF8053015F0020F14BF43F01003C3
:10AF600023F010030020214601AA8DF805308DF84A
:10AF70000600FFF7ADFD03B030BD37B5400140F02E
:10AF80001604E4B20D4601AA21460020FFF76CFE2C
:10AF90009DF8053015F0010F14BF63F07F0303F037
:10AFA0007F038DF805309DF8053015F0020F14BFB2
:10AFB00043F0200323F020030020214601AA8DF84E
:10AFC00005308DF80600FFF783FD03B030BD07B5EF
:10AFD000400140F0160101F0F60101AA0020FFF740
:10AFE00043FE9DF80530C3F38010DB0648BF40F0F8
:10AFF000020003B05DF804FB07B5400140F0160104
:10B0000001F0F60101AA0020FFF72EFE9DF80530A1
:10B01000D8099B0648BF40F0020003B05DF804FB6E
:10B0200070B50F4C000123189A68914209DD8A1A05
:10B03000C2F18075AA425E6801DC324409E0751BEA
:10B040000AE00ADA521AC2F18075AA425E6802DC8E
:10B05000B21A5A6001E035445D602044816070BDE1
:10B060008C10002037B541F001030C4601AA694657
:10B070008DF804300546FFF78FFC9DF802309DF8EF
:10B0800001201B0243EA02439DF8032043EA020128
:10B090000B0248BF41F07F415F2C19D8C4F3411225
:10B0A00014F01E040ED0022C12D105EB45051544F8
:10B0B000E8B221F07F41FFF7B3FF074B03EB051523
:10B0C000696805E005EB45052A44034B12019958D0
:10B0D000084603B030BD00BF8C10002038B50C46C8
:10B0E00068210546FFF7BEFF14B140F0010201E000
:10B0F00020F0010228466821BDE83840FFF71FBD57
:10B1000038B50C4668210546FFF7ACFF14B140F096
:10B11000100201E020F0100228466821BDE8384006
:10B12000FFF70DBD13B5184B00245A7E93F8283055
:10B1300012F0010F14BF21222022DB0748BF42F08A
:10B14000100200206821FFF7FAFC009420467E21BF
:10B1500020222346FFF7CFFCE1B200200134FFF7A5
:10B1600087FE1D2CF8D10C210020FFF77BFF014644
:10B170000020FFF7ECFD0020162143F2FF1202B081
:10B18000BDE81040FFF7C9BC08000020F0B545013C
:10B1900085B0044645F0030303AA002002A98DF8F8
:10B1A0000C30FFF7F9FB9DF80A109DF809300902F1
:10B1B00041EA03419DF80B3020461943FFF730FF69
:10B1C00015482301C21802F108010E790EB3134E7F
:10B1D0000C2707FB0464247ADCB9C6585268B71AF6
:10B1E000002FB8BF7F42B7F5000F05DB9642CCBFFA
:10B1F0000B4B0C4B134401E0C3580C71DAB20092B4
:10B200000020C3F3074205F0E001C3F30723FFF773
:10B2100072FC05B0F0BD00BF8C100020D00E0020E5
:10B22000FFFF7F00010080FF074B10B518681C4628
:10B2300001460A780B4601311AB12C2AF9D10022B5
:10B240001A700133236010BD7408002070B5124BD2
:10B2500006461B78E3B1FDF7F9F8104C054618B126
:10B2600000232371012070BDA368E268934207D2D6
:10B270005A1C23441B7C012033702071A26070BDD6
:10B2800004F11000FDF7A2FEA560E060284670BD45
:10B29000BDE87040FDF7DAB8A80E00207408002061
:10B2A00010B50E4B1B7813B10D4C23791BB9BDE8BB
:10B2B0001040FDF7B1B8226D0D2802F101032244C0
:10B2C000236582F8540002D03F2B00D829B91946D3
:10B2D0000448FDF7ADFE0023236510BDA80E002035
:10B2E00074080020C808002070B50121044686B00B
:10B2F0002020FFF7D5FF002C04DA2D200121FFF7D5
:10B30000CFFF644200230A2194FBF1F201FB1241BA
:10B3100001AE30311D46995514460133002AF2D151
:10B32000705D0121FFF7BCFF15F1FF35F8D206B0C3
:10B3300070BD2DE9F34105460DF10700FFF786FFCB
:10B34000974C002800F0C88094F894309DF80700CE
:10B35000944E03BB7378403398420DD1D4F89830A3
:10B36000002B40F0B9803179012331F0010184F8DC
:10B37000943040F0B180ADE00D2801D01B2801D100
:10B38000002305E0D4F898307E2B00F2A58001332D
:10B39000C4F89830A0E0317931F0010101D1FFF714
:10B3A0007FFF9DF807301F2B0CD9D4F898207C49DB
:10B3B0007E2A00F28280501C0A44C1F8980082F86C
:10B3C0009C307AE0082B08D1D4F89830002B74D048
:10B3D000734A013BC2F898306FE00D2B6DD1D4F861
:10B3E0009830002B69D03379112B16D16D4B012188
:10B3F000587800274030C0B2FFF752FFD4F8983099
:10B400009F4206D2684B0121D85DFFF749FF013703
:10B41000F4E70D200121FFF743FF0023D4F89880C3
:10B420002768C4F81C311A461946424537D001290D
:10B4300011D002D3022925D02FE0DFF864C10CF12E
:10B440009C00105C202828D00CEB030181F820011F
:10B450000133012121E0524800F19C0C12F80CC08C
:10B46000BCF1200F0AD1012B04D91844002180F827
:10B47000201101334D4F02211F440EE0184480F883
:10B4800020C109E0DFF818C10CF19C00105C2028F5
:10B4900003D09C448CF8200101330132C5E700221F
:10B4A000C4F81C31234483F820210123276084F849
:10B4B0009F3184F89420C4F898209DF807301B2B06
:10B4C0000AD133790021012BC4F8981084F8941024
:10B4D00002D10D20FFF7E4FE94F89F01002600281A
:10B4E0005AD02F4B83F89F61F7B2DFF8DC80C7EBAF
:10B4F000C70708EB07042D48214604F08BFF28B945
:10B50000A6796379F1072B7036D506E018F8073075
:10B510000136002BE8D12B703DE0FFF785FE2B783C
:10B520000446042B14D1224904F074FF08B9002307
:10B530000CE020461F4904F06DFF08B9012305E027
:10B540001D49204604F066FF90B902236B7013E09A
:10B550000D2B0ED1194904F05DFF0028E7D02046DD
:10B56000174904F057FF0028E8D020461549E9E7BD
:10B57000204604F04BFF6870B20704D5FFF754FE75
:10B5800004F044FFA870730705D5FFF74DFE04F0E3
:10B590003DFFC5F80300012002B0BDE8F08100BF07
:10B5A00074080020080000201009002094090020E1
:10B5B000C20C0108C60C0108CA0C0108D00C010815
:10B5C000D60C0108DB0C0108C50B010838B50D4D80
:10B5D0000446A87801214030C0B2FFF761FE6878C8
:10B5E00001214030C0B2FFF75BFE2078FFF77CFE00
:10B5F0006068FFF779FEBDE838400D200121FFF7B4
:10B600004FBE00BF080000207047FEE7FEE7FEE7E0
:10B61000FEE7704770477047704770477047704744
:10B620007047704770477047704770477047704762
:10B63000704770477047704770477047704708B54C
:10B64000014B1B68984708BDC00E002008B5024B8F
:10B650001B68984708BD00BF880F002008B5024B43
:10B660001B68984708BD00BF1C0F002008B5024B9F
:10B670001B68984708BD00BF400F00207047704707
:10B680007047704770477047704770477047704702
:10B6900070477047704770477047704770477047F2
:10B6A00070477047704770477047704770477047E2
:10B6B00070477047704770477047704770477047D2
:10B6C00070477047704700BF08B5144B98420FD0C1
:10B6D00003F5A053984213D0A3F5C05398421BD151
:10B6E0004FF40070012101F00FF94FF400700EE0EB
:10B6F0004FF48060012101F007F94FF4806006E00B
:10B700004FF40040012101F0FFF84FF40040002108
:10B71000BDE8084001F0F8B808BD00BF00280140AE
:10B7200043680A6823F4702323F4807313430A796F
:10B7300010B543EA022343608A68CB6884681A43E1
:10B74000084B234013434A7943EA420383600B7C4E
:10B75000C26A013B22F47002DBB242EA0353C362C5
:10B7600010BD00BFFDF7F1FF0023036003714371BB
:10B770008360C360012303747047836811B143F091
:10B78000010301E023F0010383607047836811B176
:10B7900043F4807301E023F4807383607047C9B27F
:10B7A00043680AB1194301E023EA0101416070478F
:10B7B000836843F00803836070478068C0F3C0006B
:10B7C0007047836843F00403836070478068C0F368
:10B7D00080007047836811B143F4A00301E023F4B3
:10B7E000A003836070478068C0F38050704743684F
:10B7F000013923F4604343EA4133436070474368AF
:10B8000011B143F4006301E023F400634360704727
:10B81000092970B50DD9A1F10A0404EB44040725E8
:10B82000A540A340C66826EA050545EA0304C460AE
:10B830000BE001EB41040725A54003FA04F4066977
:10B8400026EA050545EA04030361062A0CD8013AF5
:10B8500002EB82021F23934001FA02F2446B24EAB6
:10B8600003031A43426370BD0C2A0CD8073A02EB5B
:10B8700082021F23934001FA02F2046B24EA0303BD
:10B880001A43026370BD0D3A02EB82021F239340FC
:10B8900001FA02F2C46A24EA03031A43C26270BDC9
:10B8A000836811B143F4801301E023F480138360B3
:10B8B0007047C06C80B27047014B1868704700BF7A
:10B8C0004C240140436811B143F4806301E023F448
:10B8D000806343607047436811B143F4805301E0D3
:10B8E00023F4805343607047836823F4E043194393
:10B8F00081607047836811B143F4004301E023F491
:10B90000004383607047836811B143F4021301E080
:10B9100023F40213836070478068C0F3405070477F
:10B92000092970B50DD9A1F10A0404EB44040725D7
:10B93000A540A340C66826EA050545EA0304C4609D
:10B940000BE001EB41040725A54003FA04F4066966
:10B9500026EA050545EA04030361846B931CC4F3DE
:10B9600001555B1BDBB203EB83031F229A40994016
:10B9700024EA020444EA0103836370BD836B013946
:10B9800023F4401343EA01538363704742507047E6
:10B990002831405880B27047436823F4400323F4B1
:10B9A0000073194341607047416282627047436887
:10B9B00023F01F03194341607047054B9A6810B18B
:10B9C00042F4000201E022F400029A60704700BFD6
:10B9D00000240140036819420CBF00200120704779
:10B9E000C943016070474368006810EA112004D021
:10B9F000C9B219420CBF0020012070476FEA112123
:10BA000001607047036823F00103036000230360B3
:10BA100043608360C3602D4B984234D011D83C3BC7
:10BA200098422AD006D8283B984222D01433984214
:10BA300021D07047264B984221D01433984220D011
:10BA40007047244B98422DD008D8A3F567739842CD
:10BA50001ED003F5627398421FD070471E4B984268
:10BA600029D0143398422BD0283B98422DD11B4B20
:10BA70001DE01B4B12E01A4B15E0194B17E0184B59
:10BA80001AE0174B1DE0164B5A6842F470021BE097
:10BA9000134B5A6842F0706216E0104B5A6842F03D
:10BAA0000F0211E00D4B5A6842F0F0020CE05A68A8
:10BAB00042F4706208E0094B5A6842F4704203E0B5
:10BAC000064B5A6842F470225A6070476C0002407C
:10BAD000440002401C0402404404024000040240AE
:10BAE000000002408A6810B50C6A036814430A69B2
:10BAF00023F4FF4314434A6923F0700314438A6913
:10BB00001443CA6914434A6A14438A6A224313439A
:10BB10000360CB6843600B6883604B68C36010BDF3
:10BB20000023036043608360C360036143618361FA
:10BB3000C3610362436283627047036811B143F0DB
:10BB4000010301E023F001030360704703680AB1B9
:10BB5000194301E023EA010101607047406880B2A7
:10BB60007047C3004CBF044B044B1B6803420CBF1F
:10BB700000200120704700BF000402400000024086
:10BB8000C3004CBF014B024B586070470004024099
:10BB900000000240C3004CBF034B044B1B68034230
:10BBA0000CBF00200120704700040240000002404A
:10BBB000C3004CBF014B024B586070470004024069
:10BBC00000000240044B00221A605A609A60DA605A
:10BBD000024A5A61704700BF00040140FFFF07009E
:10BBE000837930B50168027943B3194BCC431D68A2
:10BBF00002F1804225401D605D6802F582322C40D2
:10BC00005C6014682143116002689C68D1430C4059
:10BC10009C60DC682140D9604179102906D199687F
:10BC200011439960D9680A43DA6030BD01F180435D
:10BC300003F5823319680A431A6030BD02F180436C
:10BC400003F582331A6822EA0101196030BD00BF92
:10BC50000004014000230C220360037142718371D0
:10BC60007047024B1A691043186170470004014085
:10BC7000034B5B6918420CBF00200120704700BFD6
:10BC800000040140014B5861704700BF00040140AF
:10BC9000054B1A685B69034004D010420CBF0020BA
:10BCA000012070471846704700040140014B58615D
:10BCB000704700BF00040140044B1A6802F03802CC
:10BCC0001A601A6810431860704700BF00200240D5
:10BCD000044B1A6822F008021A601A6810431860B0
:10BCE000704700BF00200240044B1A6822F0100287
:10BCF0001A601A6810431860704700BF00200240A5
:10BD0000034B044A5A6002F188325A60704700BF00
:10BD10000020024023016745024B1A6942F080026D
:10BD20001A61704700200240014BD86980087047B3
:10BD300000200240014B186A704700BF00200240FB
:10BD4000024BD869C0F34000704700BF002002409A
:10BD5000024B1868C0F34010704700BF002002403B
:10BD6000044B1A6909B1104301E022EA000018618E
:10BD7000704700BF002002400128064B03D1D8695C
:10BD800000F001007047DB6818420CBF0020012062
:10BD9000704700BF00200240014BD860704700BFD1
:10BDA00000200240084BDA68D10709D4DA6852074C
:10BDB00008D4DB6813F0100F0CBF04200320704779
:10BDC00001207047022070470020024013B504464E
:10BDD000FFF7E8FF01280FD164B100230193FF238F
:10BDE0000193019B13B1019B013BF9E7FFF7DAFFD8
:10BDF000013CEFE7052002E0002C08BF052002B05F
:10BE000010BD38B5054640F6FF70FFF7DFFF042888
:10BE100014D10B4C40F6FF70236943F002032361F9
:10BE20006561236943F040032361FFF7CFFF0128D9
:10BE300004D0226941F6FD731340236138BD00BF71
:10BE40000020024010B540F6FF70FFF7BFFF042846
:10BE500013D10A4C40F6FF70236943F004032361B9
:10BE6000236943F040032361FFF7B0FF012804D0AA
:10BE7000226941F6FB731340236110BD002002408C
:10BE800010B540F6FF70FFF7A1FF042829D1154C2B
:10BE9000154B40F6FF70A36003F18833A36023695C
:10BEA00043F020032361236943F040032361FFF73C
:10BEB0008DFF04280ED1226941F6DF731340236100
:10BEC0002369A52243F010032361084B0F201A8039
:10BED000FFF77CFF012804D0226941F6EF7313407D
:10BEE000236110BD002002402301674500F8FF1FB9
:10BEF00070B505460F200E46FFF768FF042817D1DE
:10BF00000C4C0F20236943F001032361B3B22B8053
:10BF1000FFF75CFF042804D1360C6E800F20FFF77A
:10BF200055FF012804D0226941F6FE7313402361B6
:10BF300070BD00BF0020024070B505460F200E46C0
:10BF4000FFF744FF04280FD1084C0F20236943F06A
:10BF5000010323612E80FFF739FF012804D02269F5
:10BF600041F6FE731340236170BD00BF0020024004
:10BF700070B505460F200E46FFF728FF042814D1A0
:10BF80000A4C0B4B0F20A36003F18833A360236995
:10BF900043F0100323612E80FFF718FF012804D01F
:10BFA000226941F6EF731340236170BD0020024007
:10BFB0002301674510B504460F20FFF707FF04284B
:10BFC0003ED1204B2049E443996001F188319960CA
:10BFD0001969E2B241F01001FF2A196104D1C4F3DA
:10BFE0000723FF2B08D10EE0184B0F201A81FFF713
:10BFF000EDFE04281CD1F2E7144A0F205381FFF70D
:10C00000E5FE042814D1C4F30743FF2B06D00F4AE2
:10C010000F209381FFF7DAFE042809D1240EFF2CAC
:10C0200001D1042006E0094B0F20DC81FFF7CEFE92
:10C03000012805D0034A41F6EF7311690B401361E3
:10C0400010BD00BF002002402301674500F8FF1F1C
:10C0500038B5054640F6FF70FFF7B8FE042836D124
:10C060001B4C1C4B40F6FF70A36003F18833A360A8
:10C07000236943F020032361236943F040032361D4
:10C08000FFF7A4FE04281BD1226941F6DF73134099
:10C090002361236943F0100323610F4B0DB100228C
:10C0A00000E0A5221A8040F6FF70FFF78FFE0128FE
:10C0B0000DD0074A41F6EF7311690B40136138BD8B
:10C0C000012804D0226941F6DF731340236138BD93
:10C0D000002002402301674500F8FF1FF8B5114C0E
:10C0E000114B0546A36003F18833A3600F200E4671
:10C0F0001746FFF76BFE042813D1236947F0F807B2
:10C1000043F0100323613E43084B35435D800F200D
:10C11000FFF75CFE012804D0226941F6EF7313405B
:10C120002361F8BD002002402301674500F8FF1F8E
:10C1300008B5264B98422FD011D8A3F5006398423A
:10C140001ED003F58063984220D0A3F50063984287
:10C150003AD10420012100F0D7FB04202FE01C4B32
:10C1600098421FD003F58063984221D0A3F5006365
:10C17000984229D14020012100F0C6FB40201EE05A
:10C180000820012100F0C0FB082018E01020012148
:10C1900000F0BAFB102012E02020012100F0B4FBD7
:10C1A00020200CE08020012100F0AEFB802006E082
:10C1B0004FF48070012100F0A7FB4FF48070002144
:10C1C000BDE8084000F0A0BB08BD00BF001401405E
:10C1D000001C014008B50120014600F095FBBDE8B8
:10C1E00008400120002100F08FBBCB78F0B5DA06C3
:10C1F00048BF8A78098803F00F0548BF154311F03E
:10C20000FF0F1DD0046800220127974007EA0106AE
:10C21000BE4211D197004FF00F0C0CFA07FC05FA43
:10C2200007F724EA0C04282B44EA070401D14661ED
:10C2300002E0482B08BF06610132082AE4D10460FD
:10C24000FF291FD94468002202F108060127B740E0
:10C2500007EA0106BE4211D197004FF00F0C0CFA0D
:10C2600007FC05FA07F724EA0C04282B44EA070424
:10C2700001D1466102E0482B08BF06610132082A5D
:10C28000E2D14460F0BD4FF6FF7303800223837058
:10C290000423C3707047836819420CBF002001203B
:10C2A0007047806880B27047C36819420CBF002095
:10C2B00001207047C06880B27047016170474161DA
:10C2C00070470AB10161704741617047C1607047B2
:10C2D00041F480338361816183618369836970473D
:10C2E000054B1A6822F07F021204120C114341EA36
:10C2F00000101860704700BF00000140014B18603B
:10C30000704700BF1C00204230B5134A00F44015AE
:10C31000B5F5401F536884B206D1556823F07063A9
:10C3200025F0706555600FE0C20205D5C0F30342E9
:10C33000032505FA02F203E0420D120104FA02F2AB
:10C3400023EA020343F0706319B1400D00018440F9
:10C350002343014A536030BD0000014001F0030354
:10C360009B000F229A40984001F0FC0101F18041AE
:10C3700001F5803110B58C6824EA02028A608A686F
:10C3800002438A6010BD00BF0B4B6FF070424FF04C
:10C39000FF31C3F88010C3F88420C3F88011C3F8BC
:10C3A0008421002202F1C001013200200F2A43F84B
:10C3B0002100F7D1704700BF00E100E0094B4FF0CA
:10C3C000206209495A6000229A60D9601A615A6154
:10C3D0009A61DA611A625A624FF0FF329A62DA6247
:10C3E0001A63704700ED00E00000FA0540F0BF60FE
:10C3F000024B40F40030D860704700BF00ED00E011
:10C40000C27830B503785AB31B4A4478D26885782D
:10C41000D243C2F30222C2F1040104FA01F10F2453
:10C42000D4402C400C4303F00301C9002401FF2237
:10C430008C408A4003F0FC0303F1604303F5614341
:10C44000D3F8005325EA020122400A43C3F800232F
:10C4500003780122590903F01F0302FA03F306E0EF
:10C460005909012203F01F0302FA03F32031034AA2
:10C4700042F8213030BD00BF00ED00E000E100E0F7
:10C480000023037043708370C3707047F7F765BE75
:10C49000F7F765BEF7F765BEF7F765BE0001F7F77A
:10C4A00064BEF7F765BE024B5868C0F309307047A9
:10C4B00000ED00E000F01F03012202FA03F340093F
:10C4C000044A403052F820001840C31A58425841DC
:10C4D000704700BF00E100E0014B1860704700BFEB
:10C4E00000EF00E04209012300F01F0003FA00F012
:10C4F000024B603243F82200704700BF00E100E0C9
:10C50000024B5868C0F30900704700BF00ED00E01F
:10C5100000F01F03012202FA03F34009044A8030AD
:10C5200052F820001840C31A58425841704700BFC3
:10C5300000E100E0014B1868704700BF00ED00E02B
:10C5400021F0604121F07F01014B08439860704762
:10C5500000ED00E0014A024BDA6070470400FA0582
:10C5600000ED00E0014A024BDA6070470100FA0575
:10C5700000ED00E0044B1A6909B1104301E022EA22
:10C5800000001861704700BF00ED00E0012300F0DB
:10C590001F0003FA00F0044B5A6A09B1104301E08E
:10C5A00022EA00005862704700ED00E0114B30B500
:10C5B000DB68DB43C3F30223C3F10404A140FF247F
:10C5C00024FA03F31A401143C0F30122D20094402D
:10C5D000090101FA02F2C0F38110800000F160400D
:10C5E00000F56D40836923EA0404846185692A4368
:10C5F000826130BD00ED00E0C0F383200123834061
:10C60000034A506A1840C31A58425841704700BF45
:10C6100000ED00E000F01F00012101FA00F0024BE4
:10C620005A6802435A60704700ED00E000F01F00B6
:10C63000411E012000FA01F1024B5A680A435A6078
:10C64000704700BF00ED00E0C0F38330012383405A
:10C65000034A506A1840C31A58425841704700BFF5
:10C6600000ED00E0C0F38142094B0AB9D86A704777
:10C67000012A0AD1C0F30152986AD300D840022A95
:10C6800014BF00F00F00C0B27047186B704700BFB6
:10C6900000ED00E0034B10F4800F0CBF586B986B5B
:10C6A000704700BF00ED00E00C4B1A6842F0010239
:10C6B0001A6059680A4A0A405A601A6822F084725D
:10C6C00022F480321A601A6822F480221A605A68B2
:10C6D00022F4FE025A6000229A6070470010024065
:10C6E0000000FFF80C4BB0F5803F1A6822F480324E
:10C6F0001A601A6822F480221A6003D0B0F5802FE5
:10C7000004D070471A6842F4803202E01A6842F49A
:10C71000A0221A60704700BF00100240034B1A6845
:10C7200022F0F80242EAC000186070470010024090
:10C73000014B1860704700BF00004242034B5A682B
:10C7400022F47C12114308435860704700100240E5
:10C75000014B1860704700BF60004242034B5A68AB
:10C7600022F0030210435860704700BF00100240DF
:10C77000024B586800F00C00704700BF00100240E8
:10C78000034B5A6822F0F00210435860704700BF14
:10C7900000100240034B5A6822F4E06210435860D4
:10C7A000704700BF00100240034B5A6822F46052E9
:10C7B00042EAC0005860704700100240044B1A78EB
:10C7C00009B1104301E022EA00001870704700BF71
:10C7D00009100240014B1860704700BFD800424268
:10C7E000034B5A6822F4404210435860704700BF20
:10C7F00000100240064B002201281A701A7002D065
:10C80000042802D070471870704705221A707047CC
:10C8100020100240014B1860704700BF8004424264
:10C82000024B1A6A10431862704700BF00100240A2
:10C83000014B1860704700BF3C0442421C4B10B5CE
:10C840005A6802F00C02042A01D0082A01D0194AC1
:10C850000EE05A685968C2F38342CC0302F1020227
:10C8600002D55968890301D5134900E011494A43AB
:10C8700002605968114AC1F30311545C0168E14038
:10C8800041605C68C4F30224145D21FA04F48460FE
:10C890005C68C4F3C224145DE140C1605B68C3F30B
:10C8A00081331A44137CB1FBF3F1016110BD00BF69
:10C8B0000010024000127A0000093D00A50C01089A
:10C8C000044B5A6909B1104301E022EA00005861A3
:10C8D000704700BF00100240044B9A6909B1104331
:10C8E00001E022EA00009861704700BF001002409A
:10C8F000044BDA6909B1104301E022EA0000D86173
:10C90000704700BF00100240044BDA6809B11043C1
:10C9100001E022EA0000D860704700BF001002402A
:10C92000044B1A6909B1104301E022EA00001861C2
:10C93000704700BF00100240014B1860704700BFF5
:10C9400040044242014B1860704700BF4C00424215
:10C95000014B1870704700BF071002404309012BBC
:10C96000074A01D1136803E0022B0CBF136A536A14
:10C9700000F01F0023FA00F000F00100704700BF34
:10C980000010024008B53120FFF7E8FF094B18708E
:10C990005A6801325A601A7822B95A6840F2FF1375
:10C9A0009A42F0D13120FFF7D9FF003018BF0120A3
:10C9B00008BD00BF140A0020024B5A6A42F0807280
:10C9C0005A62704700100240034B9B6818420CBF2C
:10C9D00000200120704700BF00100240014B18707A
:10C9E000704700BF0A10024008B5164B98421BD092
:10C9F00003F5744398420BD0A3F5784398421FD1B6
:10CA00004FF480400121FFF78BFF4FF4804012E08C
:10CA10004FF480500121FFF777FFBDE808404FF445
:10CA200080500021FFF770BF4FF400400121FFF755
:10CA300077FF4FF400400021BDE80840FFF770BFCA
:10CA400008BD00BF003C00400B8810B54C88028830
:10CA500023438C8802F441522343CC8823430C891E
:10CA600023434C8923438C892343CC892343134399
:10CA70009BB20380838B23F400631B041B0C838312
:10CA80000B8A038210BD838BF0B523F47B6323F004
:10CA90000F031B041B0C8383022303840B89868BE7
:10CAA000022B87B005460C46B6B223D08B8801A86E
:10CAB000002B14BF02270127FFF7C0FEE38822895D
:10CAC000B3F5007F019B4FF00A011CBF7F017A4341
:10CAD00001FB03F308BF1202B3FBF2F305330A2292
:10CAE0009BB2B3FBF2F303F001021202C3F34F0354
:10CAF00092B200E00022991E89B2FE2928BF0022CE
:10CB0000E18828BF022313430B439BB22B84238865
:10CB10006288334343F400631343A288134362895A
:10CB200013439BB2AB8307B0F0BD00230380438067
:10CB30008380C380038143818381C3810723038270
:10CB4000704700230222038043808380C3800281D8
:10CB500043817047038819B19BB243F0400303E05F
:10CB600023F040031B041B0C03807047838B19B117
:10CB70009BB243F4806303E023F480631B041B0C2B
:10CB800083837047090901238B409BB21AB18288C5
:10CB900092B2134303E0828892B222EA03038380B5
:10CBA000704783889BB20AB1194301E023EA01016F
:10CBB0008180704781817047808980B270474FF6CD
:10CBC000FF639942038803D09BB243F4807303E070
:10CBD00023F480731B041B0C03807047838819B1F6
:10CBE0009BB243F0040303E023F004031B041B0C7B
:10CBF00083807047038823F400631B041B0C0380AD
:10CC000003889BB219430180704703889BB243F4A9
:10CC1000805303807047038819B19BB243F40053DB
:10CC200003E023F400531B041B0C0380704701290D
:10CC300014BF008B808A80B27047008A80B2704730
:10CC4000B1F5804F038803D19BB243F4804303E0E6
:10CC500023F480431B041B0C038070470389194293
:10CC60000CBF002001207047202906D103890388CA
:10CC70009BB243F0400303807047402901D008294C
:10CC800001D103897047C94389B20181704701F01E
:10CC90000F02012303FA02F210B584880089A4B2BE
:10CCA00080B2104005D009098B401C420CBF002007
:10CCB000012010BD552906D1038903889BB243F09A
:10CCC000400303807047562901D0532901D10389BD
:10CCD000704701F00F01012303FA01F1C94389B242
:10CCE00001817047044B04281A680CBF42F004020B
:10CCF00022F004021A60704710E000E0014B586017
:10CD0000704700BF10E000E00128084B03D11A680B
:10CD100042F0010204E0023004D11A6822F001025C
:10CD20001A60704700229A60704700BF10E000E070
:10CD3000044B1A6810B142F0020201E022F0020234
:10CD40001A60704710E000E0014B9868704700BF20
:10CD500010E000E0C308022B044B0CBF1B68DB682B
:10CD600023FA00F000F00100704700BF10E000E07F
:10CD700030B5048C24F001042404240C0484058BB5
:10CD8000048CADB225F0F305A4B22A4324F00204CA
:10CD900042EA031344F001049DB221430583018458
:10CDA00030BD30B5048C24F010042404240C048419
:10CDB000058B048C25F44075A4B22D052D0D24F0AF
:10CDC000200444F0100445EA022242EA033344EA14
:10CDD00001119BB28CB20383048430BD08B52E4B85
:10CDE00098423AD010D8A3F50063984225D003F5B5
:10CDF000806398422BD0B0F1804F4CD10120014686
:10CE0000FFF78EFD01201DE0244B984231D004D85D
:10CE1000A3F58063984226D008BD214B984204D0E8
:10CE200003F5006398422AD008BD4FF40060012149
:10CE3000FFF76AFD4FF4006028E002200121FFF7B0
:10CE40006FFD02200021BDE80840FFF769BD042006
:10CE50000121FFF765FD0420F4E708200121FFF719
:10CE60005FFD0820EEE710200121FFF759FD10209B
:10CE7000E8E720200121FFF753FD2020E2E74FF4EF
:10CE800000500121FFF740FD4FF400500021BDE8A4
:10CE90000840FFF739BD08BD000C004000140040F9
:10CEA000002C01400388CA8803F08F0303800388A5
:10CEB0009BB213434A8813439BB203808B888385BC
:10CEC0000B880385054B984203D003F50063984215
:10CED00001D10B7A0386012383827047002C014025
:10CEE000038C70B523F001031B041B0C0384038C1B
:10CEF0008488028B0D8822F070021204120C4E8876
:10CF00002A430D8923F002031B043543ADB21B0CE9
:10CF10002B43CD88A4B285860D4DA84203D005F5DC
:10CF20000065A8420FD14D8923F008032B438D885B
:10CF300023F004032B4347F6FF452540CC8989891C
:10CF40000C43A4B22C4384800283038470BD00BFD1
:10CF5000002C0140038C30B523F010031B041B0C84
:10CF60000384038C8288048B0D8824F4E044240419
:10CF7000240C23F0200344EA05241B040D891B0C18
:10CF800043EA05134D8892B243EA0513CD88A4B253
:10CF90000587114D9BB2A84203D005F50065A84254
:10CFA00016D14D8923F080039BB243EA05134FF657
:10CFB000BF751D408B8845EA031347F2FF351540C6
:10CFC0008A899BB245EA8205CA8945EA820292B201
:10CFD00082800483038430BD002C0140038C30B573
:10CFE00023F480731B041B0C0384038C8288848BC2
:10CFF0000D8824F070042404240C23F400732C43C3
:10D000001B040D891B0C43EA05234D8892B243EAA9
:10D010000523CD889BB28587104DA84203D005F526
:10D020000065A84216D14D8923F400639BB243EA00
:10D0300005234FF6FF351D408B8845EA032344F650
:10D04000FF7515408A899BB245EA0215CA8945EAEF
:10D05000021292B282808483038430BD002C01408E
:10D06000038C30B523F480531B041B0C0384038C06
:10D070008488828B0D8822F4E0421204120C23F47F
:10D08000005342EA05221B040D891B0C43EA0533B9
:10D090004D88A4B243EA0533CD8892B2A0F840503F
:10D0A000084D9BB2A84203D005F50065A84205D102
:10D0B0008989C4F30D0444EA8114A4B28480828374
:10D0C000038430BD002C01404A880B8813438A88B2
:10D0D0001343CA8813430A8913434A8913438A892D
:10D0E00013439BB2A0F8443070474FF6FF73838020
:10D0F00000230380C38043800372704700230380B2
:10D1000043808380C380038143818381C3817047CF
:10D1100000230122038043808280C3800381704703
:10D120000023038043808380C38003814381838104
:10D130007047038819B19BB243F0010303E023F069
:10D1400001039B059B0D03807047B0F8443029B163
:10D150006FEA43436FEA53439BB201E0C3F30E030C
:10D16000A0F84430704783899BB20AB1194301E0AB
:10D1700023EA010181817047818270470A43A0F848
:10D180004820704783899BB20AB1194301E023EA22
:10D19000010181817047038923F007031B041B0CE5
:10D1A00003817047038923F070031B041B0C194390
:10D1B000018103899BB243F007030381704738B5AF
:10D1C0000D46602D114604464FF0010202D1FFF7D3
:10D1D000E8FD01E0FFF7CCFD238923F070031B0479
:10D1E0001B0C2B43238123899BB243F0070323812C
:10D1F00038BD10B5048942EA0323E4B21C43A4B24B
:10D200002143018110BD10B50446FFF7F2FF2389C9
:10D2100023F077031B041B0C43F07703238110BD1D
:10D2200010B50446FFF7E5FF23899BB243F4804322
:10D23000238110BD018582827047038823F070032B
:10D240009B059B0D194301807047038923F07003F0
:10D250001B041B0C19430181704770B50589048BB1
:10D26000068C24F44074B6B224F0030426F022069F
:10D2700025F00705240432432D04240C2D0C44F41E
:10D28000807442EA0313294344F001049EB20181F1
:10D290000483068470BD038B23F070031B041B0CF6
:10D2A000194301837047038B23F4E0431B041B0CD9
:10D2B00043EA01218BB203837047838B23F0700311
:10D2C0001B041B0C194381837047838B23F4E043B9
:10D2D0001B041B0C43EA01218BB283837047038834
:10D2E00019B19BB243F0800303E023F080039B0558
:10D2F0009B0D03807047838819B19BB243F00403F0
:10D3000003E023F004031B041B0C83807047838815
:10D3100019B19BB243F0080303E023F008031B0498
:10D320001B0C83807047838819B19BB243F00103C3
:10D3300003E023F001031B041B0C83807047038B65
:10D3400023F008031B041B0C194301837047038B54
:10D3500023F400631B041B0C43EA01218BB20383FB
:10D360007047838B23F008031B041B0C1943818334
:10D370007047838B23F400631B041B0C43EA0121D9
:10D380008BB283837047038B23F004031B041B0CB5
:10D39000194301837047038B23F480631B041B0C28
:10D3A00043EA01218BB203837047838B23F004038C
:10D3B0001B041B0C194381837047838B23F4806308
:10D3C0001B041B0C43EA01218BB283837047038B40
:10D3D00023F080031B041B0C194301837047038B4C
:10D3E000C3F30E0343EA01218BB203837047838B9F
:10D3F00023F080031B041B0C194381837047838B2C
:10D40000C3F30E0343EA01218BB283837047038C7D
:10D4100023F002031B041B0C194301847047038C87
:10D4200023F008031B041B0C194301847047038C71
:10D4300023F020031B041B0C43EA01118BB203846D
:10D440007047038C23F080031B041B0C43EA01117B
:10D450008BB203847047038C23F400731B041B0CF2
:10D4600043EA01218BB203847047038C23F40063E9
:10D470001B041B0C43EA01218BB203847047038C0D
:10D4800023F400531B041B0C43EA01318BB20384C9
:10D49000704701238B408A4010B5048CA4B224EA63
:10D4A00003030384038C13439BB2038410BD042342
:10D4B0008B408A4010B5048CA4B224EA0303038491
:10D4C000038C13439BB2038410BD01238B4010B522
:10D4D000048C1830A4B224EA0303038121F008036A
:10D4E0003BB9490844584FF68F7323404350435883
:10D4F0000AE00439C1F34E01445848F6FF73234053
:10D5000043501202435892B21A43425010BD03884E
:10D5100019B19BB243F0020303E023F002039B0521
:10D520009B0D03807047038819B19BB243F004033D
:10D5300003E023F004039B059B0D03807047838861
:10D5400019B19BB243F0800303E023F080031B0476
:10D550001B0C83807047038823F008039B059B0DF9
:10D56000038003889BB2194301807047838823F0AE
:10D5700070031B041B0C838083889BB2194381803A
:10D580007047038923F007031B041B0C03810389E5
:10D590009BB2194301817047038923F080031B0468
:10D5A0001B0C038103899BB219430181704781845D
:10D5B00070478185704781867047018770478187F2
:10D5C0007047A0F840107047038B23F00C031B0436
:10D5D0001B0C0383038B9BB2194301837047038B9E
:10D5E00023F440631B041B0C0383038B9BB243EAAD
:10D5F00001218BB203837047F8B50C464988A28895
:10D600000029B4F800E014BF00270227012A0546CC
:10D6100014BF012602262389BEF1000F11D1FFF7A6
:10D62000A7FB2846E188FFF7CFFF28463946324658
:10D630002389FFF7B6FB2846E188BDE8F840FFF7ED
:10D64000CEBFFFF7AEFB2846E188FFF7C8FF2846AC
:10D65000394632462389FFF78BFB2846E188BDE82F
:10D66000F840FFF7B1BF838B23F00C031B041B0CA6
:10D670008383838B9BB2194381837047838B23F40D
:10D6800040631B041B0C8383838B9BB243EA012101
:10D690008BB283837047F8B50E880D4604464988DF
:10D6A000AA882B893EB9FFF763FB2046E988BDE8CD
:10D6B000F840FFF789BF042E07D1FFF772FB204621
:10D6C000E988BDE8F840FFF78ABF082EEF88068C8E
:10D6D0001CD126F480763604360C0684858B068CA5
:10D6E000ADB225F0F30545EA0313B6B29BB21A4377
:10D6F00026F4007343EA012189B241F480718283E8
:10D7000001843946BDE8F840FFF7ADBF26F48056E6
:10D710003604360C0684858B068C25F440752D0561
:10D72000B6B22D0D45EA022526F4005242EA013137
:10D7300045EA033389B29BB241F48051838301846B
:10D740003946BDE8F840FFF799BF0388DBB2038094
:10D7500003889BB2194301807047808E80B2704766
:10D76000008F80B27047808F80B27047B0F8400061
:10D7700080B27047808C80B27047008D80B2704755
:10D78000038A19420CBF002001207047C94389B2A7
:10D7900001827047038A828911EA030092B203D0A2
:10D7A00011420CBF002001207047C94389B2018299
:10D7B000704700BF08B5224B98422CD008D8A3F57B
:10D7C0000063984217D003F5806398421BD008BDD0
:10D7D0001C4B984227D003F5684398422FD14FF451
:10D7E00080400121FFF790F8BDE808404FF48040E9
:10D7F0000021FFF789B84FF400300121FFF790F8BE
:10D800004FF4003016E04FF480200121FFF788F834
:10D810004FF480200EE04FF400200121FFF780F844
:10D820004FF4002006E04FF480100121FFF778F854
:10D830004FF480100021BDE80840FFF771B808BD23
:10D84000004C004000500040038ACA889BB223F479
:10D850004053134330B503820D4682890989AB8852
:10D8600092B20B43698922F4B0520B4322F00C02AE
:10D8700013439BB28381838AAA899BB223F44073AA
:10D8800087B013430446838201A8FEF7D7FF049AAA
:10D89000039B0E498C4208BF134619214B432A684B
:10D8A0009200B3FBF2F16423B1FBF3F21201100911
:10D8B00003FB101109013231B1FBF3F303F00F0345
:10D8C0001A4392B2228107B030BD00BF0038014038
:10D8D0004FF4165303600C2200238380C38003811E
:10D8E0004281838170470B8810B54C88028A23439C
:10D8F0008C88C98892B223430B4322F4706213438D
:10D900009BB2038210BD0023038043808380C380C9
:10D910007047838919B19BB243F4005303E023F4A9
:10D9200000531B041B0C83817047C1F3421310B5D5
:10D93000012401F01F01A34204FA01F101D10C30CE
:10D9400003E0022B0CBF1030143003680AB11943F6
:10D9500001E023EA0101016010BD838A9BB20AB194
:10D96000194301E023EA010181827047038A23F011
:10D970000F031B041B0C0382038A9BB21943018211
:10D980007047838923F400631B041B0C8381838904
:10D990009BB2194381817047838919B19BB243F0CF
:10D9A000020303E023F002031B041B0C8381704776
:10D9B000038A23F020031B041B0C0382038A9BB2FF
:10D9C000194301827047038A19B19BB243F4804323
:10D9D00003E023F480431B041B0C03827047C1F354
:10D9E0000801818070478088C0F3080070478389F0
:10D9F0009BB243F0010383817047038BDBB2038347
:10DA0000038B9BB243EA012101837047038B03F42C
:10DA10007F430383038B9BB2194301837047838A3F
:10DA200019B19BB243F0200303E023F020031B0451
:10DA30001B0C83827047838A19B19BB243F0100399
:10DA400003E023F010031B041B0C83827047838ABE
:10DA500019B19BB243F0080303E023F008031B0451
:10DA60001B0C83827047838A23F004031B041B0C66
:10DA70008382838A9BB2194381827047838A19B15A
:10DA80009BB243F0020303E023F002031B041B0CD0
:10DA900083827047038819420CBF00200120704721
:10DAA000C94389B20180704710B5C1F3421401F037
:10DAB0001F030122012C02FA03F201D1838903E042
:10DAC000022C0CBF038A838A9BB21340028892B255
:10DAD00043B10123090A03FA01F111420CBF0020EE
:10DAE000012010BD184610BD090A01238B40DB43FD
:10DAF0009BB20380704700BF684620F007018D4647
:10DB000001B500230B4A0C499818884204D20B49EE
:10DB1000595899500433F5E7094B0A4A934203D206
:10DB2000002243F8042BF8E702F0A4FBBDE8014013
:10DB3000854670470000002064050020FC0D0108A8
:10DB400068050020A410002010B5064C18B9236801
:10DB500001221A8210BD044B1B681B68984720687D
:10DB60000A3010BD40100020FC0F002010B5064CFC
:10DB700018B9236801221A8210BD044B1B689B68E8
:10DB8000984720680C3010BD40100020FC0F00208A
:10DB900010B5204B18B91B6802221A8210BD1E4A0C
:10DBA0001968002010800C78134614F07F040DD102
:10DBB0004A7A910644BF0221197012F0400F1A7878
:10DBC00014BF22F0010242F0010214E0012C1FD028
:10DBD000022C1ED1497901F00F02920002F180421D
:10DBE00002F5B84211F0800F126806D002F0300240
:10DBF000102A07D101221A7004E002F44052B2F553
:10DC0000805FF6E7054B1B681B699847024810BD0B
:10DC1000104610BD401000209C100020FC0F00207A
:10DC2000234A2DE9F84314689046238A267A214F27
:10DC3000A3B9042E12D120490A78012A0AD11F4A19
:10DC400010681F4A80B202445200136030223A80AA
:10DC50000B7027E010233B80072623E0A58AAB4208
:10DC60008CBF022604269D4228BF1D462846A36974
:10DC700098478146002000F06BFE2A460146484640
:10DC800000F06EFC2946002000F07EFE238A4FF44F
:10DC900040525B1B2382638A1D4430233B80094B27
:10DCA00065821A80D8F800301E72BDE8F88300BF84
:10DCB00040100020A01000201C0A0020505C0040F2
:10DCC000023000209E10002010B50A4B0A491B6844
:10DCD0004978DA7891420AD3997841B99C8834B965
:10DCE0009A72064B1B685B689847204610BD02205D
:10DCF00010BD00BF40100020D8000020FC0F002005
:10DD000038B50E4A0E4C1268236892695879D97852
:10DD1000904723689A7A7AB170B91A7962B99D7876
:10DD200055B9084B1B68DB689847236828465A7921
:10DD3000DA72DA781A7338BD022038BDD80F0020A5
:10DD400040100020FC0F002038B52F4B1B681878BE
:10DD500010F07F0004D15A7A22F020025A7238BDA6
:10DD600002284ED15A88002A4CD11A79002A49D16A
:10DD70005A79264D22F08000840004F1804101F59B
:10DD8000B84109682D7812F0800F14BF01F03001FE
:10DD900001F44051A84234D2002932D09B7A83B397
:10DDA00004F1804404F5B844120623680CD503F04E
:10DDB0003003102B1FD1C4B2204600F080FD204656
:10DDC000302100F055FC16E003F44053B3F5805FBA
:10DDD00011D128B90E4B93F82C1000F0F6FD01E09C
:10DDE00000F05DFD236823F4804323F070039BB2B1
:10DDF00083F440532360074B1B685B6998470020FE
:10DE000038BD022038BD00BF40100020D8000020DF
:10DE100050000020FC0F002038B51D4B1D4D196827
:10DE20002D784A7922F08004A30003F1804000F5A8
:10DE3000B840006812F0800F14BF00F0300000F40A
:10DE40004050AC4222D24C8804BBF8B1897AE9B187
:10DE500003F1804303F5B84312F0800F1A6807D02E
:10DE600022F4E04222F0400292B282F0100206E078
:10DE700022F4804222F0700292B282F480521A6040
:10DE8000054B1B689B699847002038BD022038BDB0
:10DE900040100020D8000020FC0F002008B5064BE1
:10DEA0001B685A7A42F020025A72044B1B68DB69E5
:10DEB0009847002008BD00BF40100020FC0F002044
:10DEC000054B1A68538A18B98988CB1A1382704790
:10DED00008681844704700BF4010002008B50B4B7D
:10DEE000002093F82C1000F070FD094B1B68187A85
:10DEF000082806D1074B4FF480521A80064B102297
:10DF00001A80B0F109035842584108BD5000002062
:10DF1000401000209E100020A0100020F7B5914F67
:10DF2000914B3A68914D92B213442E685B001C6885
:10DF3000337A092B15D0A4B2640004F1804404F5AF
:10DF4000C0442378337063787370A08800F0E8FED3
:10DF5000708020892E6800F0E3FEB080A2892B68D3
:10DF6000DA802B6801221A72DA885C78002A61D183
:10DF70001A7812F07F023AD1092C02D1FFF7A4FEE1
:10DF800044E0052C0FD193F90320002A01DA08237D
:10DF90004DE09A78002AFAD19A88002AF7D19B7A24
:10DFA000002B37D0F3E7032C13D1DA78012A07D0FE
:10DFB0006F4B20461B685B699847032828D135E0E2
:10DFC0009A88002AF4D15B7A9806F1D5FFF766FFAC
:10DFD0001CE0012CECD1DA78012AE9D19A88002AD8
:10DFE000E6D15B7A9906E3D5FFF7AEFE0EE0012A93
:10DFF00004D10B2CDCD1FFF783FE07E0022AD7D136
:10E00000012CF1D0032CD3D1FFF706FF10B1CFE7DD
:10E010000028BCD13A68574B92B213445B000022EF
:10E020001A60554B30221A80062300E009232A6823
:10E030001372D0E0062C13D11A78520678D19A7850
:10E040004B4B012A02D11B68DB6968E0022A02D12E
:10E050001B681B6A63E0032A6AD11B685B6A5EE087
:10E06000002C3DD15988002962D15A6822F47F42A0
:10E07000B2F5003F5CD11A7812F07F0204D19B8880
:10E08000002B00F0AC8053E0012A0DD1384A5879BA
:10E0900012689269904700284AD1344B1B689B7ADA
:10E0A000002B40F09C8043E0022A41D15B79334849
:10E0B00003F00F018A0002F1804202F5B8421268B3
:10E0C000007813F0800F14BF02F0300202F44052C7
:10E0D00081422DD213F0700F2AD1002A7FD127E080
:10E0E000082C03D11B785B067BD021E00A2C1FD1C2
:10E0F0001A7802F07F02012A1AD19A7AC2B159889D
:10E10000B1B95A6822F47F42B2F5803F10D1184A63
:10E110005879126892699047002864D008E03BB1B2
:10E120002A680024548293612046984720460AE0DA
:10E130000F4B1A682B68126958789047032802D150
:10E140000A4B1B6805E02B684FF6FF711A8A8A425A
:10E1500001D1092203E0022800D08AB908221A72EC
:10E1600039E000BF505C0040043000204010002027
:10E17000D80F002002300020A0100020D80000207E
:10E1800093F90010002920DAD98801910198824280
:10E19000164802D9019A1A8210E08A420ED201680A
:10E1A00091F82C108A4201D2002105E092FBF1F493
:10E1B00001FB142212B901210D4A1170026892F874
:10E1C0002C209A82FFF72CFD05E003221A72094BDE
:10E1D0004FF440521A80FFF781FE03B0F0BD064BAA
:10E1E0009EE7064B9CE7064B9AE700BFD80F00203E
:10E1F0001C0A00209E10002091DB000849DB00086B
:10E200006DDB0008F8B52B4D2C68237A032B01D069
:10E21000052B41D1A369228AABB1A2B1A68A96424D
:10E2200028BF164630469847238A07469B1B238201
:10E23000638A00203344638200F098FB3246014633
:10E24000384600F0A5F9238A53B11B4B00204FF448
:10E25000405201461A8000F097FB184B30221A807A
:10E26000238AA28A9A4202D82B68032202E01BB1B9
:10E270002B6805221A720CE02A6806211172104AD6
:10E280001168104A89B20A44520013600B4B3022C5
:10E290001A802B681B7A06E0072B03D10A4B1B68F8
:10E2A000DB68984708232A681372BDE8F840FFF737
:10E2B00015BE00BF401000209E100020A0100020BE
:10E2C000505C004002300020D80F002030B50B4BCE
:10E2D0001C780023A3420CD203F1805202F5B852FD
:10E2E00091000D6848F68F722A401A430A60013384
:10E2F000F0E7034B40F08000186030BDD8000020EC
:10E300004C5C004010B5134C23681A7A022A01D0E5
:10E31000042A04D1FFF784FC23681B7A13E0062A41
:10E3200010D15A78052A09D11A78520606D1D87820
:10E33000FFF7CCFF084B1B681B6A9847074B1B680D
:10E340009B689847082322681372BDE81040FFF7C6
:10E35000C5BD00BF40100020FC0F0020D80F0020DA
:10E36000704700BF08B5074A074B084913600222EF
:10E370001A72074B074A1360074A1B6811609847D7
:10E3800008BD00BF40100020E00F0020B4000020B6
:10E3900050000020D80F0020FC0F002070B54C4A20
:10E3A0004C4B116888B20C04188040F1908047F6FD
:10E3B000FF7111601A88484C02F00F022270002A87
:10E3C0005FD1464C464D2268464E02F440522A80A8
:10E3D000226802F030023280226822F4804222F069
:10E3E000700292B282F400522260226822F4E0426B
:10E3F00022F0400292B282F0200222601B88D806EE
:10E4000002D52368190607D5226848F60F73134012
:10E410002360FFF777FF12E01A0507D5226840F660
:10E420008F7313402360FFF779FD08E01804B6D519
:10E43000226840F68F7313402360FFF7E3FE2368E2
:10E440002A8823F4804323F070039BB2D10448BF91
:10E4500083F480539504214A48BF83F4005313602A
:10E460001368318823F4E04323F040039BB2CC06C9
:10E4700048BF83F01003880648BF83F02003136071
:10E4800070BD930003F1804303F5B8431D68290470
:10E4900009D5186840F68F7101401960124B013A96
:10E4A00053F8223098472B067FF579AF217848F64C
:10E4B0000F728B0003F1804303F5B84318680139EC
:10E4C00002401A60094B53F82130984767E770BD46
:10E4D000445C0040D60F0020DC0F0020005C0040B0
:10E4E0009E100020A0100020DC000020F80000207A
:10E4F00008B5164A164B116888B20904188024D54D
:10E5000047F6FF7111601A88124B02F00F021A7061
:10E51000930003F1804303F5B8431968080407D555
:10E52000186840F68F7101401960013A0A4B08E003
:10E530000906DED5186848F60F7101401960074BCF
:10E54000013A53F822309847D3E708BD445C0040B5
:10E55000D60F0020DC0F0020DC000020F800002097
:10E5600030B501F10051013201F54051521049001E
:10E570000023934200F1020009D010F8015C10F86A
:10E58000024C44EA052421F823400133F1E730BD71
:10E5900010B501F10051013201F54051521049000E
:10E5A0000023934205D051F8234020F81340013353
:10E5B000F7E710BD014B1860704700BF405C00409A
:10E5C000014B186880B27047405C0040014B1860F6
:10E5D000704700BF445C0040014B186880B2704730
:10E5E000445C0040014B186880B27047485C0040B2
:10E5F000014B1860704700BF4C5C0040014B18682D
:10E6000080B270474C5C00404FF6F873014A0340FB
:10E6100013607047505C0040014B186880B270472F
:10E62000505C0040800000F1804000F5B84001607F
:10E630007047800000F1804000F5B840006880B26B
:10E640007047800000F1804000F5B840036823F473
:10E65000EC4323F0700319438BB2036070478000D2
:10E6600000F1804000F5B840006800F4C0607047D9
:10E67000800000F1804000F5B8400368CA0623F42A
:10E68000E04323F040039BB248BF83F010038A06A7
:10E6900048BF83F0200303607047800000F1804092
:10E6A00000F5B8400368CA0423F4804323F07003E4
:10E6B0009BB248BF83F480538A0448BF83F400535D
:10E6C00003607047800000F1804000F5B8400129E8
:10E6D000026802D14EF6FF7303E0022903D14FF620
:10E6E000EF73134003607047800000F1804000F535
:10E6F000B840006800F030007047800000F18040B2
:10E7000000F5B840006800F440507047800000F108
:10E71000804000F5B840036823F4E04323F0400351
:10E720009BB283F0300303607047800000F18040AB
:10E7300000F5B840036823F4804323F070039BB2D4
:10E7400083F4405303607047800000F1804000F57F
:10E75000B840036823F4E04323F0700343F480736C
:10E760009BB203607047800000F1804000F5B84024
:10E77000036823F4E24323F070031B041B0C0360C3
:10E780007047800000F1804000F5B840036823F432
:10E79000E24323F070031B041B0C036070478000EE
:10E7A00000F1804000F5B840036823F4E04323F013
:10E7B000700343F480739BB203607047800000F1E4
:10E7C000804000F5B840036823F4E04323F0700371
:10E7D00043F480739BB203607047800000F1804077
:10E7E00000F5B840036823F4E24323F070031B04F0
:10E7F0001B0C03607047800000F1804000F5B840BA
:10E80000006800F03000B0F11003584258417047E2
:10E81000800000F1804000F5B840006800F44050EE
:10E82000B0F58053584258417047800000F1804055
:10E8300000F5B840036823F070031B051B0D03604F
:10E840007047800000F1804000F5B840036823F471
:10E85000E14323F070031B041B0C0360704780002E
:10E8600000F1804000F5B840036823F4E04323F052
:10E8700070031B041B0C43F480430360704780004B
:10E8800000F1804000F5B840036823F4E04323F032
:10E8900070031B041B0C43F04003036070478000AF
:10E8A00000F1804000F5B84003685B0406D50268BB
:10E8B00048F68F73134043F4804303607047800031
:10E8C00000F1804000F5B84003685B0606D5026899
:10E8D00048F68F73134043F0400303607047800095
:10E8E00000F1804000F5B840036823F4E04323F0D2
:10E8F00070031B041B0C194301607047800000F17A
:10E90000804000F5B840006800F00F007047074BEA
:10E9100049081B6849009BB203EBC00000F100509E
:10E9200000F5405040000160704700BF505C00405F
:10E93000054B49081B6849009BB203EBC000034B21
:10E9400003445B0019607047505C004004300020B5
:10E95000054B1B689BB203EBC00000F1005000F5B3
:10E960004050400000887047505C0040044B1B68DA
:10E970009BB203EBC000034B03445B001888704755
:10E98000505C004004300020044B1B689BB203EB3A
:10E99000C000034B03445B0019607047505C0040AB
:10E9A000023000203E2909D94B09C90604BF03F1F2
:10E9B000FF339BB29B0243F4004304E04B08CA07B9
:10E9C00048BF01339B02036070470E4B3E291B6812
:10E9D0009BB203EBC0000C4B03444FEA430209D93E
:10E9E0004B09C80604BF03F1FF339BB29B0243F4FB
:10E9F000004304E04B08C90748BF01339B02136082
:10EA0000704700BF505C004006300020054B1B687B
:10EA10009BB203EBC000044B03445B001868C0F3D7
:10EA200009007047505C004002300020054B1B6815
:10EA30009BB203EBC000044B03445B001868C0F3B7
:10EA400009007047505C00400630002010B50B4CA8
:10EA5000C000236849089BB2034403F1005303F547
:10EA600040535B0049001960236852089BB2184468
:10EA7000034B520003445B001A6010BD505C004021
:10EA800004300020064B49081B6849009BB203EB89
:10EA9000C00000F1005000F5405040000160704798
:10EAA000505C0040054B49081B6849009BB203EBD2
:10EAB000C000034B03445B0019607047505C00408A
:10EAC00004300020054B1B689BB203EBC00000F133
:10EAD000005000F54050400000887047505C0040F6
:10EAE000044B1B689BB203EBC000034B03445B0069
:10EAF00018887047505C004004300020012910B590
:10EB00002FD1254CC0002168244B89B201440B440D
:10EB10003E2A4FEA43010AD9530912F01F0F04BFDE
:10EB200003F1FF339BB29B0243F4004305E053081B
:10EB300012F0010F18BF01339B020B6023683E2ABD
:10EB40009BB21844164B03444FEA43031CD95109A6
:10EB5000D00604BF01F1FF3189B2890241F40041BE
:10EB600017E0022917D10C49C0000C680B4BA4B266
:10EB7000044423445B001A600B689BB21844084BA2
:10EB800003445B001A6010BD5108D20748BF013131
:10EB90008902196010BD10BD505C00400230002099
:10EBA0000630002001291BD1134B3E2A1B689BB263
:10EBB00003EBC000114B03444FEA430109D9530949
:10EBC000D00604BF03F1FF339BB29B0243F4004322
:10EBD00004E05308D20748BF01339B020B60704723
:10EBE000022908D1044B1B689BB203EBC000034B06
:10EBF00003445B001A607047505C00400230002004
:10EC000001291BD1134B3E2A1B689BB203EBC000AA
:10EC1000114B03444FEA430109D95309D00604BFFD
:10EC200003F1FF339BB29B0243F4004304E053081B
:10EC3000D20748BF01339B020B607047022908D1FD
:10EC4000044B1B689BB203EBC000034B03445B0007
:10EC50001A607047505C004006300020054B1B686E
:10EC60009BB203EBC000044B03445B001868C0F385
:10EC700009007047505C004002300020054B1B68C3
:10EC80009BB203EBC000044B03445B001868C0F365
:10EC900009007047505C0040063000200D4AC0005B
:10ECA00013689BB2C1180C4B0B445B001B8813F418
:10ECB0007C4F0DD113689BB21844084B03445B0092
:10ECC0001B88C3F30903002B0CBF002002207047F0
:10ECD00001207047505C00400630002002300020C8
:10ECE00001290BD1800000F1804000F5B840026896
:10ECF00048F68F73134043F040030CE002290BD118
:10ED0000800000F1804000F5B840026848F68F733B
:10ED1000134043F480430360704741EA002070478A
:10ED2000C3B2000A40EA0320704700BF81F00041EF
:10ED300002E000BF83F0004330B54FEA41044FEAE0
:10ED4000430594EA050F08BF90EA020F1FBF54EA7B
:10ED5000000C55EA020C7FEA645C7FEA655C00F017
:10ED6000E2804FEA5454D4EB5555B8BF6D420CDDE8
:10ED70002C4480EA020281EA030382EA000083EA6B
:10ED8000010180EA020281EA0303362D88BF30BD0B
:10ED900011F0004F4FEA01314FF4801C4CEA113161
:10EDA00002D0404261EB410113F0004F4FEA0333C0
:10EDB0004CEA133302D0524263EB430394EA050F4B
:10EDC00000F0A780A4F10104D5F1200E0DDB02FABA
:10EDD0000EFC22FA05F2801841F1000103FA0EF24E
:10EDE000801843FA05F359410EE0A5F120050EF114
:10EDF000200E012A03FA0EFC28BF4CF0020C43FA45
:10EE000005F3C01851EBE37101F0004507D54FF051
:10EE1000000EDCF1000C7EEB00006EEB0101B1F5A1
:10EE2000801F1BD3B1F5001F0CD349085FEA3000E7
:10EE30004FEA3C0C04F101044FEA445212F5800FF2
:10EE400080F09A80BCF1004F08BF5FEA500C50F18F
:10EE5000000041EB045141EA050130BD5FEA4C0C72
:10EE6000404141EB010111F4801FA4F10104E9D1FB
:10EE700091F0000F04BF01460020B1FA81F308BFF2
:10EE80002033A3F10B03B3F120020CDA0C3208DDBE
:10EE900002F1140CC2F10C0201FA0CF021FA02F199
:10EEA0000CE002F11402D8BFC2F1200C01FA02F109
:10EEB00020FA0CFCDCBF41EA0C019040E41AA2BF2E
:10EEC00001EB0451294330BD6FEA04041F3C1CDAF6
:10EED0000C340EDC04F11404C4F1200220FA04F016
:10EEE00001FA02F340EA030021FA04F345EA0301C0
:10EEF00030BDC4F10C04C4F1200220FA02F001FA82
:10EF000004F340EA0300294630BD21FA04F0294603
:10EF100030BD94F0000F83F4801306BF81F480119C
:10EF20000134013D4EE77FEA645C18BF7FEA655C0F
:10EF300029D094EA050F08BF90EA020F05D054EAE1
:10EF4000000C04BF1946104630BD91EA030F1EBFE6
:10EF50000021002030BD5FEA545C05D140004941EA
:10EF600028BF41F0004130BD14F580043CBF01F5DD
:10EF7000801130BD01F0004545F0FE4141F47001C3
:10EF80004FF0000030BD7FEA645C1ABF194610469E
:10EF90007FEA655C1CBF0B46024650EA013406BF9F
:10EFA00052EA033591EA030F41F4002130BD00BF5E
:10EFB00090F0000F04BF0021704730B54FF480641B
:10EFC00004F132044FF000054FF0000150E700BF9C
:10EFD00090F0000F04BF0021704730B54FF48064FB
:10EFE00004F1320410F0004548BF40424FF00001E8
:10EFF0003EE700BF42004FEAE2014FEA31014FEA2B
:10F0000002701FBF12F07F4393F07F4F81F0605179
:10F01000704792F0000F14BF93F07F4F704730B5E8
:10F020004FF4607401F0004521F0004120E700BF7B
:10F0300050EA010208BF704730B54FF000050AE002
:10F0400050EA010208BF704730B511F0004502D503
:10F05000404261EB41014FF4806404F132045FEA05
:10F06000915C3FF4DCAE4FF003025FEADC0C18BFAA
:10F0700003325FEADC0C18BF033202EBDC02C2F1A0
:10F08000200300FA03FC20FA02F001FA03FE40EA32
:10F090000E0021FA02F11444C1E600BF70B54FF032
:10F0A000FF0C4CF4E06C1CEA11541DBF1CEA135514
:10F0B00094EA0C0F95EA0C0F00F0DEF82C4481EA7C
:10F0C000030621EA4C5123EA4C5350EA013518BF9C
:10F0D00052EA033541F4801143F4801338D0A0FB89
:10F0E00002CE4FF00005E1FB02E506F00042E0FB36
:10F0F00003E54FF00006E1FB03569CF0000F18BF3C
:10F100004EF0010EA4F1FF04B6F5007F64F54074E3
:10F1100004D25FEA4E0E6D4146EB060642EAC62176
:10F1200041EA55514FEAC52040EA5E504FEACE2EE3
:10F13000B4F1FD0C88BFBCF5E06F1ED8BEF1004FE6
:10F1400008BF5FEA500E50F1000041EB045170BD62
:10F1500006F0004646EA010140EA020081EA0301A6
:10F16000B4EB5C04C2BFD4EB0C0541EA045170BDA2
:10F1700041F480114FF0000E013C00F3AB8014F11C
:10F18000360FDEBF002001F0004170BDC4F1000465
:10F19000203C35DA0C341BDC04F11404C4F12005E6
:10F1A00000FA05F320FA04F001FA05F240EA020041
:10F1B00001F0004221F0004110EBD37021FA04F677
:10F1C00042EB06015EEA430E08BF20EAD37070BD31
:10F1D000C4F10C04C4F1200500FA04F320FA05F090
:10F1E00001FA04F240EA020001F0004110EBD37092
:10F1F00041F100015EEA430E08BF20EAD37070BD02
:10F20000C4F1200500FA05F24EEA020E20FA04F3DA
:10F2100001FA05F243EA020321FA04F001F0004189
:10F2200021FA04F220EA020000EBD3705EEA430EFA
:10F2300008BF20EAD37070BD94F0000F0FD101F029
:10F240000046400041EB010111F4801F08BF013C62
:10F25000F7D041EA060195F0000F18BF704703F0A0
:10F260000046520043EB030313F4801F08BF013D27
:10F27000F7D043EA0603704794EA0C0F0CEA1355E3
:10F2800018BF95EA0C0F0CD050EA410618BF52EA9D
:10F290004306D1D181EA030101F000414FF00000A3
:10F2A00070BD50EA410606BF1046194652EA4306B1
:10F2B00019D094EA0C0F02D150EA013613D195EA25
:10F2C0000C0F05D152EA03361CBF104619460AD16D
:10F2D00081EA030101F0004141F0FE4141F4700177
:10F2E0004FF0000070BD41F0FE4141F4780170BD67
:10F2F00070B54FF0FF0C4CF4E06C1CEA11541DBFCC
:10F300001CEA135594EA0C0F95EA0C0F00F0A7F8CD
:10F31000A4EB050481EA030E52EA03354FEA0131FA
:10F3200000F088804FEA03334FF0805545EA13130D
:10F3300043EA12634FEA022245EA111545EA1065D5
:10F340004FEA00260EF000419D4208BF964244F16C
:10F35000FD0404F5407402D25B084FEA3202B61A8B
:10F3600065EB03055B084FEA32024FF480104FF45F
:10F37000002CB6EB020E75EB030E22BFB61A7546D3
:10F3800040EA0C005B084FEA3202B6EB020E75EB66
:10F39000030E22BFB61A754640EA5C005B084FEACE
:10F3A0003202B6EB020E75EB030E22BFB61A75469B
:10F3B00040EA9C005B084FEA3202B6EB020E75EBA6
:10F3C000030E22BFB61A754640EADC0055EA060E67
:10F3D00018D04FEA051545EA16754FEA06164FEAAA
:10F3E000C30343EA52734FEAC2025FEA1C1CC0D156
:10F3F00011F4801F0BD141EA00014FF000004FF0E3
:10F40000004CB6E711F4801F04BF01430020B4F1A3
:10F41000FD0C88BFBCF5E06F3FF6AFAEB5EB030C5B
:10F4200004BFB6EB020C5FEA500C50F1000041EB58
:10F43000045170BD0EF0004E4EEA113114EB5C0425
:10F44000C2BFD4EB0C0541EA045170BD41F48011F8
:10F450004FF0000E013C90E645EA060E8DE60CEA00
:10F46000135594EA0C0F08BF95EA0C0F3FF43BAF1D
:10F4700094EA0C0F0AD150EA01347FF434AF95EAD4
:10F480000C0F7FF425AF104619462CE795EA0C0FB8
:10F4900006D152EA03353FF4FDAE1046194622E785
:10F4A00050EA410618BF52EA43067FF4C5AE50EA5F
:10F4B00041047FF40DAF52EA43057FF4EBAE12E74F
:10F4C0004FF0FF3C06E000BF4FF0010C02E000BF30
:10F4D0004FF0010C4DF804CD4FEA410C7FEA6C5C13
:10F4E0004FEA430C18BF7FEA6C5C1BD001B050EAB6
:10F4F000410C0CBF52EA430C91EA030F02BF90EAA1
:10F50000020F0020704710F1000F91EA030F58BF5F
:10F51000994208BF90422CBFD8176FEAE37040F0C1
:10F52000010070474FEA410C7FEA6C5C02D150EA5F
:10F53000013C07D14FEA430C7FEA6C5CD6D152EA1A
:10F54000033CD3D05DF8040B704700BF84461046DF
:10F5500062468C461946634600E000BF01B5FFF7DE
:10F56000B7FF002848BF10F1000F01BD4DF808EDAE
:10F57000FFF7F4FF0CBF012000205DF808FB00BF7F
:10F580004DF808EDFFF7EAFF34BF012000205DF8D9
:10F5900008FB00BF4DF808EDFFF7E0FF94BF012026
:10F5A00000205DF808FB00BF4DF808EDFFF7CEFF27
:10F5B00094BF012000205DF808FB00BF4DF808ED66
:10F5C000FFF7C4FF34BF012000205DF808FB00BF37
:10F5D0004FEA410212F5001215D211D56FF478737B
:10F5E000B3EB625212D94FEAC12343F0004343EA1E
:10F5F000505311F0004F23FA02F018BF40427047F9
:10F600004FF00000704750EA013005D111F0004082
:10F6100008BF6FF0004070474FF00000704700BF18
:10F620004FEA4102B2F1E04324BFB3F5001CDCF124
:10F63000FE5C0DD901F0004C4FEAC0024CEA50705C
:10F64000B2F1004F40EB830008BF20F0010070478B
:10F6500011F0804F21D113F13872BCBF01F000408E
:10F66000704741F480114FEA5252C2F11802C2F1C0
:10F67000200C10FA0CF320FA02F018BF40F0010041
:10F680004FEAC1234FEAD32303FA0CFC40EA0C00F3
:10F6900023FA02F34FEA4303CCE77FEA625307D130
:10F6A00050EA01331EBF4FF0FE4040F44000704767
:10F6B00001F0004040F0FE4040F40000704700BF01
:10F6C00080F0004002E000BF81F0004142001FBF17
:10F6D0005FEA410392EA030F7FEA226C7FEA236C20
:10F6E0006AD04FEA1262D2EB1363C1BFD218414015
:10F6F00048404140B8BF5B42192B88BF704710F0AB
:10F70000004F40F4000020F07F4018BF404211F04D
:10F71000004F41F4000121F07F4118BF494292EAB5
:10F72000030F3FD0A2F1010241FA03FC10EB0C00E1
:10F73000C3F1200301FA03F100F0004302D549426E
:10F7400060EB4000B0F5000F13D3B0F1807F06D31B
:10F7500040084FEA310102F10102FE2A51D2B1F113
:10F76000004F40EBC25008BF20F0010040EA030008
:10F770007047490040EB000010F4000FA2F10102B5
:10F78000EDD1B0FA80FCACF1080CB2EB0C0200FA3F
:10F790000CF0AABF00EBC25052421843BCBFD0408D
:10F7A0001843704792F0000F81F4000106BF80F407
:10F7B00000000132013BB5E74FEA41037FEA226CCA
:10F7C00018BF7FEA236C21D092EA030F04D092F095
:10F7D000000F08BF0846704790EA010F1CBF0020C9
:10F7E000704712F07F4F04D1400028BF40F0004026
:10F7F000704712F100723CBF00F50000704700F046
:10F80000004343F0FE4040F4000070477FEA22626C
:10F8100016BF08467FEA23630146420206BF5FEA3D
:10F82000412390EA010F40F4800070474FF000033D
:10F8300004E000BF10F0004348BF40425FEA000C04
:10F8400008BF704743F0964301464FF000001CE0AC
:10F8500050EA010208BF70474FF000030AE000BF02
:10F8600050EA010208BF704711F0004302D5404240
:10F8700061EB41015FEA010C02BF844601460020B2
:10F8800043F0B64308BFA3F18053A3F50003BCFACD
:10F890008CF2083AA3EBC25310DB01FA02FC63447A
:10F8A00000FA02FCC2F12002BCF1004F20FA02F281
:10F8B00043EB020008BF20F00100704702F1200274
:10F8C00001FA02FCC2F1200250EA4C0021FA02F2D5
:10F8D00043EB020008BF20EADC7070474FF0FF0CDA
:10F8E0001CEAD0521EBF1CEAD15392EA0C0F93EAD5
:10F8F0000C0F6FD01A4480EA010C400218BF5FEA77
:10F9000041211ED04FF0006343EA501043EA5111E9
:10F91000A0FB01310CF00040B1F5000F3EBF4900E3
:10F9200041EAD3715B0040EA010062F17F02FD2AE7
:10F930001DD8B3F1004F40EBC25008BF20F00100CA
:10F94000704790F0000F0CF0004C08BF49024CEAE1
:10F95000502040EA51207F3AC2BFD2F1FF0340EA73
:10F96000C250704740F400004FF00003013A5DDCE4
:10F9700012F1190FDCBF00F000407047C2F1000225
:10F98000410021FA02F1C2F1200200FA02FC5FEA12
:10F99000310040F1000053EA4C0308BF20EADC705C
:10F9A000704792F0000F00F0004C02BF400010F4CE
:10F9B000000F013AF9D040EA0C0093F0000F01F07B
:10F9C000004C02BF490011F4000F013BF9D041EA9D
:10F9D0000C018FE70CEAD15392EA0C0F18BF93EA9F
:10F9E0000C0F0AD030F0004C18BF31F0004CD8D1C9
:10F9F00080EA010000F00040704790F0000F17BF50
:10FA000090F0004F084691F0000F91F0004F14D095
:10FA100092EA0C0F01D142020FD193EA0C0F03D1ED
:10FA20004B0218BF084608D180EA010000F00040F0
:10FA300040F0FE4040F40000704740F0FE4040F4CB
:10FA4000400070474FF0FF0C1CEAD0521EBF1CEA6A
:10FA5000D15392EA0C0F93EA0C0F69D0A2EB030288
:10FA600080EA010C49024FEA402037D04FF0805322
:10FA700043EA111143EA10130CF000408B4238BFE7
:10FA80005B0042F17D024FF4000C8B4224BF5B1AF5
:10FA900040EA0C00B3EB510F24BFA3EB510340EA43
:10FAA0005C00B3EB910F24BFA3EB910340EA9C00F1
:10FAB000B3EBD10F24BFA3EBD10340EADC001B0161
:10FAC00018BF5FEA1C1CE0D1FD2A3FF650AF8B4205
:10FAD00040EBC25008BF20F0010070470CF0004C12
:10FAE0004CEA50207F32C2BFD2F1FF0340EAC2503D
:10FAF000704740F400004FF00003013A37E792F0FE
:10FB0000000F00F0004C02BF400010F4000F013A5B
:10FB1000F9D040EA0C0093F0000F01F0004C02BF56
:10FB2000490011F4000F013BF9D041EA0C0195E7BF
:10FB30000CEAD15392EA0C0F08D142027FF47DAF58
:10FB400093EA0C0F7FF470AF084676E793EA0C0F48
:10FB500004D14B023FF44CAF08466EE730F0004C46
:10FB600018BF31F0004CCAD130F000427FF45CAFD6
:10FB700031F000437FF43CAF5FE700BF4FF0FF3C44
:10FB800006E000BF4FF0010C02E000BF4FF0010C97
:10FB90004DF804CD4FEA40024FEA41037FEA226C60
:10FBA00018BF7FEA236C11D001B052EA530C18BF82
:10FBB00090EA010F58BFB2EB030088BFC81738BFE7
:10FBC0006FEAE17018BF40F0010070477FEA226CD5
:10FBD00002D15FEA402C05D17FEA236CE4D15FEAD1
:10FBE000412CE1D05DF8040B704700BF8446084605
:10FBF0006146FFE70FB5FFF7C9FF002848BF10F1C6
:10FC0000000F0FBD4DF808EDFFF7F4FF0CBF01200A
:10FC100000205DF808FB00BF4DF808EDFFF7EAFF94
:10FC200034BF012000205DF808FB00BF4DF808ED4F
:10FC3000FFF7E0FF94BF012000205DF808FB00BF44
:10FC40004DF808EDFFF7D2FF94BF012000205DF8CA
:10FC500008FB00BF4DF808EDFFF7C8FF34BF0120D7
:10FC600000205DF808FB00BF42000ED2B2F1FE4F4B
:10FC70000BD34FF09E03B3EB126209D44FEA00237B
:10FC800043F0004323FA02F070474FF00000704742
:10FC900012F1610F01D1420202D14FF0FF307047E3
:10FCA0004FF00000704700BF73B96AB9002908BF60
:10FCB0000028BCBF00204FF00041C4BF6FF00041DE
:10FCC0004FF0FF3000F03CB882B0EC462DE9005018
:10FCD00000F006F8DDF804E002B00CBC704700BF8D
:10FCE0002DE9704F089E14461D468046894600F057
:10FCF00029F804FB01F3A4FB00AB00FB053293449D
:10FD0000B8EB0A0869EB0B09C6E90089BDE8708FFA
:10FD10002DE9704F089E14461D468046894600F026
:10FD200061F900FB05F5A0FB04AB04FB0154A344FF
:10FD3000B8EB0A0869EB0B09C6E90089BDE8708FCA
:10FD4000704700BF00292DE9F00FC0F2A180002408
:10FD5000002BC0F29880154606460F46002B3FD177
:10FD60008A4258D9B2FA82F34BB1C3F1200201FAA8
:10FD700003F720FA02F29D4000FA03F61743290C1C
:10FD8000B7FBF1F201FB1277A8B200FB02F34FEAD6
:10FD9000164C4CEA0747BB4209D97F1902F1FF3CD8
:10FDA00080F00581BB4240F20281023A2F44FF1AE3
:10FDB000B7FBF1F301FB137100FB03F0B6B246EAA7
:10FDC0000141884208D9491903F1FF3780F0F180D9
:10FDD000884240F2EE80023B43EA0242002303E005
:10FDE0008B420AD900231A461046194614B14042E4
:10FDF00061EB4101BDE8F00F7047B3FA83F8B8F149
:10FE0000000F40F088808B4202D3824200F2E280F1
:10FE100000230122E8E712B90123B3FBF2F5B5FA9A
:10FE200085F2002A3AD17F1B280C1FFA85FC01239A
:10FE3000B7FBF0F100FB11770CFB01F24FEA16481B
:10FE400048EA0747BA4207D97F1901F1FF3802D2C1
:10FE5000BA4200F2C4804146BF1AB7FBF0F200FB81
:10FE600012700CFB02FCB6B246EA0040844507D98A
:10FE7000401902F1FF3702D2844500F2AE803A46C3
:10FE800042EA0142B0E7E443524263EB430362E7D4
:10FE9000404261EB41014FF0FF3459E79540C2F118
:10FEA000200927FA09F126FA09F99740280CB1FB35
:10FEB000F0F800FB18111FFA85FC0CFB08F349EA67
:10FEC00007094FEA194747EA01418B4206FA02F651
:10FED00008D9491908F1FF327AD28B4278D9A8F1B2
:10FEE00002082944C91AB1FBF0F300FB13170CFBFD
:10FEF00003F21FFA89F949EA0747BA4207D97F197D
:10FF000003F1FF3160D2BA425ED9023B2F44BF1ADF
:10FF100043EA08438CE7C8F1200225FA02F103FA0C
:10FF200008FC27FA02F320FA02F207FA08F741EA7E
:10FF30000C0C4FEA1C49B3FBF9F109FB11331FFA12
:10FF40008CFA0AFB01FB17433A0C42EA03439B4538
:10FF500005FA08F008D913EB0C0301F1FF3235D292
:10FF60009B4533D902396344CBEB0303B3FBF9F26E
:10FF700009FB12330AFB02FABFB247EA0347BA454C
:10FF800008D917EB0C0702F1FF331BD2BA4519D978
:10FF9000023A674442EA0145A5FB0001CAEB0707A4
:10FFA0008F424FF000030AD305D02A461CE7624671
:10FFB000FDE63B4610E706FA08F68642F5D26A1ED1
:10FFC000002311E71A46E5E70B46A0E71146CBE709
:10FFD000904687E74346424606E7023A50E7023931
:10FFE0002F4439E72DE9F00F144605460E46002B45
:10FFF00043D18A4253D9B2FA82F757B1C7F12006EA
:020000040801F1
:1000000020FA06F601FA07F302FA07F400FA07F5F8
:100010001E43210CB6FBF1F201FB1266A0B200FBFD
:1000200002F32F0C47EA0646B34209D9361902F10A
:10003000FF3780F0FD80B34240F2FA80023A264456
:10004000F61AB6FBF1F301FB136100FB03F0ADB24E
:1000500045EA0141884208D9091903F1FF3680F0C9
:10006000E980884240F2E680023B43EA02420023F4
:1000700010461946BDE8F00F70478B424CD8B3FAD2
:1000800083F6002E4FD18B4202D3824200F2DD80F4
:10009000BDE8F00F0023012210461946704712B93F
:1000A0000124B4FBF2F4B4FA84F2002A40F0828016
:1000B000091B260CA7B20123B1FBF6F006FB1011B9
:1000C00007FB00F24FEA154C4CEA01418A4207D97E
:1000D000091900F1FF3C02D28A4200F2C880604652
:1000E000891AB1FBF6F206FB121107FB02F7ADB25B
:1000F00045EA0145AF4208D92C1902F1FF3180F0E1
:100100009B80A74240F29880023A42EA00421046A1
:100110001946BDE8F00F704700231A4610461946ED
:10012000BDE8F00F7047C6F1200522FA05F703FA83
:1001300006F421FA05F301FA06FB20FA05F53C4323
:100140004FEA1448B3FBF8FC08FB1C331FFA84F990
:1001500009FB0CFA45EA0B0B4FEA1B4545EA034342
:100160009A4502FA06F204D91B190CF1FF356FD338
:10017000AC46CAEB0303B3FBF8F508FB153309FBE8
:1001800005F91FFA8BFB4BEA0347B94504D93F1920
:1001900005F1FF3362D31D4645EA0C4CACFB02234C
:1001A000C9EB07079F424FF000054AD346D062468D
:1001B0002B465DE79440C2F1200921FA09FC9140E9
:1001C00020FA09F9260CBCFBF6F806FB18CCA7B2FE
:1001D00007FB08F349EA01094FEA194141EA0C4CCF
:1001E000634500FA02F509D91CEB040C08F1FF3253
:1001F0003BD2634539D9A8F10208A444C3EB0C0CE7
:10020000BCFBF6F306FB13C107FB03F21FFA89F9E7
:1002100049EA01418A4207D9091903F1FF3022D284
:100220008A4220D9023B2144891A43EA084343E722
:100230003A4605E7334618E70A4666E7B04090427B
:10024000B5D20CF1FF32002312E7334632460FE7F6
:100250009A458DD9ACF1020C23448AE7B9459AD965
:10026000023D274498E70346DEE79046C6E702389A
:10027000214435E773B55B4EFCF716FA00244FF4C2
:1002800080303470FCF72EFAFCF77CFB0128054621
:1002900025D11020FBF728FD2046FCF771FA2046F7
:1002A000FCF782FA2046FCF775FA4FF480304FF4E1
:1002B0008021FCF743FA2846FCF74AFA3920FCF77C
:1002C0004DFB0028FAD00120FBF7F6FC0120FCF7DB
:1002D00045FAFCF74DFA0428FBD1012333700420C2
:1002E0000121FCF7F9FA4FF48073ADF804300323D1
:1002F00001A98DF806303C4818238DF80730FBF72C
:1003000074FF0620FCF724FB01200146FCF7E4FA09
:100310004FF0C0500121FCF7EBFA4FF480414FF051
:100320000060FCF70DF9314D4FF44070FCF75EF8BA
:10033000F3F726FFF4F7A0FA01232B702C4A2D4B7C
:100340002D4913602D4A2E4C11602E4A1360F4F78C
:1003500079F8F8F7A9FAF8F789FAF7F7E5FEF3F76D
:10036000C3FF2078F7F754FFE078F8F787F8207894
:10037000F8F7ADF8E078F8F703FA2B780BB1F8F757
:10038000F5FDF9F78BF8F4F7EDF9FAF7CBFEF4F792
:1003900033FAF4F749FAD0F1010438BF0024F6F734
:1003A000CFFFF8F759FEF9F7B5FB174B4FF4806212
:1003B0005A61F7F7C7F8F9F7B9FBF8F74EFEF4F70B
:1003C0001BFAF4F73DFA0028F3D00CB1FAF7AAFEB5
:1003D000F9F764F80024F6F7B3FFF9F79BFBF8F799
:1003E00053FEE6E77C0F002000080140A80E002025
:1003F000C00E0020C18700089B8D0008880F0020D8
:10040000080000201C0F0020000C014000210A22DF
:1004100000F0ACB80F4B30B405461C6802E0D01AAF
:1004200016D1ABB115F8013BE21850781A4600F02E
:100430000300012808BF03F1200211F8013BE01876
:10044000407800F003000128E9D12033D01AE9D028
:1004500030BC70475C0500202DE9F00F424C82B0A3
:10046000D4F800C001900E4600E02646344614F849
:10047000015B0CEB0500407800F0080000F0FF0A7B
:100480000028F2D12D2D5BD02B2D04BF7578B41C24
:1004900033F010003CD09946BAF1000F0CBF6FF05A
:1004A000004B4FF0004BBBFBF9F8002709FB18BBD2
:1004B00038460CE0303DAB4219DD7E1C05D040458E
:1004C00023D820D009FB0050012714F8015B0CEB66
:1004D0000506767816F0040FECD116F0030606D068
:1004E000012E14BF57263726AD1BAB42E5DC7B1C23
:1004F00015D0BAF1000F21D10AB1EFB9116002B0E5
:10050000BDE8F00F70475D45DCDD4FF0FF37DCE7FD
:10051000302D1AD0002BBED10A239946BCE7019991
:10052000BAF1000F4FF022030CBF6FF000404FF004
:1005300000400B60002AE2D0611EDFE74042DBE7AB
:10054000B41C75784FF0010AA2E7207800F0DF00B4
:10055000582803D0002B9ED108239CE710236578F0
:100560009946023498E700BF5C05002030B4044C83
:100570000D46134601462A46206830BCFFF76CBF83
:10058000580500202DE9F0418AB004460D4600F0E0
:100590006BF8DFF8D080064698F900300F4601333B
:1005A0000BD02046294600F057FA30B120462946A4
:1005B00000220023FFF702F820B1304639460AB086
:1005C000BDE8F081234B98F800600890CDE9024522
:1005D000CDE90445019346BB1F4B4FF06042CDE986
:1005E00006232046294600220023FEF7BFFF70B1F4
:1005F00002239E42009322D0684600F055FAF0B1E3
:10060000089B0BBBDDE906010AB0BDE8F0810123C0
:10061000022E00930ED0684600F046FA50B10F4803
:1006200000F044FACDE90601EAE70D4B0022CDE9DE
:100630000623D6E700F040FA21230360EFE700F03D
:100640003BFA22230360DBE700F036FA089B0360E5
:10065000D8E700BFEC0D0108FFFFEFC7F00D010860
:100660000000F0FF600500202DE9F04FB1F5801F7C
:1006700087B002460B460F465BDA21F00046064380
:1006800000F0F5800029C0F2A4810022B24BFEF7F1
:1006900005FD0F460B46B14902468F426FF0350506
:1006A0004BDCC7F3130606F5152101F6647101F45E
:1006B000801484F07F5181F4401141EA0603104612
:1006C00019460022A64BFEF735FB4FEA2758B31C0C
:1006D000A8F2FF38C3F31303A844022B08EB145805
:1006E00082468B464FF000022EDC0023FEF73EFFD1
:1006F000002800F0C580B8F1000F00F0718140467D
:10070000FEF766FC80A3D3E9002306460F46FEF7FA
:10071000C5FC7FA3D3E9002304460D463046394685
:10072000FEF7BCFC02460B4620462946FEF704FBBA
:1007300007E08A4900258F42B3DD10461946FEF7CF
:10074000FBFA07B0BDE8F08F4FF08043FEF7F4FAF4
:1007500002460B4650465946FEF7CAFDCDE9020156
:100760004046FEF735FCCDE90401DDE90201024611
:100770000B46FEF793FC02460B46CDE90001FEF75F
:100780008DFC65A3D3E9002304460D46FEF786FCE5
:1007900063A3D3E90023FEF7CFFA22462B46FEF7E8
:1007A0007DFC61A3D3E90023FEF7C6FA22462B465F
:1007B000FEF774FC5EA3D3E90023FEF7BDFADDE982
:1007C0000023FEF76BFC5CA3D3E90023CDE9000115
:1007D00020462946FEF762FC59A3D3E90023FEF721
:1007E000ABFA22462B46FEF759FC57A3D3E9002368
:1007F000FEF7A2FA22462B46FEF750FC0B460246B5
:10080000DDE90001FEF798FAA6F5C223C6F5D72662
:10081000A3F27A4351361E43002E04460D4657DD9F
:100820000022504B50465946FEF738FC52465B4674
:10083000FEF734FC06460F46B8F1000F40F09680F4
:1008400022462B46FEF778FADDE90223FEF726FC66
:1008500002460B4630463946FEF76CFA02460B4616
:1008600050465946FEF766FA07B0BDE8F08F002201
:10087000002300203C49FEF73BFD07B0BDE8F08FA8
:1008800052465B4650465946FEF708FC30A3D3E972
:10089000002304460D4650465946FEF7FFFB02462C
:1008A0000B4600202F49FEF745FA02460B4620462C
:1008B0002946FEF7F3FB04460D46B8F1000F40F061
:1008C00092805046594622462B46FEF733FA38E7C7
:1008D000B8F1000F00F0AB800BA3D3E90023DDE9F2
:1008E0000401FEF7DBFB22462B4606460F46504628
:1008F0005946FEF71FFADDE90223FEF7CFFB044657
:100900000D46DDE904017CE00000E0FE422EE63FFA
:10091000763C7935EF39EA3D44523EDF12F1C23F71
:10092000DE03CB966446C73F599322942449D23FB5
:10093000935555555555E53F9FC678D0099AC33F05
:10094000AF788E1DC571CC3F04FA97999999D93F1C
:10095000555555555555D53F00005043FFFFEF7F86
:100960000000F03F0000E03F000050C336A3D3E991
:100970000023DDE90401FEF791FB2246804689460B
:100980002B4630463946FEF7D7F9DDE90223FEF75C
:1009900085FB2FA3D3E9002304460D46DDE90401BE
:1009A000FEF77CFB02460B4620462946FEF7C4F9BB
:1009B00002460B4630463946FEF7BCF952465B46C6
:1009C000FEF7B8F902460B4640464946FEF7B2F933
:1009D000B7E6FEF7AFF900220023FEF789FCB0E688
:1009E00000200021ADE64046FEF7F2FA16A3D3E957
:1009F000002380468946FEF751FB06460F464046D7
:100A0000494613A3D3E90023FEF748FB02460B46F1
:100A100020462946FEF78EF952465B46FEF78AF9D4
:100A200002460B4630463946FEF784F989E602460F
:100A30000B4650465946FEF77DF9DDE90223FEF7E5
:100A40002DFB0BE7AFF300800000E0FE422EE63FF7
:100A5000763C7935EF39EA3D31F0004310B408D0E7
:100A60000F4AA3F5801494420AD804205DF8044B81
:100A7000704700280CBF022003205DF8044B70472C
:100A8000B3F5801F01D20320F7E7064A934201D055
:100A90000020F2E7D0F1010038BF0020EDE700BFF1
:100AA000FFFFDF7F0000F07F00207047002001493A
:100AB000704700BF0000F87F014B1868704700BF07
:100AC00058050020F40100006400000001800808BF
:100AD00000000000006400000000000000000000B2
:100AE000C80000000000000000000000010003E852
:100AF0000000000000000003E80000000000020009
:100B0000FA060003000000000037060000000000A5
:100B10000000000032035400720069006E006100A2
:100B20006D006900630020005300740065007000D0
:100B300070006500720020004400650076006900C6
:100B400063006500200026035400720069006E00F7
:100B500061006D00690063004D006F007400690062
:100B60006F006E002000430074006C000403090451
:100B700009024300020100C0320904000001020220
:100B800001000524001001052401000104240202D3
:100B90000524060001070582030800FF090401007F
:100BA000020A000000070503024000000705810259
:100BB00040000012011001020000403C2A00010127
:100BC0002A01020301524F5200000106524F4C000D
:100BD0000002064D5354000003024D56500000041D
:100BE00007534150000005074741500000060353DA
:100BF00054415000070352534150000803534750DB
:100C00000000090747475000000A035354475000AB
:100C10000B0352534750000C0352465300000D0380
:100C200053494F00000E0747494F00000F0353413F
:100C30004300001D0753434F00001E0747434F006A
:100C4000001F0343434F0000200341434F00002790
:100C50000355463000004007554631000041075516
:100C600046320000420755463300004307554634DC
:100C7000000044075546350000450755463600003C
:100C800046075546370000470752554E000081057C
:100C900053544F5000800042494E00008B0000002A
:100CA0000000000000000000000102030401020334
:100CB000040607080902040608313136315631347A
:100CC00032004142530052454C00434F4F524400C2
:100CD00053544152540053544F50005354415455AF
:100CE000530000004300000000202020202020208E
:100CF00020202828282828202020202020202020CC
:100D000020202020202020202088101010101010DB
:100D10001010101010101010100404040404040427
:100D200004040410101010101010414141414141C1
:100D300001010101010101010101010101010101A3
:100D400001010101101010101010424242424242B3
:100D50000202020202020202020202020202020273
:100D6000020202021010101020000000000000001B
:100D70000000000000000000000000000000000073
:100D80000000000000000000000000000000000063
:100D90000000000000000000000000000000000053
:100DA0000000000000000000000000000000000043
:100DB0000000000000000000000000000000000033
:100DC0000000000000000000000000000000000023
:100DD0000000000000000000000000000000000013
:100DE0000000000000000000000000006C6F6700C1
:040DF00000000000FF
:080DF40050EFFF7F0100000039
:100DFC00B90C01080001000000010200000800000D
:100E0C0001000000020000000000000000000000D3
:100E1C0000000000000000000000000000000000C6
:100E2C0000000000000000000000000000000000B6
:100E3C00000000000000000000C2010000000800DB
:100E4C00458E0008098C0008098B00081D8B0008D2
:100E5C001F8B0008798B00089D8B0008E58C00081F
:100E6C00F18C0008FD8C0008000000004000000020
:100E7C00B30B010812000000700B010843000000C6
:100E8C006C0B010804000000460B01082600000052
:100E9C00140B010832000000140100201A0000009D
:100EAC000100000061E30008E58A000861E3000826
:100EBC0061E3000861E3000861E3000861E30008F6
:100ECC0061E30008FD8A00080401000061E30008EA
:100EDC0061E30008DD8B000861E3000861E30008B2
:100EEC0061E3000861E30008D98A000861E30008A7
:100EFC0061E3000861E3000861E3000861E30008B6
:100F0C0061E300081A0354004D00430053005400E1
:100F1C004500500000000000000000000000000030
:100F2C00000000001C04002084040020EC040020BD
:100F3C0000000000000000000000000000000000A5
:100F4C000000000000000000000000000000000095
:100F5C0000000000E40C010800000000000000008C
:100F6C000000000000000000000000000000000075
:100F7C000000000000000000000000000000000065
:100F8C000000000000000000000000000000000055
:100F9C000000000000000000000000000000000045
:100FAC000000000000000000000000000000000035
:100FBC000000000000000000000000000000000025
:100FCC000000000000000000010000000000000014
:100FDC000E33CDAB34126DE6ECDE05000B000000D9
:100FEC0000000000000000000000000000000000F5
:100FFC0000000000000000000000000000000000E5
:10100C0000000000000000000000000000000000D4
:10101C0000000000000000000000000000000000C4
:10134C00000000000000000030010020E80C010843
:04135C00010000008C
:04000005080041109E
:00000001FF
